:100000000C9418180C9449180C9449180C9449181D
:100010000C9449180C9449180C9449180C944918DC
:100020000C9449180C9449180C9449180C944918CC
:100030000C9449180C94625D0C9449180C9449185E
:100040000C9449180C94F1C00C9449180C9449185C
:100050000C9449180C9449180C94185F0C943A9914
:100060000C9449180C9482A10C94F3430C944918F5
:100070000C9449180C9449180C9449180C9449187C
:100080000C9449180C9449180C9449180C9449186C
:100090000C9449180C9449180C9449180C9449185C
:1000A0000C9449180C9449180C9449180C9449184C
:1000B0000C9449180C9449180C9449180C9449183C
:1000C0000C9449180C9449180C9449180C9449182C
:1000D0000C9449180C9449180C9471510C94325199
:1000E0000C944918C71AE41A151B321B471B711BC5
:1000F000DE1B441CED1C862190213F2267226B22CF
:10010000CA22B527DF222B2352237B23A723FE23DA
:100110000F242324342445245624B527C026B5278C
:10012000CB263B2741276127B4A1BAA1CBA1D6A1F9
:10013000DEA1F3A1E2A1F3A1E6A1EAA1F3A1F0A15E
:10014000ECD9EFD9DED9E2D9E8D926DAF3D9F7D953
:10015000FDD901DA05DA0BDA0FDA13DA26DA19DA61
:100160001DDA21DAC7DDCCDDD1DDDBDDE5DD5EDEEC
:10017000EFDDF7DDFFDD09DE13DE1DDE2CDE36DE12
:100180005EDE40DE4ADE54DE084AD73B3BCE016EDF
:1001900084BCBFFDC12F3D6C74319ABD56833DDADE
:1001A0003D00C77F11BED9E4BB4C3E916BAAAABEED
:1001B000000000803F05A84CCDB2D44EB93836A916
:1001C000020C50B9918688083CA6AAAA2ABE000053
:1001D00000803F004E414E494E495459494E46CD4C
:1001E000CCCC3D0AD7233C17B7D13877CC2B3295EE
:1001F00095E6241FB14F0A000020410000C84200CC
:10020000401C4620BCBE4CCA1B0E5AAEC59D744352
:10021000616E6E6F7420656E7465722073756264B2
:1002200069723A20004D3630300053706563696161
:100230006C204D656E753A2046696C616D656E7413
:100240004368616E676520526573756D650A00537A
:1002500070656369616C204D656E753A2046696C06
:10026000616D656E744368616E676520506175737A
:10027000650A004739310A4731205A2D302E310A9C
:10028000473930005370656369616C204D656E7548
:100290003A205A20446F776E20302E310A004739B9
:1002A000310A4731205A2D302E30320A473930007A
:1002B0005370656369616C204D656E753A205A20F4
:1002C000446F776E20302E30320A004739310A47AA
:1002D00031205A2B302E30320A47393000537065A6
:1002E0006369616C204D656E753A205A2055702007
:1002F000302E30320A004739310A4731205A2B302C
:100300002E310A473930005370656369616C204DA6
:10031000656E753A205A20557020302E310A0047FC
:100320003239205332005370656369616C204D652A
:100330006E753A204E657874204D65736820506F55
:10034000696E740A00473239205331005370656377
:1003500069616C204D656E753A205374617274202A
:100360004D657368204C6576656C696E670A004D53
:1003700031343020533630005370656369616C202E
:100380004D656E753A2050726568656174204265EE
:10039000640A004D353032005370656369616C202A
:1003A0004D656E753A204C6F616420465720446558
:1003B0006661756C74730A004D353030005370659A
:1003C0006369616C204D656E753A205361766520D6
:1003D000454550524F4D0A004D33303320452D31A5
:1003E0002053363020433620553100537065636901
:1003F000616C204D656E753A204175746F2054759F
:100400006E6520486F74626564205069640A004D0F
:1004100031303620533230340A4D333033204530BA
:10042000205332313020433135205531005370652F
:100430006369616C204D656E753A204175746F205B
:1004400054756E6520486F74656E64205049440A87
:10045000004D313038004D313038004D3234004DD0
:100460003234003C5370656369616C5F4D656E7535
:100470003E003C5370656369616C5F4D656E753E0F
:10048000002F002F002F002F2E2E0A002F2E2E00BF
:100490002F2E2E003C5370656369616C5F4D656E55
:1004A000753E0A003C5370656369616C204D656E52
:1004B000753E003C5370656369616C204D656E75D7
:1004C0003E003C46696C616D656E744368616E67A1
:1004D0006520526573756D653E003C46696C616DC3
:1004E000656E744368616E676520526573756D65EE
:1004F0003E003C46696C616D656E744368616E6771
:10050000652050617573653E003C46696C616D65A0
:100510006E744368616E67652050617573653E0057
:100520003C4C6F61642046572044656661756C746D
:10053000733E003C4C6F6164204657204465666101
:10054000756C74733E003C4175746F2054756E6514
:1005500020486F74626564205049443E003C4175F8
:10056000746F2054756E6520486F74626564205006
:1005700049443E003C4175746F2054756E652048B7
:100580006F74656E64205049443E003C4175746F41
:100590002054756E6520486F74656E642050494420
:1005A0003E003C457869743E003C457869743E00E5
:1005B0003C5361766520454550524F4D3E003C53BB
:1005C00061766520454550524F4D3E003C4E657862
:1005D00074204D65736820506F696E743E003C4E08
:1005E000657874204D65736820506F696E743E00A5
:1005F0003C5374617274204D657368204C65766558
:100600006C696E673E003C5374617274204D657373
:1006100068204C6576656C696E673E003C5072657B
:1006200068656174206265643E003C50726568656F
:100630006174206265643E003C5A20446F776E20EE
:10064000302E313E003C5A20446F776E20302E31E0
:100650003E003C5A20446F776E20302E30323E00F0
:100660003C5A20446F776E20302E30323E003C5A88
:1006700020557020302E30323E003C5A20557020DC
:10068000302E30323E003C5A20557020302E313E04
:10069000003C5A20557020302E313E005631313604
:1006A000004A333320004D3530300A4D343230208B
:1006B00053310A4731205A313020463234300A470C
:1006C00031205830205930204636303030004A3200
:1006D00032004A3232004731205A35204632343017
:1006E0000A473120583139302059323020463630CF
:1006F00030300A4731205A302046323430004731FA
:10070000205A3520463234300A47312058313930AA
:1007100020593139302046363030300A4731205A9E
:10072000302046323430004731205A3520463234AA
:10073000300A47312058313930205932302046367E
:100740003030300A4731205A3020463234300047AA
:1007500039310A4731205A313020463234300A4785
:1007600039300A4732380A4732390A47312058327D
:1007700030205932302046363030300A4731205A46
:10078000302046323430004A3032004A313200479D
:1007900031205A3130004F4B004731205A31300060
:1007A000473930004731204525694635303000470C
:1007B0003120452D302E3146256900473120453006
:1007C0002E31462569004731205A256946256900A2
:1007D0004731205A2D302E31462569004731205AA5
:1007E000302E314625690047312059256946256953
:1007F00000473120592D302E3146256900473120E0
:1008000059302E3146256900473120582569462543
:100810006900473120582D302E3146256900473177
:100820002058302E3146256900473931004732388B
:1008300000473238205A00473238205900473238B2
:100840002058004132305620004731205A313000C4
:100850004A3034004A3231004A3230004B494C4C65
:1008600045442E20004A3136004A303400454E447B
:1008700000464E20004A3032003939393A39393988
:10088000004D0048004137562000413656202D2D9E
:100890002D004A30320041365620005A3A20005985
:1008A0003A2000583A200041355600413456200085
:1008B000413356200041325620004131562000413C
:1008C000305620004D3237004D3834004739310A58
:1008D000473120452D312046313830300A473930F4
:1008E000004A3136004D313235204C32004A313821
:1008F000004A3134004A3030004A3031004A313049
:1009000000434F4D4D554E49434154494F4E0044CD
:10091000525952554E004552524F525300494E467D
:100920004F004543484F0047322F473320626164F0
:1009300020706172616D65746572730A00206F6664
:1009400020004D424C2047323920706F696E742070
:1009500000290A0059206F7574206F662072616E3D
:1009600067652028312D00290A0058206F757420F2
:100970006F662072616E67652028312D004D6573AA
:10098000682070726F62696E6720646F6E652E0AF0
:10099000005374617274206D6573682070726F62A9
:1009A000696E672077697468202247323920533195
:1009B000222066697273742E0A004732380A473261
:1009C000392053320053746174653A20004D6573C9
:1009D0006820626564206C6576656C696E67206866
:1009E0006173206E6F20646174612E0A0053206F62
:1009F0007574206F662072616E67652028302D3512
:100A0000292E0A004D65736820706F696E7420632B
:100A1000616E6E6F74206265207265736F6C7665AF
:100A2000640A00456E642066696C65206C697374A5
:100A30000A00426567696E2066696C65206C69739F
:100A4000740A004D31323500286E6F2066696C657E
:100A500029005344207072696E74696E6720627950
:100A6000746520004E6F74205344207072696E7458
:100A7000696E670A0043757272656E742066696CF0
:100A8000653A200046696C652064656C6574656430
:100A90003A0044656C6574696F6E206661696C65C7
:100AA000642C2046696C653A20005072696E74208F
:100AB00074696D653A20006F6E2E0A006F66662EAF
:100AC0000A00473236204465627567200022091DFE
:100AD0000916090F0901096F66660044454255472A
:100AE0003A004D3131332053006F6B002C20002C25
:100AF0002000544845524D414C5F50524F5445439D
:100B000054494F4E004155544F5245504F52545F37
:100B100053445F53544154555300454D4552474546
:100B20004E43595F50415253455200434153455F34
:100B30004C494748545F4252494748544E455353E5
:100B400000544F47474C455F4C4947485453005366
:100B50004F4654574152455F504F574552004255FA
:100B6000494C445F50455243454E54004C45564510
:100B70004C494E475F44415441005A5F50524F42E6
:100B800045004155544F4C4556454C005052494E36
:100B9000545F4A4F420050524F4752455353004111
:100BA00055544F5245504F52545F54454D50005686
:100BB0004F4C554D455452494300454550524F4DB9
:100BC0000053455249414C5F584F4E5F584F46467F
:100BD000004649524D574152455F4E414D453A4DB1
:100BE00061726C696E20312E312E3920284769746C
:100BF0006875622C20646176696472616D69726FD8
:100C000029204D41524C494E2D4149334D5F5645A7
:100C10005253494F4E3A76312E342E3620534F558B
:100C20005243455F434F44455F55524C3A68747494
:100C300070733A2F2F6769746875622E636F6D2F1A
:100C4000646176696472616D69726F2F4D61726C57
:100C5000696E2D4149334D2050524F544F434F4CF4
:100C60005F56455253494F4E3A312E30204D414345
:100C700048494E455F545950453A416E7963756213
:100C80006963206933204D6567612045585452558A
:100C90004445525F434F554E543A312055554944CF
:100CA0003A63656465326132662D343161322D34C8
:100CB0003734382D396231322D633535633632663B
:100CC00033363766660A002F2F200020540020524A
:100CD00000416363656C65726174696F6E3A2050A0
:100CE000005741524E494E4721204C6F77205A20E1
:100CF0004A65726B206D6179206C65616420746F48
:100D000020756E77616E74656420706175736573AC
:100D10002E0A00546F6F206661722066726F6D201C
:100D20007265666572656E636520706F696E740AC0
:100D30000020466C6F773A20000001363726032BDF
:100D4000FFFFFF3C3D382AFFFFFFFF2E303E12FF22
:100D5000FFFFFFFFFFFF0809FF2C071A1C18FFFF0A
:100D6000FF08440A2C4324221E20643A0020693ADA
:100D70000020703A00496E76616C69642065787471
:100D800072756465720A0043290A0061626C6564C9
:100D900020286D696E2074656D702000436F6C644F
:100DA0002065787472756465732061726520002017
:100DB000643A0020693A0020703A004E6F20636167
:100DC0007365206C696768740A00454550524F4D41
:100DD000204F4B0A00205A004475616C20456E6418
:100DE00073746F702041646A7573746D656E7420DE
:100DF000286D6D293A20003F4B2076616C75652087
:100E00006F7574206F662072616E67652028302DC3
:100E10003130292E0A00416476616E6365204B3DB6
:100E200000416374697665204578747275646572F3
:100E30003A2000496E76616C696420657874727539
:100E40006465720A00696E206D6F76655F746F2845
:100E50002920666565645F76616C756520666F72D2
:100E60002058593A002C2065793D0029202D3E203C
:100E70002865783D002C2073793D0020436F6E6E0D
:100E8000656374696E67207769746820766572742B
:100E90006963616C206C696E65202873783D002C55
:100EA0002065793D0029202D3E202865783D002CC5
:100EB0002073793D0020436F6E6E656374696E67C1
:100EC000207769746820686F72697A6F6E74616CDC
:100ED000206C696E65202873783D003F5370656310
:100EE000696669656420582C5920636F6F72646964
:100EF0006E617465206F7574206F6620626F756E09
:100F000064732E0A003F285229657065617420764B
:100F1000616C7565206E6F7420706C6175736962A9
:100F20006C653B206D757374206265206174206C64
:100F30006561737420312E0A003F2852296570655F
:100F40006174206D757374206265207370656369C8
:100F500066696564207768656E206E6F74207573AE
:100F6000696E6720616E204C43442E0A003F537027
:100F700065636966696564206E6F7A7A6C65207452
:100F8000656D7065726174757265206E6F74207026
:100F90006C61757369626C652E0A003F53706563FE
:100FA00069666965642066696C616D656E7420733D
:100FB000697A65206E6F7420706C61757369626CFC
:100FC000652E0A003F537065636966696564207029
:100FD00072696D65206C656E677468206E6F742031
:100FE000706C61757369626C652E0A003F5072699E
:100FF0006D65206C656E677468206D757374206212
:101000006520737065636966696564207768656EDD
:10101000206E6F74207573696E6720616E204C437B
:10102000442E0A003F537065636966696564206EEB
:101030006F7A7A6C652073697A65206E6F742070A0
:101040006C61757369626C652E0A003F496E76614A
:101050006C69642052657472616374696F6E2F5598
:101060006E72657472616374696F6E207261746907
:101070006F2E204D757374206265207769746869DE
:101080006E20356D6D2E0A0020556E72657472618A
:101090006374696F6E20616D6F756E742061757415
:1010A0006F6D61746963616C6C7920736574207411
:1010B0006F20003F53706563696669656420556EF3
:1010C00072657472616374696F6E206C656E6774AB
:1010D00068206E6F7420706C61757369626C652E28
:1010E0000A003F556E72657472616374696F6E2099
:1010F0006C656E677468206D75737420626520730B
:1011000070656369666965642E0A003F53706563A4
:1011100069666965642052657472616374696F6E93
:10112000206C656E677468206E6F7420706C6175DA
:101130007369626C652E0A003F5265747261637454
:10114000696F6E206C656E677468206D75737420AE
:101150006265207370656369666965642E0A003F85
:10116000537065636966696564206C617965722096
:10117000686569676874206E6F7420706C61757340
:1011800069626C652E0A003F537065636966696524
:1011900064206265642074656D7065726174757237
:1011A00065206E6F7420706C61757369626C652068
:1011B0002834302D31343043292E0A00473236206E
:1011C000636F6D6D616E6420737461727465642EFB
:1011D0002057616974696E6720666F722068656167
:1011E0007465722873292E0A0024F4D43050C38EFB
:1011F00020C2A24017828B7011127A910D816CD996
:101200000AA861E108C7586607615143061E4B5D95
:1012100005C145A7041A411104093D9803713931EC
:10122000034036DB0265339102D4305402802E1D18
:1012300002632CEE01752AC501B028A00110278198
:10124000018F2564012B244B01E0223401AC211FC6
:10125000018D200D01801FFC00841EED00971DDF15
:1012600000B81CD200E61BC600201BBC00641AB2EA
:1012700000B219A8000A19A0006A189900D11791A4
:101280000040178B00B516840031167E00B3157927
:10129000003A157300C7146F0058146A00EE136605
:1012A000008813630025135E00C7125B006C1257A1
:1012B0000015125400C111510070114F0021114B43
:1012C00000D61049008D104700461044000210421D
:1012D00000C00F4000800F3E00420F3C00060F3B55
:1012E00000CB0E3800930E37005C0E3500270E340D
:1012F00000F30D3200C10D3100900D3000600D2E55
:1013000000320D2D00050D2C00D90C2B00AE0C2940
:1013100000850C29005C0C2700350C27000E0C26DC
:1013200000E80B2400C40B2400A00B23007D0B233A
:10133000005A0B2100390B2100180B2000F80A1F5E
:1013400000D90A1E00BB0A1E009D0A1D00800A1D4E
:1013500000630A1C00470A1B002C0A1B00110A1A12
:1013600000F7091A00DD091900C4091900AB0919B1
:1013700000920917007B091800630917004C091631
:101380000036091600200916000A091500F508158F
:1013900000E0081400CC081400B8081400A40814D5
:1013A00000900813007D0812006B08130058081203
:1013B0000046081200340811002308110012081119
:1013C0000001081100F0071000E0071000D007101E
:1013D00000C0071000B0070F00A107100091070E12
:1013E0000083070F0074070F0065070E0057070EF4
:1013F0000049070E003B070D002E070E0020070DC9
:101400000013070D0006070D00F9060C00ED060D90
:1014100000E0060C00D4060C00C8060C00BC060C4C
:1014200000B0060C00A4060B0099060C008D060BFC
:101430000082060B0077060B006C060B0061060AA3
:101440000057060B004C060A0042060A0038060A3E
:10145000002E060A0024060A001A060A00100609D1
:101460000007060A00FD050900F4050900EB05095F
:1014700000E2050900D9050900D0050900C70509E2
:1014800000BE050900B5050800AD050800A5050961
:10149000009C050800940508008C050800840508D8
:1014A000007C050800740508006C05070065050848
:1014B000005D050700560508004E050700470507B3
:1014C000004005080038050700310507002A050718
:1014D00000230507001C050600160507000F050779
:1014E000000805060002050700FB040600F50407D6
:1014F00000EE040600E8040600E2040700DB040630
:1015000000D5040600CF040600C9040600C3040683
:1015100000BD040600B7040600B1040500AC0406D3
:1015200000A6040600A00405009B0406009504051F
:1015300000900406008A0405008504050080040666
:10154000007A04050075040500700405006B0405AD
:101550000066040500610405005C040500570405ED
:1015600000520405004D040500480405004304052D
:10157000003E0404003A040500350405003004046C
:10158000002C04050027040400230405001E0404A5
:10159000001A04040016040500110404000D0404DC
:1015A00000090405000404040000040400FC030412
:1015B00000F8030400F4030400F0030400EC030447
:1015C00000E8030400E4030400E0030400DC030477
:1015D00000D8030400D4030400D0030400CC0304A7
:1015E00000C8030300C503030024F404D9201BC46E
:1015F0000C5C0E9804C4095F0265077101F405F9DB
:1016000000FB04B30048048700C103690058035578
:101610000003034500BE023A008402310053022A4F
:10162000002902250004022000E4011C00C8011961
:1016300000AF01170098011400840113007101101C
:10164000006101100051010E0043010D0036010B35
:10165000002B010B0020010B00150109000C0109F2
:101660000003010800FB000800F3000800EB00077E
:1016700000E4000600DE000600D8000600D20006E6
:1016800000CC000500C7000500C2000500BD000435
:1016900000B9000400B5000400B1000400AD00046E
:1016A00000A9000400A5000300A20003009F00049D
:1016B000009B0003009800030095000200930003C4
:1016C00000900003008D0002008B000300880002E0
:1016D000008600020084000300810002007F0002F7
:1016E000007D0002007B000200790002007700010B
:1016F0000076000200740002007200010071000216
:10170000006F0002006D0001006C0002006A000121
:101710000069000200670001006600010065000129
:10172000006400020062000100610001006000012D
:10173000005F0002005D0001005C0001005B000131
:10174000005A000100590001005800010057000133
:101750000056000100550001005400010053000034
:10176000005300010052000100510001005000012F
:10177000004F0001004E0000004E0001004D00012E
:10178000004C0001004B0000004B0001004A00012A
:101790000049000100480000004800010047000126
:1017A0000046000000460001004500000045000121
:1017B000004400010043000000430001004200001B
:1017C0000042000100410000004100010040000112
:1017D000003F0000003F0001003E0000003E00010D
:1017E000003D0000003D0001003C0000003C000006
:1017F000003C0001003B0000003B0001003A0000FB
:10180000003A0001003900000039000100380000F2
:1018100000380000003800010037000000370001E8
:1018200000360000003600000036000100350000E0
:1018300000350000003500010034000000340000D5
:1018400000340001003300000033000000330001C9
:1018500000320000003200000032000100310000C0
:1018600000310000003100010030000000300000B5
:1018700000300001002F0000002F0000002F0000AA
:10188000002F0001002E0000002E0000002E00019D
:10189000002D0000002D0000002D0000002D000193
:1018A000002C0000002C0000002C0000002C000187
:1018B000002B0000002B0000002B0000002B00017B
:1018C000002A0000002A0000002A0000002A00016F
:1018D0000029000000290000002900000029000064
:1018E0000029000100280000002800000028000056
:1018F0000028000000280001002700000027000049
:10190000002700000027000000270001002600003B
:10191000002600000026000000260000002600012E
:101920000025000000250000002500000025000023
:101930000025000000250001002400000024000014
:101940000024000000240000002400010023000007
:1019500000230000002300000023000000230000FB
:1019600000230000002300010022000000220000EC
:1019700000220000002200000022000000220001DE
:1019800000210000002100000021000000210000D3
:1019900000210000002100000021000100200000C3
:1019A00000200000002000000020000000200000B7
:1019B000002000000020000000200001001F0000A7
:1019C000001F0000001F0000001F0000001F00009B
:1019D000001F0000001F0001001E0000001E00008C
:1019E000001E0000001E000000232C0000B8220092
:1019F00000561800003A0F0000B8080000B10400BB
:101A000000710200003E0100001000C90210012C0C
:101A1000014001220170011801B0010E01F0010422
:101A2000015002FA00B002F0003003E600D003DCFF
:101A3000009004D2007005C800A006BE000008B4E3
:101A400000B009AA00D00BA000600E960060118CB7
:101A5000000015820020197800C01D6E00A02264CD
:101A600000B0275A00902C500000314600E0343C72
:101A70000010383200903A2800603C1E00A03D144F
:101A800000803E0A00203F00002CFFFFFFFFFF0008
:101A900001010101016265640A002C2073797374ED
:101AA000656D2073746F7070656421204865617482
:101AB00065725F49443A200042656420686561743C
:101AC000696E67206661696C656400486561746968
:101AD0006E67206661696C65640045312048656108
:101AE00074696E67206661696C656400486561743D
:101AF000696E67206661696C6564004B494C4C45B2
:101B0000442E200070012C0190012701B001220118
:101B1000C0011D01F00118011002130130020E0175
:101B20006002090190020401C002FF000003FA00F4
:101B30004003F5008003F000D003EB002004E60032
:101B40007004E100E004DC004005D700C005D200CD
:101B50004006CD00D006C8008007C3003008BE0094
:101B6000F008B900C009B400B00AAF00B00BAA0079
:101B7000D00CA500000EA000500F9B00C0109600D6
:101B80005012910000148C00C0158700B01782001D
:101B9000B0197D00D01B7800001E730040206E003D
:101BA00090226900F024640040275F0090295A00C9
:101BB000E02B5500102E500020304B001032460014
:101BC000E033410090353C00103737007038320068
:101BD000A0392D00B03A2800A03B2300603C1E0035
:101BE000103D1900903D1400103E0F00703E0A0099
:101BF000C03E0500003F0000403FFBFF803FF6FF76
:101C0000C03FF1FF453120544845524D414C2052D0
:101C1000554E415741590042454420544845524D84
:101C2000414C2052554E4157415900546865726DE0
:101C3000616C2052756E6177617900453120457283
:101C4000723A204D415854454D50004572723A2029
:101C50004D415854454D5020424544004D41585443
:101C6000454D50207472696767657265640045313F
:101C7000204572723A204D494E54454D50004572F0
:101C8000723A204D494E54454D5020424544004D36
:101C9000494E54454D50207472696767657265649A
:101CA000004D383420582059205A204500202F005C
:101CB0002042403A0020403A00024B642000236456
:101CC0006566696E652044454641554C545F004B3E
:101CD00069200023646566696E6520444546415568
:101CE0004C545F004B70200023646566696E65206C
:101CF00044454641554C545F005049442041757459
:101D00006F74756E652066696E69736865642120FD
:101D100050757420746865206C617374204B702C4E
:101D2000204B6920616E64204B6420636F6E737476
:101D3000616E74732066726F6D2062656C6F7720C0
:101D4000696E746F20436F6E66696775726174693E
:101D50006F6E2E680A00504944204175746F747587
:101D60006E65206661696C6564212074696D656FBC
:101D700075740A00453120544845524D414C20525B
:101D8000554E415741590042454420544845524D13
:101D9000414C2052554E4157415900546865726D6F
:101DA000616C2052756E617761790045312048651C
:101DB0006174696E67206661696C65640042656480
:101DC0002068656174696E67206661696C6564008E
:101DD00048656174696E67206661696C656400506E
:101DE0004944204175746F74756E65206661696C35
:101DF0006564212054656D7065726174757265202B
:101E0000746F6F20686967680A00204B643A20008D
:101E1000204B693A2000204B703A20000A20436C86
:101E2000617373696320504944200A002054753A55
:101E30002000204B753A2000206D61783A20002068
:101E40006D696E3A200020643A2000206269617357
:101E50003A2000504944204175746F74756E6520B6
:101E60006661696C6564212054656D70657261748A
:101E700075726520746F6F20686967680A00504941
:101E800044204175746F74756E652073746172744B
:101E90000A00504944204175746F74756E65206660
:101EA00061696C6564212042616420657874727593
:101EB000646572206E756D6265720A004F66660A0F
:101EC0000046616465204865696768742000426562
:101ED00064204C6576656C696E6720004661696CAC
:101EE000656420746F20656E61626C652042656474
:101EF000204C6576656C696E670A004D65736820D5
:101F0000426564204C6576656C20646174613A0AB0
:101F1000004D65736820706F696E742063616E6E2A
:101F20006F74206265207265736F6C7665640A0059
:101F30004D34323120696E636F7272656374207044
:101F40006172616D657465722075736167650A0001
:101F5000496E736572742066696C616D656E74207C
:101F6000616E642073656E64204D3130380A005311
:101F7000656E64204D31303820746F20686561745F
:101F8000206E6F7A7A6C650A00496E7365727420F0
:101F900066696C616D656E7420616E642070726537
:101FA000737320627574746F6E20286F72204D31C8
:101FB0003038290A004D38383820636F6F6C646FF1
:101FC000776E20726F7574696E6520646F6E650A36
:101FD000004D383400546172676574206E6F742050
:101FE000726561636865642C207175657565642030
:101FF000616E206172630A00556C74726162617374
:102000006520636F6F6C646F776E20737461727498
:1020100065640A00486F6D696E67206661696C656A
:102020006400206E6F7420656E74657265642E0A9C
:102030000050726F7465637465642050696E0A00A5
:1020400046696C616D656E7420757365643A200035
:1020500053746174733A20002C204C6F6E67657363
:1020600074206A6F623A2000546F74616C20746946
:102070006D653A200053746174733A20002C204639
:1020800061696C65643A20002C2046696E6973684A
:1020900065643A20005072696E74733A200053747C
:1020A0006174733A20004A3036004A3034004A30B6
:1020B000370020573A004A3038004A30390020575C
:1020C0003A00205A3A0020593A0020436F756E7446
:1020D00020583A0020453A00205A3A0020593A0048
:1020E000583A003A004361703A00205A00205900E3
:1020F000580020204D61783A2000205A00205900D5
:10210000580020204D696E3A20004F6E20004F6627
:102110006600536F667420656E6473746F70733AF3
:10212000200020746F6F206C6F6E6720657874726A
:102130007573696F6E2070726576656E7465640A7A
:102140000020636F6C6420657874727573696F6EBC
:102150002070726576656E7465640A00454550525C
:102160004F4D206461746173697A65206572726F86
:10217000722E0A00290A002062797465733B20637D
:102180007263200053657474696E67732053746FB3
:10219000726564202800290A002062797465733B07
:1021A0002063726320002073746F7265642073650E
:1021B0007474696E6773207265747269657665649C
:1021C000202800202863616C63756C617465642944
:1021D000210A0020213D2000454550524F4D20430B
:1021E0005243206D69736D61746368202D202873DC
:1021F000746F7265642920002053697A653A200063
:10220000496E6465783A2000204D61726C696E3DBC
:10221000563535290A0028454550524F4D3D004559
:102220004550524F4D2076657273696F6E206D690F
:10223000736D6174636820004A3135004A313200A1
:102240004A3137002020506C616E6E6572427566AF
:1022500066657242797465733A200020467265653E
:10226000204D656D6F72793A2000436F6D70696C17
:1022700065643A2041707220203420323031390AAE
:1022800000207C20417574686F723A202864617662
:10229000696472616D69726F290A00323031392DBB
:1022A00030342D303300204C6173742055706461DC
:1022B0007465643A200076312E342E360A004D6162
:1022C000726C696E2D4149334D00312E312E390A21
:1022D000004D61726C696E0020536F667477617295
:1022E000652052657365740A0020576174636864E1
:1022F0006F672052657365740A002042726F776EB3
:10230000206F75742052657365740A0020457874D7
:1023100065726E616C2052657365740A00506F7748
:10232000657255700A0073746172740A004D32341C
:10233000004D3233202573006175746F25692E6757
:10234000006572726F722077726974696E672074AB
:102350006F2066696C650A00205A3A0020593A00DD
:1023600020583A00656E6473746F707320686974E6
:102370003A2000446F6E6520736176696E6720664F
:10238000696C652E0A004D32390025697300256994
:102390006D20256973002569682025696D202569F0
:1023A0007300256964202569682025696D202569E9
:1023B00073002569792025696420256968202569CD
:1023C0006D2025697300656E7175657565696E6749
:1023D0002022005072696E7465722073746F707081
:1023E00065642064756520746F206572726F727306
:1023F0002E2046697820746865206572726F72209D
:10240000616E6420757365204D39393920746F20F1
:10241000726573746172742E202854656D706572D4
:1024200061747572652069732072657365742E20FE
:1024300053657420697420616674657220726573D7
:1024400074617274696E67290A004E6F2043686573
:10245000636B73756D2077697468206C696E652095
:102460006E756D6265722C204C617374204C696EC0
:10247000653A20004E6F20436865636B73756D206D
:1024800077697468206C696E65206E756D6265721F
:102490002C204C617374204C696E653A200063688F
:1024A00065636B73756D206D69736D617463682C02
:1024B000204C617374204C696E653A20004C696E43
:1024C00065204E756D626572206973206E6F742091
:1024D0004C617374204C696E65204E756D62657237
:1024E0002B312C204C617374204C696E653A2000AE
:1024F0004D313130004D33310053442072656164F9
:10250000206572726F720A00446F6E652070726986
:102510006E74696E672066696C650A0020496E7684
:10252000616C69642065787472756465722000005E
:1025300000A0C000000000000000000000574300A1
:1025400000574300004D43627573793A20706175FE
:1025500073656420666F7220696E7075740A00621C
:102560007573793A2070617573656420666F7220A7
:10257000757365720A00627573793A2070726F63C1
:10258000657373696E670A004A3135004B494C4CDC
:1025900045442E20004B494C4C20636175736564A3
:1025A000206279204B494C4C20627574746F6E2FF9
:1025B00070696E0A004B494C4C45442E20004B4933
:1025C0004C4C2063617573656420627920746F6F71
:1025D000206D75636820696E616374697665207427
:1025E000696D65202D2063757272656E7420636F4E
:1025F0006D6D616E643A20004A3131005072696E2F
:102600007465722068616C7465642E206B696C6CF3
:1026100028292063616C6C6564210A000000A0C059
:102620000000000000000000000048420000484296
:1026300000008040000000005761726E696E673ACA
:1026400020486F6D696E672042756D702044697611
:1026500069736F72203C20310A000202040000A05E
:10266000400000A0400000004000005C4300005714
:102670004300004D43FFFFFF486F74656E64207494
:102680006F6F20636F6C640A00486F74656E64201E
:10269000746F6F20636F6C640A007C3C3E5E2B3D60
:1026A0003F2F5B5D3B2C2A225C0043616E6E6F7492
:1026B000206F70656E2073756264697220005344E8
:1026C0002063617264206F6B0A006F70656E526FD9
:1026D0006F74206661696C65640A00766F6C756D55
:1026E000652E696E6974206661696C65640A0045CF
:1026F00072726F723A00534420696E697420666189
:10270000696C0A006563686F3A00526573656E64B0
:102710003A20006F6B0020746F6F206C6F6E672023
:10272000657874727573696F6E2070726576656E08
:102730007465640A0020636F6C6420657874727538
:1027400073696F6E2070726576656E7465640A00D9
:10275000FFFDFCFAF8F6F4F2F0EEECEAE9E7E5E367
:10276000E1E0DEDCDAD9D7D5D4D2D0CFCDCBCAC820
:10277000C7C5C3C2C0BFBDBCBAB9B7B6B4B3B2B0A7
:10278000AFADACAAA9A8A6A5A4A2A1A09E9D9C9A03
:1027900099989795949392908F8E8D8B8A8988873C
:1027A0008684838281807F7E7D7B7A797877767557
:1027B00074737271706F6E6D6C6B6A696867666551
:1027C00064636261605F5E5D5C5B5A59585857563E
:1027D000555453525150504F4E4D4C4B4A4A494814
:1027E000474646454443424241403F3E3E3D3C3BD6
:1027F0003B3A393838373635353433323231303088
:102800002F2E2E2D2C2B2B2A29292827272625252C
:1028100024232322212120201F1E1E1D1C1C1B1BC4
:102820001A19191818171616151514131312121150
:1028300011100F0F0E0E0D0D0C0C0B0A0A090908D2
:102840000807070606050504040303020201000049
:10285000545249474745524544006F70656E003AEF
:1028600020007A325F6D696E007A5F6D696E007963
:102870005F6D696E00785F6D696E005265706F7292
:1028800074696E6720656E6473746F702073746111
:102890007475730A000A4D65617375726564207002
:1028A0006F696E74733A0A005A206F6666736574B6
:1028B0003A20004E756D20582C593A20352C350A97
:1028C0000000000001000000010000800055555587
:1028D000000000400033333300AAAA2A00499224A2
:1028E0000000002000C7711C0099991900D14517FC
:1028F00000555515003BB113002449120011111168
:1029000000000010000F0F0F00E3380E0043790D98
:1029100000CCCC0C00C3300C00E8A20B0064210BEF
:1029200000AAAA0A00703D0A009DD80900427B094E
:102930000092240900DCD3080088880800104208AF
:102940000000000800F0C1070087870700755007E6
:1029500000711C07003EEB0600A1BC060069900652
:102960000066660600703E06006118060017F40552
:102970000074D105005BB00500B2900500627205DD
:10298000005555050078390500B81E0500050505F8
:10299000004EEC040087D40400A1BD040090A704FD
:1029A0000049920400C17D0400EE690400C756048A
:1029B00000444404005C3204000821040041100477
:1029C00000000004003FF00300F8E0030026D203FB
:1029D00000C3C30300CCB503003AA803000A9B035D
:1029E00000388E0300C08103009F750300D0690387
:1029F00000505E03001D53030034480300913D0363
:102A0000003333030016290300381F030097150312
:102A100000300C0300030303000BFA020049F1022B
:102A200000BAE802005CE002002DD802002DD002BE
:102A30000059C80200B0C0020031B90200DAB10288
:102A400000AAAA0200A0A30200BC9C0200FA950200
:102A5000005C8F0200DF88020082820200457C0257
:102A6000002776020027700200436A02007C64029D
:102A700000D05E02003F590200C853020048617254
:102A800064636F6465642044656661756C7420538B
:102A9000657474696E6773204C6F616465640A00C5
:102AA000B80B0000D00700003C0000001027000019
:102AB0000000FA430000FA430000C04000007042EA
:102AC0000000A0420000A0420000C8433333B942D6
:102AD00020286D6D290020204D36303320002055F0
:102AE000004C0046696C616D656E74206C6F6164AA
:102AF0002F756E6C6F6164206C656E677468733AD5
:102B00000A0020204D393030204B004C696E656141
:102B10007220416476616E63653A0A0020440020A9
:102B2000490020204D3330342050002044002049FB
:102B30000020204D3330312050005049442073652F
:102B40007474696E67733A0A00205A0020204D366B
:102B5000363600456E6473746F702061646A7573F5
:102B6000746D656E743A0A00205A002059002020C6
:102B7000473239205333205800205A0020204D344A
:102B800032302053004D65736820426564204C65E7
:102B900076656C696E673A0A00205A002059002059
:102BA000204D323036205800486F6D65206F6666C4
:102BB0007365743A0A00204500205A00205900200D
:102BC000580020540020530020204D323035205131
:102BD0000020453C6D61785F655F6A65726B3E0001
:102BE00020583C6D61785F785F6A65726B3E205952
:102BF0003C6D61785F795F6A65726B3E205A3C6D0F
:102C000061785F7A5F6A65726B3E00416476616EDF
:102C10006365643A20513C6D696E5F7365676D65ED
:102C20006E745F74696D655F75733E20533C6D69AA
:102C30006E5F66656564726174653E20543C6D69C3
:102C40006E5F74726176656C5F66656564726174EF
:102C5000653E0020540020520020204D32303420A8
:102C60005000416363656C65726174696F6E202802
:102C7000756E6974732F7332293A20503C707269F3
:102C80006E745F616363656C3E20523C7265747262
:102C90006163745F616363656C3E20543C74726170
:102CA00076656C5F616363656C3E0A0020450020B9
:102CB0005A0020590020204D3230312058004D61FB
:102CC00078696D756D20416363656C6572617469C7
:102CD0006F6E2028756E6974732F7332293A0A005B
:102CE000204500205A0020590020204D323033204A
:102CF00058004D6178696D756D2066656564726117
:102D00007465732028756E6974732F73293A0A00ED
:102D1000204500205A0020590020204D39322058EB
:102D20000053746570732070657220756E69743A13
:102D30000A0020204D3230302044300A0020204D3F
:102D40003230302044002044697361626C65640A4B
:102D50000046696C616D656E742073657474696E8C
:102D600067733A002020473231202020203B00208A
:102D700066697273740A005A0059005800486F6DF2
:102D80006520004A3233004D323500473930004764
:102D90003120452D3320463138303000473931005D
:102DA00057726974696E6720746F2066696C653A42
:102DB00020006F70656E206661696C65642C20462A
:102DC000696C653A20006F70656E206661696C659C
:102DD000642C2046696C653A200046696C65207356
:102DE000656C65637465640A002053697A653A20EE
:102DF0000046696C65206F70656E65643A2000203E
:102E000066696C653A2000646F696E67006672657A
:102E10007368004E6F772000454E44205355425250
:102E20004F5554494E450A002220706F73002220EE
:102E3000706172656E743A2200535542524F555478
:102E4000494E452043414C4C207461726765743A89
:102E500022004B494C4C45442E2000747279696E17
:102E60006720746F2063616C6C207375622D6763DB
:102E70006F64652066696C65732077697468207477
:102E80006F6F206D616E79206C6576656C732E2096
:102E90004D4158206C6576656C2069733A006F70FF
:102EA000656E206661696C65642C2046696C653AC4
:102EB000200000002100240027002A002D003000FF
:102EC000330001010000040107010A010000220093
:102ED000250028002B002E003100340002010000E4
:102EE000050108010B010000200023002600290035
:102EF0002C002F003200000100000301060109012F
:102F000005050505070508080808020202020A0A65
:102F10000808040404040101010101010101030383
:102F2000030303030303040707070C0C0C0C0C0C2E
:102F30000C0C0202020206060606060606060B0B2B
:102F40000B0B0B0B0B0B010210202008081020406C
:102F5000102040800201020108040201010204085D
:102F600010204080804020100804020180040201EB
:102F70008040201008040201080402010102040834
:102F800010204080010204081020408000000A0B3D
:102F900002090C0D0E0807030401000000000000E8
:102FA0000000000000000000000000000000000021
:102FB00000000000000000001211100000000000DE
:102FC0000000000000000000000000000000000001
:102FD0000000556E6B6E6F776E20636F6D6D616E66
:102FE000643A202200496E736572742066696C61D0
:102FF0006D656E7420616E642070726573732062FB
:103000007574746F6E20286F72204D313038290A24
:10301000004572726F722077726974696E672074EE
:103020006F20454550524F4D210A0000E8EDC7ED95
:1030300011241FBECFEFD1E2DEBFCDBF00E00CBF39
:1030400014E0A0E0B2E0ECEBF8EF01E00BBF02C04F
:1030500007900D92A034B107D9F72CE1A0E4B4E0B9
:1030600001C01D92AF37B207E1F718E1C7E1D8E11F
:1030700000E006C021970109802FFE010E94B6FBE7
:10308000C631D10780E00807A9F70E94F5E70C9444
:103090004DFC0C9400002F923F924F925F926F92E2
:1030A0007F928F929F92AF92BF92CF92DF92EF92D8
:1030B000FF920F931F93CF93DF93CDB7DEB7A79700
:1030C0000FB6F894DEBF0FBECDBFC0906304D090A2
:1030D0006404E0906504F090660420E030E040EA8B
:1030E00050E4C701B6010E943DF487FD52C120E0C3
:1030F00030E041E953E4C701B6010E94E0FA181636
:103100000CF447C110920112109200128091090133
:103110004091FF11042E000C550B817021E0822795
:1031200090E04817590709F433C080910901817074
:1031300028272093FF1181111BC00E946BB3E5EF7C
:10314000F8E084918F01882351F0082E000C990B30
:103150000E9466B30F5F1F4FF8018491F4CF8DE09A
:1031600090E00E9466B38AE090E00E9466B310C0CF
:10317000E9EFF8E084918F01882389F3082E000C91
:10318000990B0E9466B30F5F1F4FF8018491F4CF33
:10319000809166108330C1F12CF4882369F081306E
:1031A000F1F0ACC0843059F1853009F0A7C0E1EEF0
:1031B000F8E084918F0169C08091E30D882309F4C0
:1031C0009DC081E0809366100E942E996093F61155
:1031D0007093F7118093F8119093F9118FC080913B
:1031E000E30D81118BC08091AF0F882311F082E035
:1031F00049C080916710882309F4F6C07FC0809190
:1032000040128823A1F37AC0EDEEF8E084918F019B
:10321000882351F0082E000C990B0E9466B30F5FB3
:103220001F4FF8018491F4CF8DE090E00E9466B3C7
:103230008AE090E00E9466B38091E30D81115EC048
:103240008091650D9091660D891B8F7009F056C0B5
:1032500080916710823088F411E01093671080919C
:10326000021281110AC085EE98E09093EE1B8093C4
:10327000ED1B0E94B19D10930212809140128111AA
:10328000B6CF84E08093661039C0882351F0082EB1
:10329000000C990B0E9466B30F5F1F4FF8018491D9
:1032A000F4CF8DE090E00E9466B38AE090E00E9447
:1032B00066B39091E30D911108C08091650D209146
:1032C000660D821B8F7009F4A2C0809102128111D9
:1032D00015C0911113C08091650D9091660D891BE9
:1032E0008F7009F499C00AC08DE090E00E9466B327
:1032F0008AE090E00E9466B3109267108091E81116
:103300009091E91103974CF57CE8272E74E0372E55
:10331000E0E68E2EEAEE9E2EA12CB12C8BE493E1FA
:103320000E94074018161906C4F48091E811909184
:10333000E911049794F48BE493E10E94CB3F8093CE
:10334000EE11E091EF11F091F0118A3019F08D300B
:1033500009F0D7C0309709F0DDC08091E811909155
:10336000E911009711F40C94FF2901979093E9114A
:103370008093E8118091EA119091EB11019664E03D
:1033800070E00E94A3FB9093EB118093EA110C94E0
:10339000FF2980910012909101128136FAEE9F0769
:1033A000E8F01092011210920012EDEFF8E0849113
:1033B0008F01882351F0082E000C990B0E9466B3F0
:1033C0000F5F1F4FF8018491F4CF8DE090E00E94D1
:1033D00066B38AE090E00E9466B398CE019690931F
:1033E00001128093001292CE10926610E1EFF8E085
:1033F00084918F01882309F477CF082E000C990B54
:103400000E9466B30F5F1F4FF8018491F3CF1092B3
:1034100066101092671059CF8CEC98E09093EE1BD9
:103420008093ED1B0E94B19D0E94CBD6811153C0A9
:1034300080E090E0A0EAB0E488A399A3AAA3BBA38C
:1034400020E030E048EC51E460915B0470915C0452
:1034500080915D0490915E040E94BAF86B017C013A
:1034600020E030E04DE453E40E943DF487FD06C0C7
:10347000C12CD12CFDE4EF2EF3E4FF2EC982DA82B9
:10348000EB82FC82BE01605E7F4FCE0101960E94FE
:10349000699B80E090E0A8ECB2E48CA39DA3AEA36E
:1034A000BFA380E090E0ADE4B3E488A399A3AAA30E
:1034B000BBA380E090E0A0EAB0E489839A83AB8369
:1034C000BC83AE014C5D5F4FBE01605E7F4FCE019D
:1034D00001960E94489B88EC98E09093EE1B8093A5
:1034E000ED1B0E94B19D84EC98E09093EE1B8093BD
:1034F000ED1B0E94B19D1092671081E08093021233
:10350000FDCE8A3309F426CFEF35F10514F40C947F
:10351000D12720CF8091EC119091ED1120E6289FCA
:103520008001299F100D1124C8018A599F4EE80F70
:10353000F91F1282980128593F4E790161E470E029
:10354000C9010E940AFC009711F40C94B5279093CE
:10355000F2118093F1118E199F09800F911F60E085
:1035600070E087599F4E0E943EF00E94FEF9CB0109
:10357000770FAA0BBB0B8232910510F00C94B52784
:10358000FC018827EE58FF4F8F4F0C94B6FBEFEBF2
:10359000F8E084918F01882351F0082E000C990BDC
:1035A0000E9466B30F5F1F4FF8018491F4CF20E0B3
:1035B00030E040E05FE360916304709164048091C7
:1035C0006504909166041EC0EAEBF8E084918F01D7
:1035D000882351F0082E000C990B0E9466B30F5FF0
:1035E0001F4FF8018491F4CF6091510470915204FF
:1035F000072E000C880B990B0E9443F420E030E06A
:1036000040E05FE30E94BAF80E94FEF9CB010E94FD
:1036100031460E94FFD58DE090E00E9466B38AE0BB
:1036200090E00E9466B30C94B527E5EBF8E0849136
:103630008F01882351F0082E000C990B0E9466B36D
:103640000F5F1F4FF8018491F4CF20E030E040E09D
:103650005FE360914D0470914E0480914F0490910E
:103660005004D0CFE0EBF8E084918F01882351F033
:10367000082E000C990B0E9466B30F5F1F4FF801D4
:103680008491F4CF60914B0470914C04B1CF2091A0
:10369000540B3091550B44E6429FC001439F900D5F
:1036A00011246FEF70E00E94A3FB8B01653671055A
:1036B00010F004E610E0EBEAF8E084917F01882343
:1036C00059F0082E000C990B0E9466B3FFEFEF1A19
:1036D000FF0AF7018491F3CFB80180E090E00C94E9
:1036E000F523E7EAF8E084918F01882351F0082E52
:1036F000000C990B0E9466B30F5F1F4FF801849175
:10370000F4CF80E290E00E9466B3E3EAF8E08491AF
:103710008F01882351F0082E000C990B0E9466B38C
:103720000F5F1F4FF8018491F4CF609153047091A3
:10373000540480915504909156040E9400D680E272
:1037400090E00E9466B3EFE9F8E084918F0188234E
:1037500051F0082E000C990B0E9466B30F5F1F4FAB
:10376000F8018491F4CF60915704709158048091CE
:10377000590490915A040E9400D680E290E00E9481
:1037800066B3EBE9F8E084918F01882351F0082EAD
:10379000000C990B0E9466B30F5F1F4FF8018491D4
:1037A000F4CF60915B0470915C0480915D04909112
:1037B0005E040E9400D680E290E0D9C68091E30DBD
:1037C000882309F450C0E6E9F8E084918F0188234A
:1037D00051F0082E000C990B0E9466B30F5F1F4F2B
:1037E000F8018491F4CF8091E40D882359F1809100
:1037F000AF0F882329F18091591090915A10A09110
:103800005B10B0915C100097A105B105C1F0BC013F
:10381000CD016D597F4F8F4F9F4F24E630E040E040
:1038200050E00E945CF860915D1070915E10809194
:103830005F10909160100E945CF8822F01C080E0C0
:1038400090E0E5CEE2E9F8E084918F01882309F465
:10385000E2CE082E000C990B0E9466B30F5F1F4F3B
:10386000F8018491F3CFEAE8F8E084918F0188238E
:1038700009F4D1CE082E000C990B0E9466B30F5F9D
:103880001F4FF8018491F3CFE5E8F8E084918F01B0
:10389000882351F0082E000C990B0E9466B30F5F2D
:1038A0001F4FF8018491F4CF8091F6119091F71198
:1038B000A091F811B091F911892B8A2B8B2B09F467
:1038C00077C00E942E99A50194010E945CF86901BD
:1038D0007A016091F6117091F7118091F811909131
:1038E000F911A50194010E945CF88601021B130BDB
:1038F000C8016CE370E00E948FFBCB019927EAE0DE
:10390000F0E0BF010E94A3FB282FCB01BF010E9462
:10391000A3FB805D80934104205D209342041092BC
:10392000430481E494E00E94FFD580E290E00E948D
:1039300066B3E3E8F8E084917F01882359F0082E0C
:10394000000C990B0E9466B3FFEFEF1AFF0AF70114
:103950008491F3CF80E290E00E9466B3C8016CE3EB
:1039600070E00E948FFB6AE070E00E94A3FB605D44
:1039700060934104805D809342041092430481E48B
:1039800094E00E94FFD580E290E00E9466B3E1E8F7
:10399000F8E084918F01882309F43DCE082E000CB5
:1039A000990B0E9466B30F5F1F4FF8018491F3CF0C
:1039B00080E290E00E9466B3E9E7F8E084918F012D
:1039C000882309F428CE082E000C990B0E9466B3B8
:1039D0000F5F1F4FF8018491F3CF10922112809155
:1039E000090180FF11C0E5E7F8E084918F01882389
:1039F00009F411CE082E000C990B0E9466B30F5FDC
:103A00001F4FF8018491F3CF83E50E9495D5882359
:103A100041F00E94B0D50E9403FA7093F5116093B3
:103A2000F411E1E7F8E084918F01882351F0082E2A
:103A3000000C990B0E9466B30F5F1F4FF801849131
:103A4000F4CF8DE090E00E9466B38AE090E00E949F
:103A500066B380913F12882309F4A1C28091F411CA
:103A60009091F5118430910509F4D2C040F4892B6E
:103A700009F03BC4E1E9F6E084918F010CC0883085
:103A8000910509F47EC10C9709F02FC4E9E0F5E037
:103A900084918F012FC2882351F0082E000C990BBE
:103AA0000E9466B30F5F1F4FF8018491F4CF8DE041
:103AB00090E00E9466B38AE090E00E9466B3E6E878
:103AC000F6E084918F01882351F0082E000C990BA9
:103AD0000E9466B30F5F1F4FF8018491F4CF8DE011
:103AE00090E00E9466B38AE090E00E9466B3EAE745
:103AF000F6E084918F01882351F0082E000C990B79
:103B00000E9466B30F5F1F4FF8018491F4CF8DE0E0
:103B100090E00E9466B38AE090E00E9466B3EEE611
:103B2000F6E084918F01882351F0082E000C990B48
:103B30000E9466B30F5F1F4FF8018491F4CF8DE0B0
:103B400090E00E9466B38AE090E00E9466B3E0E6EF
:103B5000F6E084918F01882351F0082E000C990B18
:103B60000E9466B30F5F1F4FF8018491F4CF8DE080
:103B700090E00E9466B38AE090E00E9466B3E2E5BE
:103B8000F6E084918F01882351F0082E000C990BE8
:103B90000E9466B30F5F1F4FF8018491F4CF8DE050
:103BA00090E00E9466B38AE090E00E9466B3E5E48C
:103BB000F6E084918F01882351F0082E000C990BB8
:103BC0000E9466B30F5F1F4FF8018491F4CF8DE020
:103BD00090E00E9466B38AE090E00E9466B3E8E35A
:103BE000F6E084918F01882351F0082E000C990B88
:103BF0000E9466B30F5F1F4FF8018491F4CF8DE0F0
:103C000090E00E9466B38AE090E00E9466B36DC3C4
:103C1000EAE2F6E084918F01882351F0082E000C2F
:103C2000990B0E9466B30F5F1F4FF8018491F4CF88
:103C30008DE090E00E9466B38AE090E00E9466B357
:103C4000ECE1F6E084918F01882351F0082E000CFE
:103C5000990B0E9466B30F5F1F4FF8018491F4CF58
:103C60008DE090E00E9466B38AE090E00E9466B327
:103C7000E6E0F6E084918F01882351F0082E000CD5
:103C8000990B0E9466B30F5F1F4FF8018491F4CF28
:103C90008DE090E00E9466B38AE090E00E9466B3F7
:103CA000E0EFF5E084918F01882351F0082E000C9D
:103CB000990B0E9466B30F5F1F4FF8018491F4CFF8
:103CC0008DE090E00E9466B38AE090E00E9466B3C7
:103CD000EEEDF5E084918F01882351F0082E000C61
:103CE000990B0E9466B30F5F1F4FF8018491F4CFC8
:103CF0008DE090E00E9466B38AE090E00E9466B397
:103D0000ECECF5E084918F01882351F0082E000C33
:103D1000990B0E9466B30F5F1F4FF8018491F4CF97
:103D20008DE090E00E9466B38AE090E00E9466B366
:103D3000EEEBF5E084918F01882351F0082E000C02
:103D4000990B0E9466B30F5F1F4FF8018491F4CF67
:103D50008DE090E00E9466B38AE090E00E9466B336
:103D6000E0EBF5E084918F01882309F448CF082E19
:103D7000000C990B0E9466B30F5F1F4FF8018491EE
:103D8000F3CFE9EAF5E084918F01882351F0082E02
:103D9000000C990B0E9466B30F5F1F4FF8018491CE
:103DA000F4CF8DE090E00E9466B38AE090E00E943C
:103DB00066B3E2EAF5E084918F01882351F0082E82
:103DC000000C990B0E9466B30F5F1F4FF80184919E
:103DD000F4CF8DE090E00E9466B38AE090E00E940C
:103DE00066B3EBE8F5E084918F01882351F0082E4B
:103DF000000C990B0E9466B30F5F1F4FF80184916E
:103E0000F4CF8DE090E00E9466B38AE090E00E94DB
:103E100066B3E4E7F5E084918F01882351F0082E22
:103E2000000C990B0E9466B30F5F1F4FF80184913D
:103E3000F4CF8DE090E00E9466B38AE090E00E94AB
:103E400066B3EDE5F5E084918F01882351F0082EEB
:103E5000000C990B0E9466B30F5F1F4FF80184910D
:103E6000F4CF8DE090E00E9466B38AE090E00E947B
:103E700066B3E6E4F5E084918F01882351F0082EC3
:103E8000000C990B0E9466B30F5F1F4FF8018491DD
:103E9000F4CF8DE090E00E9466B38AE090E00E944B
:103EA00066B3E3E3F5E084918F01882351F0082E97
:103EB000000C990B0E9466B30F5F1F4FF8018491AD
:103EC000F4CF8DE090E00E9466B38AE090E00E941B
:103ED00066B3E0E2F5E084918F01882309F48FCE88
:103EE000082E000C990B0E9466B30F5F1F4FF8015C
:103EF0008491F3CF882351F0082E000C990B0E9477
:103F000066B30F5F1F4FF8018491F4CF8DE090E00E
:103F10000E9466B38AE090E00E9466B3E2EFF4E0AC
:103F200084918F01882351F0082E000C990B0E9478
:103F300066B30F5F1F4FF8018491F4CF8DE090E0DE
:103F40000E9466B38AE090E00E9466B3EAEDF4E076
:103F500084918F01882351F0082E000C990B0E9448
:103F600066B30F5F1F4FF8018491F4CF8DE090E0AE
:103F70000E9466B38AE090E00E9466B3E2ECF4E04F
:103F800084918F01882309F43ACE082E000C990BF6
:103F90000E9466B30F5F1F4FF8018491F3CF8091A9
:103FA000E40D882309F478C181E0809361101092B8
:103FB00063101092621083E39EE00E94E9AC8BE1F3
:103FC000E3E3FEE0DE01159601900D928A95E1F79C
:103FD0008091310E9091320E9C838B8385EF92E01D
:103FE0009A83898340E050E0BE016F5F7F4F80E09D
:103FF00090E00E945DB5CE0101960E9406A4C0909B
:104000006210D09063100091F4111091F511C60167
:10401000801B910B049720F06801F3E0CF0ED11CB8
:1040200053EB452E54E0552E64EA662E64E0762E5E
:10403000C016D10608F459C10115110509F09DC03B
:1040400067EE7DE083E39EE00E94B1AB6BE173E03D
:1040500087EE9DE00E9415FC892B09F048C0F20113
:10406000849143EBE42E44E0F42E882359F0082E8B
:10407000000C990B0E9466B3FFEFEF1AFF0AF701DD
:104080008491F3CF8DE090E00E9466B38AE090E0E7
:104090000E9466B3F301849134EAE32E34E0F32EF8
:1040A000882359F0082E000C990B0E9466B3FFEF8D
:1040B000EF1AFF0AF7018491F3CF8DE090E00E94A0
:1040C00066B38AE090E00E9466B380E090E00E94D0
:1040D000F9D5E4E9F4E084917F012FEFE21AF20AC6
:1040E000882309F4D6C00E94009DF701F4CFE0E9CF
:1040F000F4E084917F01882359F0082E000C990B7D
:104100000E9466B3FFEFEF1AFF0AF7018491F3CF25
:104110008DE090E00E9466B38AE090E00E9466B372
:10412000F10184912CE8E22E24E0F22E882359F04C
:10413000082E000C990B0E9466B3FFEFEF1AFF0ADE
:10414000F7018491F3CF8DE090E00E9466B38AE09E
:1041500090E00E9466B380E090E00E94F9D5E7E825
:10416000F4E084917F012FEFE21AF20A882309F428
:1041700090C00E94009DF701F4CF60E070E0C8019C
:1041800001970E9433D78091E50D882309F45AC026
:10419000E5E8F4E084917F01882359F0082E000CB3
:1041A000990B0E9466B3FFEFEF1AFF0AF7018491A3
:1041B000F3CF87EE9DE00E94FFD58DE090E00E9456
:1041C00066B38AE090E00E9466B3E3E8F4E084918D
:1041D0007F01882359F0082E000C990B0E9466B3CA
:1041E000FFEFEF1AFF0AF7018491F3CF84EF9DE010
:1041F0000E94FFD58DE090E00E9466B38AE090E0D7
:104200000E9466B3C8010E94F9D5E1E8F4E0849108
:104210007F012FEFE21AF20A882321F00E94009D0D
:10422000F701F5CF94EFE92E9DE0F92EF70181918A
:104230007F01882319F00E94009DF8CF8AE00E9438
:10424000009D27C087EE9DE00E94FFD58DE090E0A5
:104250000E9466B38AE090E00E9466B384EF9DE01E
:104260000E94FFD58DE090E00E9466B38AE090E066
:104270000E9466B3C8010E94F9D584EFE82E8DE054
:10428000F82EF70181917F018823C1F20E94009DE1
:10429000F8CF0F5F1F4FCCCEE2E7F4E084918F019F
:1042A000882351F0082E000C990B0E9466B30F5F13
:1042B0001F4FF8018491F4CF8DE090E00E9466B327
:1042C0008AE090E00E9466B3E3E6F4E084918F0117
:1042D000882309F494CC082E000C990B0E9466B335
:1042E0000F5F1F4FF8018491F3CFEDE6F8E0849162
:1042F0008F01882309F48FC9082E000C990B0E94A6
:1043000066B30F5F1F4FF8018491F3CF8091E30DE7
:10431000882319F00E94F6D428C610926710B7C0FF
:1043200080916610823019F0833609F088C01091B0
:104330006710123009F444C028F4112379F01130C9
:1043400011F165C0143009F45CC008F44DC015309B
:1043500009F05DC083E08093661057C00E942E99DB
:104360006093F6117093F7118093F8119093F911FF
:104370008091E40D882319F081E08093E30D81E0C2
:104380008093661044C08BE594E09093EE1B80937D
:10439000ED1B0E94B19D109202120E942E99609313
:1043A000F6117093F7118093F8119093F9118091A1
:1043B000E40D81111093E30D81E0809366101EC01F
:1043C00086E594E09093EE1B8093ED1B0E94B19DD7
:1043D00010923902109240048091E40D882371F00C
:1043E00081E08093E30D0AC08FE594E09093EE1B8B
:1043F0008093ED1B0E94B19D1092021210926710E3
:1044000006C083E08093661082E080936710E9E63F
:10441000F8E084918F01882351F0082E000C990B4D
:104420000E9466B30F5F1F4FF8018491F4CF8DE0B7
:1044300090E00E9466B38AE090E00E9466B38091AB
:104440004A04882309F491C581E594E09093EE1B1A
:104450008093ED1B0E94B19D0E94F9A310924A0423
:10446000109240041092390280916710843018F045
:1044700082508093671083E08093661076C58091A8
:10448000E30D811104C080916610833619F40E94F7
:10449000B2B46BC5E5E6F8E084918F01882351F052
:1044A000082E000C990B0E9466B30F5F1F4FF80196
:1044B0008491F4CF8DE090E00E9466B38AE090E0B2
:1044C0000E9466B310926610109267104EC58CE57C
:1044D00098E00E9428A480916610833609F445C5AF
:1044E0000091F1111091F2117801F4E0EF0EF11C3E
:1044F0006AE270E0C7010E940AFCF80124812F32B1
:1045000021F4B8016B5F7F4F03C02C3331F4B70146
:1045100081E292E10E941EFC7EC810922112009757
:1045200019F0FC01319710828091F1119091F211F4
:1045300040E061E004960E9431D88091AF0F88235B
:10454000C9F0E8E5F8E084918F01882351F0082E46
:10455000000C990B0E9466B30F5F1F4FF801849106
:10456000F4CF8DE090E00E9466B38AE090E00E9474
:1045700066B351C8E4E5F8E084918F01882389F39C
:10458000082E000C990B0E9466B30F5F1F4FF801B5
:104590008491F4CF8091650D9091660D891B8F7089
:1045A00009F0E3C480916610823009F4DEC48336DA
:1045B00009F4DBC48091AF0F81110BC5D6C483E52C
:1045C0000E9495D5811126C083E40E9495D5882349
:1045D00009F4CBC48091650D9091660D891B8F7095
:1045E00009F0C3C420E030E040E251E460915B0494
:1045F00070915C0480915D0490915E040E943DF492
:1046000087FF08C089E498E09093EE1B8093ED1B30
:104610000E94B19D0E94B0D520E030E0A9010E9427
:104620003DF487FD10C00E94B0D520E030E849E895
:1046300053E40E94E0FA18164CF00E94B0D50E9494
:1046400003FACB0105C080E090E002C083E191E075
:104650000E94E75F8AC483E50E9495D5882309F408
:1046600084C40E94B0D520E030E0A9010E943DF44E
:1046700087FD10C00E94B0D520E030E046E153E451
:104680000E94E0FA18164CF00E94B0D50E9403FA7E
:10469000CB0105C080E090E002C086E990E00E9476
:1046A000674663C483E50E9495D58823E1F00E94A4
:1046B000B0D520E030E04FE753E40E94A2F420E0C0
:1046C00030E048EC52E40E9496F90E9403FA6F3FF2
:1046D000710519F010F06FEF70E07093550B609357
:1046E000540B0C940B1B8FEF90E09093550B809321
:1046F000540B0C940B1B8091650D9091660D891BDA
:104700008F7011F00C940B1B8091E30D81110C94B0
:104710000B1B0E94916B5F9A809149048E7F80935E
:1047200049048A9A479A809149048D7F809349046D
:10473000809108018095817080930601479A80914D
:1047400049048B7F80934904129A0C940B1B83E5D8
:104750000E9495D5882319F10E94B0D520E030E061
:1047600040E252E40E943DF487FD0FC00E94B0D5A4
:1047700020E030EC49E754E40E94E0FA181644F0D7
:104780000E94B0D50E94FEF905C068E270E002C048
:1047900067EE73E07093010260930002E6C3E3E406
:1047A000F8E084918F01882351F0082E000C990BBA
:1047B0000E9466B30F5F1F4FF8018491F4CFC09041
:1047C0000002D09001020D2C000CEE08FF08F7FE4D
:1047D0000EC06DE28BE493E10E947E3F662777274F
:1047E000CB016C197D098E099F094AE003C04AE09C
:1047F000C701B6010E94B9D50C940B1B8091650DC1
:104800009091660D891B8F7009F0AFC3809166107F
:10481000823009F4AAC3833609F075C3A6C3809118
:10482000650D9091660D891B8F7011F00C940B1B18
:1048300080916610823011F40C940B1B833609F0C2
:1048400000C40C940B1B8091650D9091660D891B23
:104850008F7009F08AC380916610823009F485C395
:10486000833609F044C581C38091650D9091660D32
:10487000891B8F7009F079C380916610823009F42A
:1048800074C3833609F069C570C38091650D90913A
:10489000660D891B8F7009F068C3809166108230A5
:1048A00009F463C3833609F08EC55FC3809121127A
:1048B000811103C00E946BB34BC28E3271F580919F
:1048C00022128E3209F0CDC18091840F882309F421
:1048D0003FC281508093840F882361F090E001975C
:1048E0004FE1489F9001499F300D1124C901825B1F
:1048F000914F02C080E19EE02BE1FC013496A3E3DE
:10490000BEE001900D922A95E1F7FC01828193812E
:104910009093320E8093310E1BC28C3309F0A1C1EB
:104920006DE173E081E292E10E9415FC892B21F494
:1049300081E080933F120CC26CE273E081E292E16D
:104940000E9415FC892B79F4EDE2F4E084918F014B
:104950000F5F1F4F882321F00E94009DF801F6CFC2
:104960008FE094E01FC163E473E081E292E10E9472
:1049700015FC892B79F4EBEEF3E084918F010F5F46
:104980001F4F882321F00E94009DF801F6CF88ED8B
:1049900093E008C16AE573E081E292E10E9415FCB0
:1049A000892B31F5EDEBF3E084918F010F5F1F4F01
:1049B000882321F00E94009DF801F6CF88EB93E058
:1049C0009093EE1B8093ED1B0E94B19D84E594E0D3
:1049D00099A388A389E690E09A838983BE01605EEB
:1049E0007F4FCE0101960E94C2D48DE796E02DC084
:1049F00068E673E081E292E10E9415FC892B99F54B
:104A0000E8E9F3E084918F010F5F1F4F882321F0C5
:104A10000E94009DF801F6CF83E993E09093EE1B8E
:104A20008093ED1B0E94B19D8DE796E099A388A32A
:104A300089E690E09A838983BE01605E7F4FCE0154
:104A400001960E94C2D484E594E099A388A382EDE4
:104A500090E09A838983BE01605E7F4FCE0101960C
:104A60000E94C2D475C16BE773E081E292E10E94BB
:104A700015FC892B79F4E8E7F3E084918F010F5F4F
:104A80001F4F882321F00E94009DF801F6CF8FE68A
:104A900093E088C069E873E081E292E10E9415FC2E
:104AA000892B71F40CE413E0F8018491882329F038
:104AB0000F5F1F4F0E94009DF7CF85E493E072C007
:104AC0006FE973E081E292E10E9415FC892B79F491
:104AD000E6E2F3E084918F010F5F1F4F882321F0FE
:104AE0000E94009DF801F6CF8FE193E05BC061EB7F
:104AF00073E081E292E10E9415FC892B79F4E7E0F2
:104B0000F3E084918F010F5F1F4F882321F00E94F3
:104B1000009DF801F6CF86EF92E044C06CEB73E0A5
:104B200081E292E10E9415FC892B79F4EDEDF2E02F
:104B300084918F010F5F1F4F882321F00E94009DF9
:104B4000F801F6CF8BEC92E02DC068EC73E081E2C7
:104B500092E10E9415FC892B79F4E0EBF2E084915C
:104B60008F010F5F1F4F882321F00E94009DF801E5
:104B7000F6CF8EE992E016C066ED73E081E292E135
:104B80000E9415FC892BA9F4E4E8F2E084918F01DE
:104B90000F5F1F4F882321F00E94009DF801F6CF80
:104BA00083E792E09093EE1B8093ED1B0E94B19DF2
:104BB000CFC063EE73E081E292E10E9415FC892B85
:104BC000D9F4EFE4F2E084918F010F5F1F4F882347
:104BD00021F00E94009DF801F6CF82E080936710DB
:104BE00085E292E09093EE1B8093ED1B0E94B19DB5
:104BF00083E080936610ACC06AEF73E081E292E1DB
:104C00000E9415FC892B09F5EAE2F2E084918F01FC
:104C10000F5F1F4F882321F00E94009DF801F6CFFF
:104C200086E594E09093EE1B8093ED1B0E94B19D6E
:104C300010923902109240048091E40D882309F407
:104C400087C081E08093E30D83C062E174E081E27C
:104C500092E10E9415FC892B09F07AC010923F1254
:104C600077C01D8218861C821B8285EF92E09A8392
:104C700089838091360E811103C060E17EE002C01D
:104C80006FE27EE06115710519F06C5F7F4F02C025
:104C900060E070E021E041E252E1CE0105960E9421
:104CA0001EB1882361F18BE1FE013596A3E3BEE0DE
:104CB00001900D928A95E1F72B813C813093320E61
:104CC0002093310E8091840F8A3008F03DC091E02E
:104CD000980F9093840FFFE18F9FC0011124DC0196
:104CE000AE5AB14F4BE1E3E3FEE001900D924A95DD
:104CF000E1F7FC01E25BF14F3383228325C0E4E05E
:104D0000F7E284918F010F5F1F4F882321F00E94EB
:104D1000009DF801F6CFEFE0F2E084918F010F5F84
:104D20001F4F882321F00E94009DF801F6CF01E279
:104D300012E1F80181918F01882319F00E94009DF2
:104D4000F8CF8AE00E94009DCE0101960E9406A441
:104D5000109221128091090180FF07C1E7E8F7E076
:104D600084918F01882311F40C940B1B082E000CE6
:104D7000990B0E9466B30F5F1F4FF8018491F2CF29
:104D80008FE40E9495D581110C940B1B83E40E9443
:104D900095D50C940B1B83E50E9495D5811159C0C4
:104DA0008FE40E9495D5882319F08FE497E007C01F
:104DB00084E50E9495D5882349F087E297E0909397
:104DC000EE1B8093ED1B0E94B19D43C083E40E94C3
:104DD00095D5882319F08EEF96E0F1CF81E50E94FA
:104DE00095D5882319F086ED96E0E9CF88E40E94F6
:104DF00095D58823C9F0E2EDF6E084918F018823F0
:104E000051F0082E000C990B0E9466B30F5F1F4FE4
:104E1000F8018491F4CF8DE090E00E9466B38AE0BF
:104E200090E00E9466B315C08CE40E9495D588235B
:104E300081F0EEECF6E084918F01882361F3082E77
:104E4000000C990B0E9466B30F5F1F4FF80184910D
:104E5000F4CFE6E9F7E084918F01882311F40C94F4
:104E60000B1B082E000C990B0E9466B30F5F1F4F9F
:104E7000F8018491F2CF8091650D8091660D0C94BC
:104E80000B1B83E50E9495D5882309F46EC086EA42
:104E900096E09093EE1B8093ED1B0E94B19DE6E996
:104EA000F7E084918F01882311F40C940B1B082EDA
:104EB000000C990B0E9466B30F5F1F4FF80184919D
:104EC000F2CFE1EAF6E084918F01882351F0082EB9
:104ED000000C990B0E9466B30F5F1F4FF80184917D
:104EE000F4CFECE9F6E084918F01882311F40C945F
:104EF0000B1B082E000C990B0E9466B30F5F1F4F0F
:104F0000F8018491F2CF88E50E9495D5811106C001
:104F100089E50E9495D5882309F485C088E50E941B
:104F200095D5882341F08DE398E09093EE1B809314
:104F3000ED1B0E94B19D89E50E9495D5882341F023
:104F400087E398E09093EE1B8093ED1B0E94B19D48
:104F50008AE50E9495D5882341F081E398E09093FB
:104F6000EE1B8093ED1B0E94B19D8091EC119091FE
:104F7000ED11019664E070E00E94A3FB9093ED11A7
:104F80008093EC118091E8119091E9110196909332
:104F9000E9118093E8111092F0111092EF110C9426
:104FA0008E194091EC115091ED119F012F5F3F4FF1
:104FB0003093F0112093EF1190E6949F9001959F0C
:104FC000300D11242A593F4EE20FF31F82830C94B7
:104FD0008E19109267100E942E996093F6117093AB
:104FE000F7118093F8119093F9118091E40D8823C3
:104FF00019F081E08093E30D81E0809366101092B8
:105000000212E0E5F8E084918F01882311F40C94FA
:105010000B1B082E000C990B0E9466B30F5F1F4FED
:10502000F8018491F2CF8AE50E9495D5811176CF5F
:1050300083E40E9495D5882309F497CF8DE298E008
:105040008ECF86E40E9495D5882309F44DC10E9435
:10505000B0D50E9403FA8B0189E298E09093EE1B91
:105060008093ED1B0E94B19D88E50E9495D5882311
:1050700009F451C00E94B0D52B013C012DEC3CEC51
:105080004CE45EE30E943DF49E012F5F3F4F7901A7
:10509000181674F020E030E0A901C301B2010E94AB
:1050A000E0FA18162CF41F930F938EE198E005C1D7
:1050B0002DEC3CEC4CEC5DEBC301B2010E943DF4E5
:1050C00018167CF020E030E040E85FEBC301B2014D
:1050D0000E94E0FA18162CF41F930F9382E198E0D7
:1050E000ECC01F930F93C301B2010E94FEF97F939E
:1050F0006F9388E098E09F938F93FF92EF920E94C6
:105100000FF40FB6F894DEBF0FBECDBFCE010196EF
:105110000E948C9DDFC089E50E9495D5882309F403
:1051200041C00E94B0D52B013C012DEC3CEC4CE47D
:105130005EE30E943DF4FE0131967F01181674F083
:1051400020E030E0A901C301B2010E94E0FA181684
:105150002CF41F930F938DEF97E0AFC02DEC3CEC38
:105160004CEC5DEBC301B2010E943DF418167CF0DB
:1051700020E030E040E85FEBC301B2010E94E0FABA
:1051800018162CF41F930F9381EF97E096C01F938E
:105190000F93C301B2010E94FEF97F936F9387EED4
:1051A00097E0A9CF8AE50E9495D5882309F441C0EC
:1051B0000E94B0D52B013C012DEC3CEC4CE45EE3AD
:1051C0000E943DF4FE0131967F01181674F020E034
:1051D00030E0A901C301B2010E94E0FA18162CF4D4
:1051E0001F930F938CED97E068C02DEC3CEC4CECDA
:1051F0005DEBC301B2010E943DF418167CF020E083
:1052000030E040E85FEBC301B2010E94E0FA1816FB
:105210002CF41F930F9380ED97E04FC01F930F93D3
:10522000C301B2010E94FEF97F936F9386EC97E071
:1052300062CF85E40E9495D5882309F44BC00E9473
:10524000B0D52B013C012DEC3CEC4CE45EE30E941C
:105250003DF4FE0131967F01181674F020E030E035
:10526000A901C301B2010E94E0FA18162CF41F93A1
:105270000F938BEB97E021C02DEC3CEC4CEC5DEBFD
:10528000C301B2010E943DF418167CF020E030E02A
:1052900040E85FEBC301B2010E94E0FA18162CF45B
:1052A0001F930F938FEA97E008C0C301B2010E94D9
:1052B000FEF97F936F9384EA97E09F938F93FF9219
:1052C000EF920E940FF40F900F900F900F900F909D
:1052D0000F901CCF80EA97E09093EE1B8093ED1B1C
:1052E0000E94B19D0C940B1B00E010E0B5CE20E0B5
:1052F00030E040E251E460915B0470915C04809185
:105300005D0490915E040E943DF487FF08C089E926
:1053100097E09093EE1B8093ED1B0E94B19D82E37A
:1053200090E090934C0480934B040E944F5F88EC74
:1053300090E00E94E75FE6E9F7E084918F0188231F
:1053400011F40C940B1B082E000C990B0E9466B3F1
:105350000F5F1F4FF8018491F2CF20E030E040E270
:1053600051E460915B0470915C0480915D049091C4
:105370005E040E943DF487FF08C08FE897E0909399
:10538000EE1B8093ED1B0E94B19D80E590E0909311
:105390004C0480934B040E944F5F80EF90E00E948A
:1053A000E75FE6E9F7E084918F01882311F40C941C
:1053B0000B1B082E000C990B0E9466B30F5F1F4F4A
:1053C000F8018491F2CF80E090E00E94E75F1092B4
:1053D0004C0410924B040E944F5FEBE8F7E084917D
:1053E0008F01882311F40C940B1B082E000C990BD1
:1053F0000E9466B30F5F1F4FF8018491F2CFA7960A
:105400000FB6F894DEBF0FBECDBFDF91CF911F91D5
:105410000F91FF90EF90DF90CF90BF90AF909F9053
:105420008F907F906F905F904F903F902F90089556
:105430002F923F924F925F926F927F928F929F92A4
:10544000AF92BF92CF92DF92EF92FF920F931F9392
:10545000CF93DF93CDB7DEB7C354D1090FB6F8941D
:10546000DEBF0FBECDBF11E01093FC1B80918F13E8
:105470008D3409F459C5843511F40C94753E873484
:1054800011F00C94C13E80918D1390918E138B314D
:10549000910509F403C2A4F48430910534F48230F8
:1054A000910594F597FF29C03BC58430910509F417
:1054B000BFC14A9709F034C50E9475460C94C33E9B
:1054C0008A32910509F421C444F48C31910509F420
:1054D00015C24D9709F417C223C58B35910509F400
:1054E0009FC48C35910509F49FC48A35910509F054
:1054F00017C5109278040C94C33E80911902811153
:105500000C94C83E0C94C33E20911902222311F43E
:105510000C94C33E11E0029709F010E00E94DD797F
:1055200019821A821B821C821D821E821F8218868B
:1055300082E50E94D844882309F42AC10E94584475
:105540004B015C0120E030E0A9010E943DF488237A
:1055500009F434C1409153045091540460915504AE
:105560007091560448A759A76AA77BA76091570472
:10557000709158048091590490915A046CA77DA7AA
:105580008EA79FA780914C1C90914D1CA0914E1C02
:10559000B0914F1C88AB99ABAAABBBAB4091501CF0
:1055A0005091511C6091521C7091531C4CAB5DABDF
:1055B0006EAB7FAB9C01AD0168A579A58AA59BA5C3
:1055C0000E943DF481110DC02CA93DA94EA95FA9EF
:1055D0006CA57DA58EA59FA50E943DF4882309F4A6
:1055E000EDC020E030E0A901C501B4010E943DF406
:1055F000881F8827881F181749F060E070E080E84E
:105600009FEB6CAF7DAF8EAF9FAF08C080E090E0A6
:10561000A0E8BFE38CAF9DAFAEAFBFAF28A539A563
:105620004AA55BA568A979A98AA99BA90E94B9F88E
:1056300068AF79AF8AAF9BAF2CA53DA54EA55FA5FE
:105640006CA97DA98EA99FA90E94B9F86B017C0164
:1056500028AD39AD4AAD5BADCA01B9010E94A2F4D3
:105660002B013C01A7019601C701B6010E94A2F4DB
:105670009B01AC01C301B2010E94BAF80E9425FB54
:105680002B013C0120E030E040E05FE30E94A2F407
:1056900024966CAF7DAF8EAF9FAF2497A501940188
:1056A000C501B4010E94A2F44B015C0124962CAD0B
:1056B0003DAD4EAD5FAD2497CA01B9010E94A2F481
:1056C0009B01AC01C501B4010E94B9F80E9425FB01
:1056D0002CAD3DAD4EAD5FAD0E94A2F44B015C011F
:1056E000C701B6019058A30192010E9496F9A50145
:1056F00094010E94A2F46B017C0128A939A94AA94E
:105700005BA968A579A58AA59BA50E94BAF820E0A7
:1057100030E040E05FE30E94A2F49B01AC01C701CE
:10572000B6010E94BAF828A539A54AA55BA50E9432
:10573000B9F869837A838B839C832CA93DA94EA9F0
:105740005FA96CA57DA58EA59FA50E94BAF820E053
:1057500030E040E05FE30E94A2F46B017C01A30112
:10576000920168AD79AD8AAD9BAD0E9496F9A50115
:1057700094010E94A2F49B01AC01C701B6010E94F2
:10578000BAF82CA53DA54EA55FA50E94B9F812C098
:1057900089E40E94D844882331F00E9458446983E8
:1057A0007A838B839C838AE40E94D844882331F0D7
:1057B0000E9458446D837E838F83988720E030E079
:1057C000A90169817A818B819C810E943DF48111BC
:1057D0000EC020E030E0A9016D817E818F81988527
:1057E0000E943DF4811103C0EFEEF6E20DC0412F9F
:1057F000BE016F5F7F4F8CE49CE10E9422B70C9446
:10580000C33E0E94009DF80184918F010F5F1F4FDE
:105810008111F7CFE7E2F9E084918F010F5F1F4F0D
:10582000882311F40C94C33E0E94009DF801F4CF2C
:1058300080E50E94D844882329F00E940E9C6B01C9
:105840007C0103C0C12CD12C760183E50E94D84491
:10585000882361F00E94584420E030E04AE754E495
:105860000E94A2F40E9403FA6B017C010E94938DB6
:105870000E942E99C60ED71EE81EF91E0E942E9970
:10588000DC01CB018C199D09AE09BF09B7FD02C02F
:105890000C94C33E80E00E946DA4F0CF0E94CBD652
:1058A00081110C94C33E80E090E0A0EAB0E48983CB
:1058B0009A83AB83BC8380E090E0ADE4B3E48D8356
:1058C0009E83AF83B88780E090E0A0EAB1E4898747
:1058D0009A87AB87BC8780E50E94D844882319F05B
:1058E0000E94284401C060E068A3BE016F5F7F4F43
:1058F000CE0180960E9413CC0C94C33E80E00E949F
:10590000EF780C94C33E83E50E94D844882321F1AC
:105910000E943844182F863070F0EDEEF9E0849143
:105920008F010F5F1F4F882311F40C94C33E0E9418
:10593000009DF801F4CF833009F44AC130F481307E
:1059400091F1823009F43FC008C0843009F4ABC142
:10595000853009F4B8C101C010E00E94B5998111E9
:1059600003C0EDECF9E013C08091171C882319F0F7
:1059700069E174E002C06DE174E085EC99E00E9499
:1059800038C28AE00E94009D0E94A9CCA2C18491E5
:105990007F019FEFE91AF90A882309F49AC10E944E
:1059A000009DF701F4CF0E945CCD1092030210928B
:1059B00002028AEB99E09093EE1B8093ED1B0E940C
:1059C000B19D0C94C33E809102029091030297FF17
:1059D0000EC0E1E9F9E084918F010F5F1F4F88232A
:1059E00011F40C94C33E0E94009DF801F4CF00977F
:1059F000A1F480913A028093790419821A821B8261
:105A00001C8218A219A21AA21BA2BE016F5F7F4FAF
:105A1000CE0180960E94699B27C0815065E00E945C
:105A200082FB80FF03C024E0291B922FA5E09A028D
:105A3000F0011124E80FF11D87FDFA95EE0FFF1F0D
:105A4000EE0FFF1FE659F44E80915B0490915C04C9
:105A5000A0915D04B0915E0480839183A283B3839F
:105A60008091790480933A0280910202909103021E
:105A7000893191050CF067C010923A029C012F5FAA
:105A80003F4F309303022093020265E00E9482FBA5
:105A900080FF03C024E0291B922F40915B045091AA
:105AA0005C0460915D0470915E0448A359A36AA3ED
:105AB0007BA319821A821B821C82B4E08B029001A4
:105AC0001124F901E556F24F4F01208131814281C5
:105AD0005381F4E09F02C0011124BC016155724F53
:105AE0005B01DB016D917D918D919C91FE01319661
:105AF0006F01E12CF12C00EA10E40E94599A1982FE
:105B00001A821B821C82B601CE0180960E94699B7C
:105B1000F50180819181A281B38180935304909398
:105B20005404A0935504B0935604F40180819181EC
:105B3000A281B3818093570490935804A093590491
:105B4000B0935A04C8C080E090E0A0EAB0E480932B
:105B50005B0490935C04A0935D04B0935E040E9488
:105B6000029A0E94938D8FEF9FEF90930302809390
:105B70000202EDE7F9E084918F010F5F1F4F882348
:105B800021F00E94009DF801F6CF83E992E09A830C
:105B9000898304E610E019A308A3BE016F5F7F4F5D
:105BA000CE0180960E94C2D48AEB92E09A838983C8
:105BB00019A308A3BE016F5F7F4FCE0180960E949C
:105BC000C2D481E00E94EF7881E00E94E29983C014
:105BD00088E50E94D8448823D1F00E9428441FEF12
:105BE000160F1530D8F065E070E08AE699E00E9463
:105BF0001FC2E7E6F9E084918F010F5F1F4F8823F2
:105C000011F40C94C33E0E94009DF801F4CF88E586
:105C10000E94009D0E94E5E70C94C33E89E50E9426
:105C2000D8448823D1F00E9428440FEF060F053096
:105C3000D8F065E070E084E599E00E941FC2E1E5DC
:105C4000F9E084918F010F5F1F4F882311F40C94AA
:105C5000C33E0E94009DF801F4CF89E50E94009D9B
:105C60000E94E5E70C94C33E8AE50E94D84488234D
:105C700099F00E94584425E0129FF0011124E00F92
:105C8000F11DEE0FFF1FEE0FFF1FE659F44E60836C
:105C900071838283938335C08AE50E94009D0E94B0
:105CA000E5E70C94C33E8AE50E94D8448823A1F31B
:105CB0000E9458446093661B7093671B8093681B17
:105CC0009093691B1EC080E00E94E2990E945CCD07
:105CD00018C01230B1F46091020270910302693170
:105CE000710514F069E170E082E499E00E941FC23E
:105CF00069E170E08DE399E00E941FC28AE00E9492
:105D0000009D0E943F740C94C33E80911902882329
:105D100011F40C94C33E89E40E94D844E82E8823F1
:105D200021F00E942844062F01C000E08AE40E946E
:105D3000D844F82E882321F00E942844162F01C051
:105D400010E0EE2011F0053020F4FF2081F0153036
:105D500070F0E4E0FAE084918F010F5F1F4F882319
:105D600011F40C94C33E0E94009DF801F4CF0E94F0
:105D7000E444EE2091F044E00402F0011124E155E6
:105D8000F24F80819181A281B38180934C1C9093CA
:105D90004D1CA0934E1CB0934F1CFF2091F054E07B
:105DA0001502F0011124E556F24F80819181A28104
:105DB000B3818093501C9093511CA093521CB093BC
:105DC000531C80E50E94D844882319F00E9449445E
:105DD00003C080E50E948F4486E40E94D844882353
:105DE000D9F00E9458446B017C0120E030E0A90109
:105DF0000E94E0FA181684F420E030E040E752E414
:105E0000C701B6010E9496F960933B0270933C0271
:105E100080933D0290933E020E9436BB0C94C33E99
:105E2000109378040C94C33E27E5222E22E0322EF4
:105E300038E0E32E3BE0F32E63E574E079A768A732
:105E400047E6C42E44E0D42E00E010E0D1018D914D
:105E50001D010E94D844882309F44BC00E94584475
:105E60002B013C01133049F0F60120813181428140
:105E700053810E94B9F82B013C01A8A5B9A52D9129
:105E80003D914D915C91C301B2010E94B9F84B0163
:105E90005C012DEB37E346E855EB0E94E0FA87FD05
:105EA0000AC02DEB37E346E855E3C501B4010E9473
:105EB0003DF41816F4F4133051F440925F045092FC
:105EC0006004609261047092620401E012C0A50156
:105ED0009401F70160817181828193810E94BAF8F7
:105EE000D7016D937D938D939C931397812F0E947F
:105EF000879B1F5FB4E0EB0EF11CE8A5F9A5349673
:105F0000F9A7E8A7F4E0CF0ED11C143009F09ECF1A
:105F1000002309F4F6CE8FE594E00E94FBDBF1CE7E
:105F20000E94F1DC0C94C33E80918D1390918E13EE
:105F30008637910511F40C9403380CF0C5C08C34ED
:105F4000910509F4FDC40CF058C08931910509F49C
:105F5000DDC21CF58431910509F4C6C17CF48131A0
:105F6000910509F447C22CF4029708F4C0C10C94BF
:105F7000723E429709F4D9C60C94723E863191055F
:105F800009F47EC20CF478C28731910509F47EC20F
:105F9000489709F491C20C94723E8E31910509F430
:105FA00073C384F48B31910509F4CCC20CF4BCC2E8
:105FB0008C31910509F45EC34D9711F40C94C33EE6
:105FC0000C94723E8A32910509F461C44CF48F310D
:105FD000910509F437C4809709F4E8C30C94723E24
:105FE0008133910509F487C48B34910511F00C9429
:105FF000723E0E9453C20C94C33E8A36910509F446
:10600000C7C58CF58335910509F48BC69CF48E3495
:10601000910509F49DC40CF497C48135910509F4E8
:106020006EC68235910511F00C94723E1092770481
:106030000C94C33E8C35910509F4C3C654F48435E1
:10604000910509F472C68535910509F4A1C60C9431
:10605000723E8836910509F47FC48936910509F4AA
:1060600037C50C94723E8F36910509F4B1C48CF497
:106070008C36910511F40C94C33E0CF4A7C58D36F3
:10608000910509F467C58E36910509F48EC40C9408
:10609000723E8237910509F41CC75CF48037910584
:1060A00011F40C94C33E8137910509F4E4C40C94B7
:1060B000723E8337910509F414C18537910511F4B7
:1060C0000C94C33E0C94723E8F3221E0920711F47F
:1060D0000C94813C0CF073C08B3C910511F40C9432
:1060E000C8388CF58C38910509F438C584F48837A4
:1060F000910509F4D8C70CF4D3C78937910509F481
:10610000D8C78D37910509F473C50C94723E8E3B48
:10611000910509F439C534F48B39910509F4F3C4B8
:106120000C94723E883C910509F4C8C7893C9105DE
:1061300011F00C94723EB7E5EB2EB2E0FB2E0EEBA5
:1061400014E10C94AE388C3D910511F40C94C13AD5
:10615000B4F48D3C910511F40C94593914F40C9459
:10616000E4388E3C910511F40C94D839833D9105A7
:1061700011F00C94723E0E942A730C94C33E8C3230
:1061800051E0950711F40C94653B64F48D3D910545
:1061900011F40C94CE3A823E910511F40C943C3BE0
:1061A0000C94723E8D3271E0970711F40C948E3B83
:1061B0008E32914011F40C942E3C0C94723E873F29
:1061C000B1E09B0711F40C94213D0CF044C0843ADB
:1061D000F1E09F0711F40C94153DD4F4833641E0AF
:1061E000940709F47AC03CF48033914011F40C9484
:1061F000843C0C94723E803971E0970711F40C9442
:10620000123D8A39914011F40C94C33E0C94723EB5
:10621000843FB1E09B0711F40C941B3D6CF4853A6C
:10622000F1E09F0711F40C94183D8C3A914011F461
:106230000C94FB390C94723E853F41E0940711F4B5
:106240000C941E3D863F914011F00C94723E0E94CA
:1062500033D30C94C33E8A3962E0960711F40C9450
:10626000DF3DDCF48C30A2E09A0711F40C944E3D33
:106270003CF4883F914011F40C942A3D0C94723EFA
:106280008835F2E09F0711F40C94573D8B3592400E
:1062900011F40C945A3D0C94723E8B3843E09407F1
:1062A00011F40C94C33E6CF4883763E0960711F444
:1062B0000C940A3E8438934011F40C940D3E0C94D7
:1062C000723E803AA3E09A0709F4AFC2873E93403A
:1062D00011F40C94623E0C94723EEFEEF6E20C94D4
:1062E000FF3CE1EDFBE034C6E2E3FAE087C0A090BA
:1062F0008B13B0908C1380E50E94D844882359F00A
:106300000E940E9C6B017C0111E0672B682B692BAE
:1063100031F410E004C010E0C12CD12C760183E5EB
:106320000E94D844882311F40C94CD3E0E94584416
:1063300020E030E04AE754E40E94A2F40E9403FA0D
:106340006B017C0111110BC0672B682B692B39F491
:10635000A114B10421F0F5018081811102C010E087
:1063600001C011E00E94938D1123B9F0E4E0F7E23F
:1063700084918F010F5F1F4F882321F00E94009DA1
:10638000F801F6CFD5018D915D01882319F00E94A7
:10639000009DF8CF8AE00E94009D83E08093FC1B63
:1063A00081E080934004C114D104E104F104B1F010
:1063B0000E942E99C60ED71EE81EF91E0E942E9925
:1063C000DC01CB018C199D09AE09BF09B7FF0EC0D6
:1063D0008091400481110C94D23E08C08091400409
:1063E000882321F080E00E946DA4F8CF1092400431
:1063F0000C94C33E0E947CAA0C94C33E84918F01EE
:106400000F5F1F4F882321F00E94009DF801F6CFF7
:106410001092611084E19EE00E94E9AC8BE1E4E11E
:10642000FEE0DE01159601900D928A95E1F78091CC
:10643000120E9091130E9C838B8385EF92E09A83CA
:10644000898340E050E0BE016F5F7F4F80E090E0C5
:106450000E945DB5CE0101960E9406A4E3E2FAE037
:1064600084918F010F5F1F4F882311F40C94C33E5A
:106470000E94009DF801F4CF0E946BB30C94C33EC0
:106480001092E30D1092E40D0C94C33EE0918B1337
:10649000F0918C138081882329F0803209F41082D6
:1064A0003196F8CF40E061E080918B1390918C138E
:1064B0000E9431D80C94C33E80E090E0A0E0B0E4AC
:1064C00089839A83AB83BC8318A219A21AA21BA248
:1064D0001CA21DA21EA21FA28091560B882359F058
:1064E00020E0AE014F5F5F4FBE01605E7F4FCE0187
:1064F00084960E94A1DE8091E40D882319F081E04A
:106500008093E30D0E9453C20C94C33E1092E30D9E
:106510000E94CFE583E49AE09093EE1B8093ED1BFD
:106520000E94B19D0C94C33E8091E40D882311F428
:106530000C94C33E83E50E94D84481110C94D73E4D
:106540000C94C33E83E40E948F44882309F450C016
:10655000E5E7FAE084918F010F5F1F4F882321F058
:106560000E94009DF801F6CF8091AF0F811103C00A
:10657000E8E4FAE012C0BE016F5F7F4F8CEA9FE053
:106580000E94B1AB8E010F5F1F4FF80181918F0107
:10659000882349F10E94009DF8CF84918F010F5FFD
:1065A0001F4F882301F10E94009DF801F6CF9DEC5A
:1065B000C92E9AE0D92EE12CF12C20E080912A06F8
:1065C00090E00E2C02C0959587950A94E2F780FD25
:1065D0002FC2EFEFEE1AFE0AF2E0CF0ED11C45E01B
:1065E000E416F10459F78AE00E94009D0C94C33E22
:1065F0008091E40D882339F08091E30D882319F010
:10660000E2E5FAE003C0E4E6FAE028C084918F01F5
:106610000F5F1F4F882321F00E94009DF801F6CFE5
:1066200060915D1070915E1080915F10909160108C
:106630004AE00E948CA08FE20E94009D6091591058
:1066400070915A1080915B1090915C104AE00E940A
:106650008CA08AE00E94009D0C94C33E84918F011F
:106660000F5F1F4F882311F40C94C33E0E94009DBE
:10667000F801F4CF40E060E080918B1390918C138F
:106680000E9431D80C94C33E8091E40D882311F40C
:106690000C94C33E8CEA9FE00E94BFE38CEA9FE02B
:1066A0000E948CAB1092E20D1092E10D8091E40DEE
:1066B000882311F40C94C33E00918B1310918C131A
:1066C0000E94A3B4B801CE0180960E9475D78C01B8
:1066D000892B11F40C94C33E68A179A16115710551
:1066E00011F06C5F7F4F19821C8222E0A801CE015D
:1066F00001960E941EB1811102C0F12C14C0CE017E
:1067000001960E94CBB48823C1F361E0CE010196CB
:106710000E9495AB009789F325EEDC012C931C8237
:106720000E9468E1F82ECE0101960E94FA9CF110B9
:1067300003C0E2E9FAE022C0E4E8FAE084917F01D4
:10674000BFEFEB1AFB0A882321F00E94009DF7019E
:10675000F5CFF80181918F01882319F00E94009DE7
:10676000F8CF8AE00E94009D10925D1010925E109A
:1067700010925F10109260100C94C33E84917F01C0
:106780002FEFE21AF20A882321F00E94009DF70100
:10679000F5CFD8018D918D01882319F00E94009DBD
:1067A000F8CF8EE20E94009D0C94C33E8091E30DD1
:1067B00081110E94938D8091E40D882311F40C9433
:1067C000C33E80E50E94D844882319F00E944944C2
:1067D00003C080E50E948F44182F482F61E080910C
:1067E0008B1390918C130E9431D883E50E94D8447A
:1067F000882381F00E942844AB01BC0140935D10C6
:1068000050935E1060935F10709360108CEA9FE06D
:106810000E94A2AA8091E40D882319F081E0809360
:10682000E30D11110C94C33E6DCE80918B139091AA
:106830008C1321E02093E20D40E060E00E9431D80B
:106840000C94C33E0E9480E568A379A38AA39BA30E
:10685000BE016F5F7F4FCE0180960E941E9CE4E0D8
:10686000F7E284918F010F5F1F4F882321F00E9470
:10687000009DF801F6CFBE016F5F7F4F8AEA9AE074
:106880000E9438C28AE00E94009D0C94C33E83E5BA
:106890000E94D844882311F40C94C33E0E943844CB
:1068A000E82E80E50E94D844882339F00E943844BD
:1068B000182F87FF03C00C94C33E1DE089E40E949B
:1068C000D844882341F00E94494481110C944F3FE1
:1068D000E9E3FDE00BC089E40E948F44F6CF3196D6
:1068E000BDE0E936FB0711F40C944F3F8491181377
:1068F000F6CF0C94233FF090730481E0F826F092D9
:106900007304E2ECFAE084918F010F5F1F4F88233C
:1069100021F00E94009DF801F6CFFF2019F0E7EB6F
:10692000FAE002C0ECEBFAE084918F010F5F1F4F99
:10693000882311F40C94C33E0E94009DF801F4CF0B
:106940000E94CFE50C94C33E0E949AC20C94C33EB1
:106950000E94D5760C94C33E88E690E00E94509D3C
:1069600081110C94C33E80912A0683FF02C00C94CF
:10697000C33E83E50E94D844882399F00E9458447E
:106980000E94FEF9CB010E94E75F0E94584420E07C
:1069900030E04AEA52E40E943DF4181614F00E94D6
:1069A0009AC20E944BC40C94C33E8EE40E94D84409
:1069B000882311F40C94C33E0E9428446093F11B79
:1069C0007093F21B8093F31B9093F41B0C94C33EC3
:1069D00083E50E948F44882359F083E50E94D844C0
:1069E000882319F00E94384401C080E080932A0671
:1069F000E4E0F7E284918F010F5F1F4F811103C024
:106A0000EBEDFAE004C00E94009DF801F3CF849101
:106A10008F010F5F1F4F882321F00E94009DF80116
:106A2000F6CF80912A068111C2CDE7EDFAE018C0B9
:106A3000BB24B394B20E222319F08CE20E94009D75
:106A4000F60185919491FC0184918F010F5F1F4F96
:106A5000882321F00E94009DF801F6CF2B2DB9CD9F
:106A600084918F010F5F1F4F882309F4BCCD0E94D2
:106A7000009DF801F5CF83E50E94D844811103C041
:106A8000E4E0F7E20DC00E9438448D3320F4809397
:106A900028020C94C33E8CE3809328020C94C33EDE
:106AA00084918F010F5F1F4F882321F00E94009D6A
:106AB000F801F6CF4091280250E060E070E082EEED
:106AC0009AE00E94E5C18AE00E94009D0C94C33EBA
:106AD00089E690E00E94509D811111C0E9EEFAE034
:106AE00084918F010F5F1F4F882321F00E94009D2A
:106AF000F801F6CF0E94955E8AE00E94009D1092F8
:106B0000FC1B0C94643F83E50E94D844882311F455
:106B10000C94C33E0E943844182F8D3308F01CE3B8
:106B20001093070B0E942E996B017C01212F30E0FE
:106B3000A8EEB3E00E94AAF8C60ED71EE81EF91E02
:106B4000C092030BD092040BE092050BF092060B5F
:106B50000C94C33E0E945B7B0C94C33E80912A063A
:106B600083FF02C00C94C33E83E50E94D84488236F
:106B700011F40C94C33E0E9458440E94FEF9CB01CC
:106B80000E9467460C94C33E0E9409750C94C33E54
:106B900080E50E94D844811106C083E50E94D84454
:106BA000882361F006C00E94384481110C94C33ED2
:106BB000F4CF0E9428446F3F710510F06FEF70E032
:106BC0007093550B6093540B0C94C33E80E50E9468
:106BD000D844811106C01092550B1092540B0C949E
:106BE000C33E0E942844672B11F00C94C33EF3CFA0
:106BF0008CE40E948F44882381F00E9458446B01EA
:106C00007C0120E030E0A9010E94E0FA87FF0BC080
:106C1000F7FAF094F7F8F09406C0C12CD12C80E874
:106C2000E82E80E4F82EF7FAF094F7F8F094CCA26E
:106C3000DDA2EEA2FFA280E090E0A0EAB0E48983AA
:106C40009A83AB83BC8380E090E0ADE4B3E48D83B2
:106C50009E83AF83B88780E090E0A0EAB1E48987A3
:106C60009A87AB87BC8788E50E94D844882379F04F
:106C700088E50E94D844882319F00E94584403C034
:106C800060E070E0CB0169837A838B839C8389E524
:106C90000E94D844882379F089E50E94D84488234B
:106CA00019F00E94584403C060E070E0CB016D838E
:106CB0007E838F8398878AE50E94D844882379F061
:106CC0008AE50E94D844882319F00E94584403C0E2
:106CD00060E070E0CB0169877A878B879C8718A278
:106CE00019A21AA21BA2AE01405E5F4FBE016F5FE8
:106CF0007F4FCE0184960E944EA90C94C33E0E9401
:106D0000F75F0E94BCC61092550B1092540B68EEB0
:106D100073E080E090E00E9471670E944B180C9431
:106D2000C33E109377040C94C33E83E50E94D8447D
:106D30008823A1F00E94584420E030E04AE754E460
:106D40000E94A2F40E9403FA6093290270932A021F
:106D500080932B0290932C020C94C33E88E50E94F2
:106D60008F4481110C94E73E89E50E948F44811184
:106D70000C94E73E8AE50E948F4481110C94E73E13
:106D800085E40E948F4481110C94E73E0C94153FDA
:106D900083E50E948F44882309F4F5C70E94584474
:106DA00020E030E04AE754E40E94A2F40E9403FA93
:106DB0006093FF0A7093000B8093010B9093020B7A
:106DC000E2C717E5C12E12E0D12E0CE2E02E0CE155
:106DD000F02E10E0D6018D916D010E948F44882322
:106DE00009F46DC0133009F063C00E9458444B0190
:106DF0005C0120E030E040EA51E40E943DF487FF6E
:106E00004EC0A50194016091381C7091391C80918D
:106E10003A1C90913B1C0E9496F92B013C019B016E
:106E2000AC016091FE057091FF0580910006909184
:106E300001060E94A2F46093FE057093FF05809303
:106E4000000690930106A301920160911A067091C9
:106E50001B0680911C0690911D060E94A2F460936F
:106E60001A0670931B0680931C0690931D06609172
:106E7000BA147091BB148091BC149091BD140E94FF
:106E800041F4A30192010E94A2F40E9403FA6093CC
:106E9000BA147093BB148093BC149093BD14809269
:106EA000381C9092391CA0923A1CB0923B1C07C02F
:106EB0000E945844F70160837183828393831F5F2C
:106EC000F4E0EF0EF11C143009F084CF0E94ECC501
:106ED0005AC70E94938D83E50E94D844882311F4F9
:106EE0000C94812E0E9428446230710511F00C949C
:106EF000812E0E9410BF8BE50E94009D609192142C
:106F000070919314809194149091951442E00E9492
:106F100011A140919614509197146091981470911A
:106F200099148FEE9AE00E9402C240919A145091F7
:106F30009B1460919C1470919D148CEE9AE00E94B9
:106F400002C28DE50E94009D8AE00E94009D1BC741
:106F500084918F010F5F1F4F882321F00E94009DB5
:106F6000F801F6CF60E081EC9BE00E94087461E0DC
:106F70008AEB9BE00E94087461E08FEA9BE00E942C
:106F8000087461E08FE99BE00E94087460E086E984
:106F90009BE00E94087461E08CE89BE00E9408740A
:106FA00060E082E89BE00E94087460E08AE79BE072
:106FB0000E94087461E08CE69BE00E94087460E027
:106FC0008EE59BE00E94087460E08FE49BE00E94E5
:106FD000087460E081E49BE00E94087460E08BE24A
:106FE0009BE00E94087461E08AE19BE00E940874C3
:106FF00060E085E09BE00E94087461E082EF9AE027
:107000000E940874C0C600918B1310918C1383E00A
:10701000D12C40E08150E9F0D8019C91292F2B7FA1
:107020002134C1F711962C912133A1F7913421F02D
:10703000953421F441E002C0DD24D39498012E5F01
:107040003F4F89012F5F3F4FF80190819032C9F384
:10705000E1CF442369F0E4E0F7E284917F012FEF70
:10706000E21AF20A882321F00E94009DF701F5CF71
:10707000DD2069F0E7ECFCE084917F014FEFE41A3A
:10708000F40A882321F00E94009DF701F5CFD80172
:107090008D918D01882309F4A6CA0E94009DF7CF27
:1070A0000E941BCE70C681E080934B0680934A06F7
:1070B0006AC610924B0610924A0665C688EC90E0AC
:1070C0000E94509D81115FC684E40E948F448823F2
:1070D00009F441C00E9458446B017C0111E020E09A
:1070E00030E0A9010E943DF4811101C010E010932D
:1070F000CE1B20E030E0A901C701B6010E943DF49B
:10710000882349F10E945844E0919205B4E0EB9F36
:10711000F0011124ED52F44E6083718382839383D6
:1071200020E030E0A9016091D31B7091D41B8091C5
:10713000D51B9091D61B0E943DF481110CC080E0BC
:1071400090E0A0EEBFE38093D31B9093D41BA09359
:10715000D51BB093D61B0E94FBC615C6F7018191C3
:107160007F010E948F44882351F00E9458440E945E
:1071700003FAD8016D937D938D939C9313970C5FC5
:107180001F4FB4E10E3C1B0749F70E947BC4FBC5AF
:10719000A7E5EA2EA2E0FA2E0EE016E0F7018191B3
:1071A0007F010E948F44882341F00E945844D801F7
:1071B0006D937D938D939C9313970C5F1F4FB6E057
:1071C0000E311B0759F7DFC583E50E94D844882399
:1071D000A1F00E94584460930A0670930B068093B6
:1071E0000C0690930D066093060670930706809335
:1071F00008069093090610E001C011E080E50E94A6
:10720000D844882359F00E94584460930A0670932A
:107210000B0680930C0690930D0610E082E50E9409
:10722000D844882359F00E9458446093F81B709307
:10723000F91B8093FA1B9093FB1B10E084E50E94DE
:10724000D844882359F00E945844609306067093EE
:107250000706809308069093090695C5112309F443
:1072600092C540910A0650910B0660910C067091F0
:107270000D0681ED9CE00E9402C24091F81B5091E6
:10728000F91B6091FA1B7091FB1B8EEC9CE00E9435
:1072900002C240910606509107066091080670915F
:1072A00009068BEC9CE00E9402C28AE00E94009DCD
:1072B0006AC581E50E948F44882351F00E940E9C8C
:1072C00060931E0670931F068093200690932106FC
:1072D00083E50E948F44882351F00E9458446093B4
:1072E000260670932706809328069093290684E546
:1072F0000E948F44882351F00E94584460932206D4
:1073000070932306809324069093250688E50E94B7
:107310008F44882351F00E9458446093F205709383
:10732000F3058093F4059093F50589E50E948F4459
:10733000882351F00E9458446093F6057093F70536
:107340008093F8059093F9058AE50E948F4488237D
:10735000F1F00E9458446093FA057093FB05809306
:10736000FC059093FD052DEC3CEC4CEC5DE30E949C
:107370003DF4181664F0E1EEFCE084918F010F5F9C
:107380001F4F882321F00E94009DF801F6CF85E46D
:107390000E948F44882309F4F6C40E9458446093E5
:1073A000FE057093FF058093000690930106EBC4E1
:1073B000E7E5CE2EE2E0DE2EFCE4EF2EF6E0FF2E37
:1073C00010E0F60181916F010E948F44882359F0EB
:1073D0000E945844D7016D937D938D939C9313978E
:1073E000812F0E94879B1F5FB4E0EB0EF11C1330CE
:1073F00041F70C94812E0E94CBD68111C4C40CE1BC
:1074000016E2E3E5F4E0F9A7E8A7AE014F5F5F4FAE
:107410004A0175E7A72E76E2B72E1A01F8016591A9
:10742000759185919491A8A5B9A5CD90DD90ED9029
:10743000FD90B9A7A8A7A70196010E94B9F82B0152
:107440003C01F101608371838283938320E030E00B
:1074500040EA51EC0E94E0FA87FD0AC020E030E0EB
:1074600040EA51E4C301B2010E943DF418162CF425
:10747000F501849118160CF4DBC4D101CD90DD9098
:10748000ED90FD901D0120E030E040EA51ECC70195
:10749000B6010E94E0FA87FD0AC020E030E040EA31
:1074A00051E4C701B6010E943DF418164CF5EFEE09
:1074B000F6E284918F010F5F1F4F811103C0E3E15A
:1074C000FDE004C00E94009DF801F3CF84918F017C
:1074D0000F5F1F4F882321F00E94009DF801F6CF17
:1074E00088E290E099A388A388EC90E09DA38CA308
:1074F000BE01605E7F4FCE0184960E94C2D443C419
:107500000C5F1F4FBFEFAB1ABB0AE8E2F6E2E017D1
:10751000F10709F083CF6CE4E62E66E0F62E10E06A
:10752000F40181919191A191B1914F01F701819362
:107530009193A193B1937F01812F0E94879B1F5F3D
:10754000133071F70E943F7483E992E09DA38CA3EE
:1075500004E610E019A308A3BE016C5D7F4FCE01C5
:1075600080960E94C2D48AEB92E09DA38CA319A3BB
:1075700008A3BE016C5D7F4FCE0180960E94C2D4ED
:1075800002C483E50E94D844882309F4FCC30E9406
:1075900028447093010260930002F5C38DED90E0E2
:1075A0000E94509D8111EFC383E50E94D844811150
:1075B00003C0E4E0F7E23AC00091920510E00E94B7
:1075C0002844000F111FF801E15BFD4F71836083B8
:1075D0008091920590E07C01EE0CFF1CEE0CFF1CEC
:1075E0008701025E1D4F880F991FFC01E15BFD4F73
:1075F00060817181072E000C880B990B0E9443F467
:107600002AE037ED43E25CE30E94A2F4F701E15384
:10761000F44E20813181428153810E94A2F4D8012D
:107620006D937D938D939C931397ADC384918F013C
:107630000F5F1F4F882321F00E94009DF801F6CFB5
:1076400085E40E94009D80919205805D0E94009DCE
:10765000E0919205F0E0EE0FFF1FE15BFD4F6081CE
:10766000718181E39DE00E941FC285E20E94009D1E
:107670008AE00E94009D87C380E50E948F44882392
:1076800009F481C30E9428446B017C0183E50E94B8
:10769000D844882321F00E9428448B0102C00FEFB8
:1076A0001FEFC8010196039708F06DC3D7FC6BC3A9
:1076B0008C2DE9E3FDE09491891709F4C4C3319658
:1076C000BDE0E936FB07B9F7C1C383E50E94D844A2
:1076D000882319F00E94284402C064E071E079A375
:1076E00068A380E50E94D844882339F00E9428448A
:1076F0006938E3E17E0730F402C068EE73E07A8314
:10770000698304C088E893E19A838983BE01605E3F
:107710007F4FCE0101960E94C2D435C385E40E94FA
:10772000D844811110C080E50E948F44882391F0D5
:107730000E94584460937B0570937C0580937D057F
:1077400090937E0507C00E943844882361F3EFEED2
:10775000F6E271C089E40E948F44882381F00E9480
:1077600058442CEA35EC47E25EE30E94A2F46093B1
:107770007705709378058093790590937A0584E472
:107780000E948F44882381F00E9458442CEA35ECF3
:1077900047E25EE30E9496F960937F05709380054F
:1077A0008093810590938205E4E0F7E284918F0154
:1077B0000F5F1F4F882321F00E94009DF801F6CF34
:1077C00040917B0550917C0560917D0570917E050F
:1077D00081E79DE00E9402C22CEA35EC47E25EE3BD
:1077E00060917705709178058091790590917A057F
:1077F0000E9496F9AB01BC018DE69DE00E9402C299
:107800002CEA35EC47E25EE360917F0570918005DC
:1078100080918105909182050E94A2F4AB01BC0188
:1078200089E69DE00E9402C28AE00E94009DABC2F0
:107830000E94009DF80184918F010F5F1F4F8111FD
:10784000F7CFE5E7FDE084918F010F5F1F4F88239D
:1078500009F499C20E94009DF801F5CF83E50E94CA
:107860008F44182F882371F00E9458440E94FEF91B
:10787000709352026093510221E0672B09F020E0DF
:1078800020930D1C80E50E948F44882351F02091A5
:10789000510230915202232B09F0FBD780930D1C2B
:1078A00072C2111170C2E4E0F7E284918F010F5FA0
:1078B0001F4F882321F00E94009DF801F6CF809190
:1078C0000D1C882319F061E274E002C064E274E0E8
:1078D0008CE99DE00E9438C2609151027091520281
:1078E0008BE89DE00E941FC2E7E8FDE084918F01D4
:1078F0000F5F1F4F882309F446C20E94009DF801C4
:10790000F5CF0E94CE6B3FC280E50E948F44882352
:1079100049F0CED760937305709374058093750515
:107920009093760589E4FBD7882379F0C1D72CEAB8
:1079300035EC47E25EE30E94A2F460936F0570931A
:107940007005809371059093720584E4E8D78823CD
:1079500079F0AED72CEA35EC47E25EE30E9496F967
:1079600060936B0570936C0580936D0590936E0525
:10797000E4E0F7E284918F010F5F1F4F882321F02D
:107980000E94009DF801F6CF409173055091740557
:10799000609175057091760587EB9DE00E9402C2AB
:1079A0002CEA35EC47E25EE360916F05709170055B
:1079B00080917105909172050E9496F9AB01BC010E
:1079C00083EB9DE00E9402C22CEA35EC47E25EE3C5
:1079D00060916B0570916C0580916D0590916E05BD
:1079E0000E94A2F4AB01BC018FEA9DE00E9402C29A
:1079F0008AE00E94009DC7C10E94009DF801849109
:107A00008F010F5F1F4F8111F7CFEBEBFDE08491EA
:107A10008F010F5F1F4F882309F4B5C10E94009D9D
:107A2000F801F5CF0E94938DAEC10E94CA69ABC127
:107A30000E94DF68A8C10E940C94A5C10E94009416
:107A4000A2C183E56CD7882311F023D781270E9438
:107A500050CE99C181E0809331060E94C58D10926D
:107A60003106882309F48FC1E4E0F7E284918F01A5
:107A70000F5F1F4F811103C0EAECFDE004C00E94BC
:107A8000009DF801F3CF84918F010F5F1F4F882372
:107A900009F479C10E94009DF801F5CF8091E30DB2
:107AA000882309F470C181E08093E60D6CC10E94C7
:107AB000387169C18BE592E00E94509D811163C1CC
:107AC00085E52DD78823D1F10091920510E0F0D6FD
:107AD0006B017C0120E030E0A9010E94E0FA87FF01
:107AE00004C0F7FAF094F7F8F094000F111F000F9C
:107AF000111FF801E052F44EC082D182E282F3827B
:107B000000919205F4E00F9F800111240052144E61
:107B100020E030E046E154E4D8016D917D918D91F3
:107B20009C910E94E0FA18164CF480E090E0A6E1E7
:107B3000B4E4F80180839183A283B3838CE4EFD60D
:107B4000882309F420C10091920510E0B1D66B01A1
:107B50007C0120E030E0A9010E94E0FA87FF04C028
:107B6000F7FAF094F7F8F094000F111F000F111FAF
:107B7000F801EC51F44EC082D182E282F38200918E
:107B80009205F4E00F9F800111240C51144E20E067
:107B900030E046E154E4D8016D917D918D919C9146
:107BA0000E94E0FA18160CF0EEC080E090E0A6E12A
:107BB000B4E4F80180839183A283B383E4C08AE5AF
:107BC000F7D6811103C0E8EDFDE00AC071D66093DD
:107BD000E81B7093E91B8093EA1B9093EB1BD3C0C7
:107BE00084918F010F5F1F4F882321F00E94009D19
:107BF000F801F6CF4091E81B5091E91B6091EA1B18
:107C00007091EB1B85ED9DE00E9402C28AE00E940C
:107C1000009DB9C00E949367B6C08BE4C9D681119C
:107C200003C0E4E0F7E234C08BE4C2D68823B9F0A5
:107C30003FD66B017C0120E030E0A9010E94E0FA10
:107C400087FD0AC020E030E040E251E4C701B60100
:107C50000E943DF4181634F4E7EFFDE00EC0C12C8D
:107C6000D12C76010E94938DC0920206D092030619
:107C7000E0920406F092050686C084918F010F5FA2
:107C80001F4F882309F47FC00E94009DF801F5CFA3
:107C900084918F010F5F1F4F882321F00E94009D68
:107CA000F801F6CF40910206509103066091040658
:107CB0007091050686E19EE00E9402C28AE00E9461
:107CC000009D61C081E08093190283E571D688230D
:107CD00031F0DFD5811157C00E9446BF54C083E503
:107CE0001ED6F8CF0E94F1DC4EC0F0908D130E949A
:107CF000938D1091171C80E00E94E299FF2029F1DA
:107D0000E4E0F7E284918F010F5F1F4F882321F099
:107D10000E94009DF801F6CF84E50E94009D6F2D22
:107D200070E080E090E04AE00E948CA080E20E9437
:107D3000009DE3E3FEE084918F010F5F1F4F8823D6
:107D400011F10E94009DF801F6CF1092200B812FB7
:107D50000E94E299E4E0F7E284918F010F5F1F4FE8
:107D6000882321F00E94009DF801F6CF6091200B3E
:107D700070E081E29EE00E941FC28AE00E94009DA6
:107D800002C00E94F1DC1092FC1B0E9429BF9CC023
:107D90000E94DD790E9436BBF6CF11110C94AF31F1
:107DA0000C94A83180E00E946DA40C94DE3150D573
:107DB000AB01BC0140935D1050935E1060935F1067
:107DC000709360108CEA9FE00E94A2AADCCF0E9410
:107DD000938D88E5A4D5882331F05F9A809149047A
:107DE0008E7F8093490489E59AD5882339F08A9A51
:107DF000479A809149048D7F809349048AE58FD505
:107E0000882361F08091080180958170809306013C
:107E1000479A809149048B7F8093490485E47FD5FC
:107E2000882309F4B0CF129AAECF0E94BCC6ABCF64
:107E3000F7FAF094F7F8F094D101CD92DD92ED923B
:107E4000FC9213971ACB0E94CAE79DCF0E94938D94
:107E5000BC2C60E08C2D0E9464DD0F3FBFEF1B0740
:107E600059F48C2D0E940EDD31E020E0892B09F0C1
:107E700030E0032F122F05C00130110569F401E035
:107E800010E08B2D0E940EDD8017910709F47BCF47
:107E900080E00E946DA4F5CF00E010E0F2CF61E039
:107EA000812F0E9464DD6E2D812F0E9436DDF12C22
:107EB000B701812F0E94A0DD193009F064CFF09244
:107EC000550BE092540B5FCFCD5BDF4F0FB6F894AC
:107ED000DEBF0FBECDBFDF91CF911F910F91FF90FD
:107EE000EF90DF90CF90BF90AF909F908F907F905A
:107EF0006F905F904F903F902F9008950F931F9336
:107F0000CF93DF93FC01A685B7858D0100581F4FE5
:107F1000E8018881998101968F779927AD014E57A5
:107F20005F4FEA012881398128173907D1F3E80129
:107F300028813981A20FB31F6C93A685B785A058FD
:107F4000BF4F11969C938E93A689B7892C9181E09F
:107F500090E0078C02C0880F991F0A94E2F7822BE9
:107F60008C9381E081A30488F589E02D8081806471
:107F7000808381E090E0DF91CF911F910F91089570
:107F8000FC0181A1882329F0A489B5898C9186FF01
:107F9000FBCF11A20895FC01A485B585FD01E05831
:107FA000FF4F2081318132968081918128173907D6
:107FB00079F080819181A80FB91F8C912081318146
:107FC0002F5F3F4F2F7733273183208390E0089531
:107FD0008FEF9FEF0895DC011C96ED91FC911D97AA
:107FE000DF01A058BF4F2D913C91119712968D91B2
:107FF0009C9111972817390739F08D919C91E80FC2
:10800000F91F808190E008958FEF9FEF0895FC01A4
:1080100024853585F901E058FF4F808191813296A2
:108020002081318180589F4F821B930B60E870E064
:108030000C94A3FB0895089580E090E00895CF92FA
:10804000DF92EF92FF92C0903B02D0903C02E09012
:108050003D02F0903E02FC0180819181A281B381BA
:1080600080933B0290933C02A0933D02B0933E026A
:108070000E9436BBC0923B02D0923C02E0923D028D
:10808000F0923E02FF90EF90DF90CF9008952F92F4
:108090003F924F925F926F927F928F929F92AF9298
:1080A000BF92CF92DF92EF92FF920F931F93CF93E5
:1080B000DF9300D000D0CDB7DEB79A8389830E94CA
:1080C0002E99E981FA81C680D780E084F184C114B9
:1080D000D104E104F10409F0ACC22485222309F49F
:1080E00069C332852150248721E0230F22874585EB
:1080F000241301C01286E981FA8124E0329FE00D49
:10810000F11D1124C684D784E088F188E981FA81C1
:10811000C282D382E482F582DC01CB018C0D9D1DED
:10812000A11DB11D86839783A087B1878481958126
:10813000892B09F43FC3FFB7FD83F894E981FA81E5
:10814000228033802101612C712C04811581809162
:108150001D028F3121F08F3F09F068C205C0E9EBA5
:10816000FCE124912E83DAC08FE180931D02E9EBBC
:10817000FCE184918E838F3F09F458C2823009F468
:1081800069C030F5882309F44CC0813009F0C6C0BD
:10819000109280001092810080918100886080930D
:1081A000810080918100816080938100EFE1FFE296
:1081B000E491F0E0EE0FFF1FE453F14D85919491AF
:1081C000E5E6FFE2E491E0938A04E1E0EE8330C16A
:1081D0009E81943009F482C008F460C0953009F0A3
:1081E0009DC0109220011092210180912101886090
:1081F0008093210180912101816080932101EFE131
:10820000FFE2E491F0E0EE0FFF1FE453F14D8591A2
:108210009491E5E6FFE2E491E093870495E09E8384
:1082200007C114BC15BC84B5826084BD85B581606E
:1082300085BDEFE1FFE2E491F0E0EE0FFF1FE453B4
:10824000F14D85919491E5E6FFE2E491E0938B0492
:108250001E82ABC21092B0001092B1008091B000AB
:1082600082608093B0008091B10081608093B10002
:10827000EFE1FFE2E491F0E0EE0FFF1FE453F14D78
:10828000859194919093940580939305E5E6FFE2A0
:10829000E491E0939505F2E0FE8387C2109290008E
:1082A000109291008091910088608093910080915C
:1082B0009100816080939100EFE1FFE2E491F0E0B2
:1082C000EE0FFF1FE453F14D85919491E5E6FFE237
:1082D000E491E093890423E02E83AAC01092A000C9
:1082E0001092A1008091A10088608093A1008091EC
:1082F000A10081608093A100EFE1FFE2E491F0E052
:10830000EE0FFF1FE453F14D85919491E5E6FFE2F6
:10831000E491E093880484E08E838AC0EE81E7FDD7
:1083200085C161E08FE10E9464DD8E818D7F09F05F
:1083300083C04801A12CB12C60E072E18AE790E093
:10834000A50194010E947EF829833A834B835C83C4
:1083500069017A01F1E0CF1AD108E108F1082FEFA5
:10836000C216D104E104F10409F008F44EC060E43F
:1083700072E48FE090E0A50194010E947EF869010B
:108380007A0181E0C81AD108E108F1089E81923093
:1083900009F5EFEFCE16D104E104F10409F008F479
:1083A000CBC160E970ED83E090E0A50194010E94EB
:1083B0007EF869017A01F1E0CF1AD108E108F108ED
:1083C0002FEFC216D104E104F10411F008F041C10D
:1083D00083E027C08FEFC816D104E104F104B9F09F
:1083E000B0F068E478EE81E090E0A50194010E948D
:1083F0007EF869017A0191E0C91AD108E108F10813
:10840000EE81EE2309F49AC163C181E001C082E0EC
:108410009E81911106C095B5987F892B85BD7AC044
:1084200085E09091B100987F892B8093B10072C054
:1084300061E08FE10E9464DD4801A12CB12C60E075
:1084400072E18AE790E0A50194010E947EF869013B
:108450007A01E1E0CE1AD108E108F108C114D10493
:10846000F1E0EF06F10488F068E478EE81E090E056
:10847000A50194010E947EF869017A0181E0C81A81
:10848000D108E108F10883E001C081E09E819130CC
:1084900071F490918100987F892B80938100452809
:1084A00046284728D9F52FEF3FEFA90168C0EE8194
:1084B000E33071F490919100987F892B8093910023
:1084C00045284628472851F52FEF3FEFA90179C0ED
:1084D000FE81F43071F49091A100987F892B8093F4
:1084E000A100452846284728C9F42FEF3FEFA901EE
:1084F0007AC02E81253071F490912101987F892BCB
:108500008093210145284628472841F42FEF3FEF6B
:10851000A9017BC045284628472869F0D801AA0F41
:10852000BB1F91010E94AAF828EE33E040E050E022
:108530000E945CF803C02FEF3FEFA9018E818230CB
:1085400081F12CF4882361F08130C9F06FC09E81E5
:10855000943009F448C0ACF1953009F456C066C0B7
:10856000C7BC20939C0430939D0440939E04509379
:108570009F0480916E00826080936E0057C0D092FD
:108580008900C09288002093980430939904409306
:108590009A0450939B0480916F00826080936F00D7
:1085A00045C0C092B3002093960530939705409341
:1085B00098055093990580917000826080937000B7
:1085C00035C0D0929900C0929800209394043093C3
:1085D00095044093960450939704809171008260B3
:1085E0008093710023C0D092A900C092A80020936C
:1085F000900430939104409392045093930480919B
:10860000720082608093720011C0D0922901C092E2
:10861000280120938C0430938D0440938E04509352
:108620008F0480917300826080937300ED81EFBFAF
:10863000C1C0DC01CB018C199D09AE09BF09B7FD92
:10864000B9C04698E981FA81168217821086118690
:10865000B1C068E478EE81E090E0A50194010E9449
:108660007EF869017A01F1E0CF1AD108E108F1083A
:108670002FEFC216D104E104F10441F138F164E2B4
:1086800074EF80E090E0A50194010E947EF86901FA
:108690007A01F1E0CF1AD108E108F1082FEFC216F4
:1086A000D104E104F10409F008F4BACE62E17AE7FA
:1086B00080E090E0A50194010E947EF869017A01B2
:1086C00081E0C81AD108E108F10819C084E0A9CEF8
:1086D0002FEFC216D104E104F10409F008F463C0DD
:1086E00062E17AE780E090E0A50194010E947EF8C3
:1086F00069017A01F1E0CF1AD108E108F1082FEF02
:10870000C216D104E104F104A9F0A0F089819A8194
:10871000AB81BC812AE0B595A795979587952A9559
:10872000D1F76C017D01F1E0CF1AD108E108F10821
:1087300087E077CE86E075CE82E073CEEFEFCE167F
:10874000D104E104F10469F160F162E17AE780E0CB
:1087500090E0A50194010E947EF869017A0181E010
:10876000C81AD108E108F1089FEFC916D104E10445
:10877000F104A9F0A0F089819A81AB81BC813AE033
:10878000B595A795979587953A95D1F76C017D0199
:10879000E1E0CE1AD108E108F10885E03CCE84E0A2
:1087A0003ACE83E038CE84E033CE61E08FE10E94A0
:1087B00064DDBFCD26960FB6F894DEBF0FBECDBFE9
:1087C000DF91CF911F910F91FF90EF90DF90CF90AD
:1087D000BF90AF909F908F907F906F905F904F90E1
:1087E0003F902F9008951F920F920FB60F92112471
:1087F0000BB60F922F938F939F93EF93FF938091DC
:10880000700A20916F0A821791F0E82FF0E0E55985
:10881000F54F90818F5F83709093C6008093700AAC
:108820009091C00090649093C000281305C080917F
:10883000C1008F7D8093C100FF91EF919F918F9137
:108840002F910F900BBE0F900FBE0F901F90189599
:108850008091710A9091720A009731F04AE050E0DD
:1088600060E070E00C9491F160E070E0CB0108955D
:10887000EFDF97FD0AC0ECDF6F3F710581059105C1
:1088800009F02CF4E5DF862F089580E008958FEF3E
:1088900008958091710A9091720A892B31F0E8DF76
:1088A00091E0811103C090E001C091E0892F08950B
:1088B0000F931F93CF938091710A9091720A009742
:1088C00011F1FC018F01C1912C2F2F7DA9F0C5342E
:1088D00011F0C536B9F7F801108260E070E08091C0
:1088E000710A9091720A0E943EF0F801C083562FDF
:1088F000472F382F292F0BC060E070E0CF911F91D8
:108900000F910C943EF050E040E030E020E0652F05
:10891000742F832F922FCF911F910F91089581541F
:108920008A3108F042C0E82FF0E04091871350915F
:1089300088136091891370918A1304C076956795A6
:10894000579547958A95D2F7842F817040FF2FC0A5
:10895000E359FC4E9081992309F1E091F61BF091C7
:10896000F71BE90FF11D908120ED290F2A3098F0B7
:108970009E3211F491810CC09D3211F09B3271F442
:10898000918120ED290F2A3030F09E3239F4928106
:1089900090539A3018F42E2F9F2F02C020E090E0C1
:1089A0002093710A9093720A089580E008950895C3
:1089B000B6DF882341F081E02091710A3091720A7C
:1089C000232B09F480E0089580E1E3E5F4E0ACE4D2
:1089D000BCE101900D928A95E1F708952F923F92A4
:1089E0004F925F926F927F928F929F92AF92BF92BF
:1089F000CF92DF92EF92FF920F931F93CF93DF936B
:108A000000D01F921F92CDB7DEB77C018B016A01A7
:108A100019018090530490905404A0905504B09094
:108A20005604A5019401FC016081718182819381CA
:108A30000E943DF4F1E0FD83811112C020915704A2
:108A4000309158044091590450915A04F8016081C2
:108A50007181828193810E943DF4811101C01D8248
:108A6000F601408051806280738020910402309131
:108A700005024091060250910702C301B2010E9413
:108A80003DF4882309F453C0409204025092050239
:108A9000609206027092070220E030E040E450E469
:108AA000609116067091170680911806909119062C
:108AB0000E9496F969837A838B839C8380924C1CF5
:108AC00090924D1CA0924E1CB0924F1C8091570466
:108AD00090915804A0915904B0915A048093501C6D
:108AE0009093511CA093521CB093531CF6018081AB
:108AF0009181A281B3818093541C9093551CA093C3
:108B0000561CB093571C80915F0490916004A09113
:108B10006104B09162048093581C9093591CA093F7
:108B20005A1CB0935B1CCE01019689DA4DDFFD81A2
:108B3000FF2309F1609012067090130680901406CE
:108B400090901506A0900E06B0900F06C0901006EB
:108B5000D09011069501A601B301C4010E94E0FA6C
:108B6000181614F05301640120E030E040E251E4B3
:108B7000B501C6010CC020E030E040EC5FE360913D
:108B80001A0670911B0680911C0690911D060E948A
:108B900096F969837A838B839C83209173042223C3
:108BA00049F0AB01BC0185E49EE00E9402C28AE06C
:108BB0000E94009DF70180819181A281B381809301
:108BC0004C1C90934D1CA0934E1CB0934F1CF8016D
:108BD00080819181A281B3818093501C9093511C1C
:108BE000A093521CB093531CF1012081318142812A
:108BF00053816091581C7091591C80915A1C90911E
:108C00005B1C0E94BAF86093581C7093591C8093A7
:108C10005A1C90935B1CCE01019611DAD5DE0F90A1
:108C20000F900F900F900F90DF91CF911F910F91A8
:108C3000FF90EF90DF90CF90BF90AF909F908F907C
:108C40007F906F905F904F903F902F90089580E1BC
:108C5000ECE4FCE1A3E5B4E001900D928A95E1F724
:108C600008959C0197FD0EC08436910584F064E65A
:108C700070E00E94A3FBCB016AE070E00E94A3FBBE
:108C8000805D06C03195219531098DE201C080E2F9
:108C9000809345042A30310564F0EAE0F0E0C90130
:108CA000BF010E94A3FBCB01BF010E94A3FB805D1B
:108CB00001C080E280934604C9016AE070E00E942E
:108CC000A3FB805D8093470485E494E00895883792
:108CD00091051CF028E780E002C0282F892F2093FF
:108CE0004B0480934C040C944F5F2F923F924F9211
:108CF0005F926F927F928F929F92AF92BF92CF922C
:108D0000DF92EF92FF920F931F93CF93DF93CDB734
:108D1000DEB7C455D1090FB6F894DEBF0FBECDBF84
:108D2000ECEBF1E184918F010F5F1F4F882321F05D
:108D30000E94009DF801F6CF0E94CBD681110C94C1
:108D4000185180E090E0A0E8BFE38093401C90932E
:108D5000411CA093421CB093431C8093481C9093E9
:108D6000491CA0934A1CB0934B1C8AE999E9A9E9D4
:108D7000BFE38093441C9093451CA093461CB09382
:108D8000471C8DEC9CECACE4BEE380933C1C9093C0
:108D90003D1CA0933E1CB0933F1C80E090E0A0EAF5
:108DA000B0E48093110590931205A0931305B0933E
:108DB00014058CE390E09093100580930F0588ECE8
:108DC00090E090930E0580930D0510920C058FE4B2
:108DD000EFDD882311F06CDD04C060E070E080E11D
:108DE00090E46BAF7CAF8DAF9EAF83E4E1DD882371
:108DF00011F04FDD02C083E492DD61968FAF619781
:108E00008BE4D6DD882311F044DD02C08BE487DDDE
:108E100060968FAF609782E4CBDD8823E9F048DD70
:108E20000E94FEF97093100560930F05611571059E
:108E300099F0685271096536710570F0E7E8F1E163
:108E400084918F010F5F1F4F882311F40C941851E8
:108E50000E94009DF801F4CF8CE4AADD882351F133
:108E600027DD6B017C0160933C1C70933D1C80935B
:108E70003E1C90933F1C20E030E0A9010E94E0FAE4
:108E800087FD0AC020E030E040E050E4C701B601B1
:108E90000E943DF4181674F4EFE5F1E184918F011E
:108EA0000F5F1F4F882311F40C9418510E94009DEE
:108EB000F801F4CF81E533DD882309F440C08091C7
:108EC000710A9091720A892B19F4E8E3F1E12BC041
:108ED000EFDC6B017C016093481C7093491C80930C
:108EE0004A1C90934B1C2DEC3CEC4CE45DE30E943F
:108EF000E0FA87FD0AC020E030E040E751E4C70116
:108F0000B6010E943DF41816D4F4EBE0F1E184912F
:108F10008F010F5F1F4F882311F40C9418510E948A
:108F2000009DF801F4CF84918F010F5F1F4F8823BC
:108F300011F40C9418510E94009DF801F4CF8AE5B9
:108F4000EEDC882309F440C08091710A9091720A86
:108F5000892B19F4E2EEF0E12BC0AADC6B017C0155
:108F60006093441C7093451C8093461C9093471C4F
:108F70002DEC3CEC4CE45DE30E94E0FA87FD0AC076
:108F800020E030E040E751E4C701B6010E943DF423
:108F90001816D4F4E3EBF0E184918F010F5F1F4FBB
:108FA000882311F40C9418510E94009DF801F4CF0D
:108FB00084918F010F5F1F4F882311F40C94185177
:108FC0000E94009DF801F4CF8AE5A9DC811104C05C
:108FD00081E5A5DC81110AC08AE5A1DC882309F4BA
:108FE00059C081E59CDC811121C054C02AE939E9CE
:108FF00049E95FE36091481C7091491C80914A1CCB
:1090000090914B1C0E94A2F4AB01BC014093441C04
:109010005093451C6093461C7093471C88E890E170
:109020000E9402C28AE00E94009DD6CF2091481C77
:109030003091491C40914A1C50914B1C6091441C3A
:109040007091451C8091461C9091471C0E94B9F874
:109050006B017C0120E030E040EA50EC0E94E0FA35
:1090600087FD0AC020E030E040EA50E4C701B601C5
:109070000E943DF4181674F4EBE4F0E184918F0142
:109080000F5F1F4F882311F40C9418510E94009D0C
:10909000F801F4CF83E58CDC882319F109DC4B015E
:1090A0005C012DEC3CEC4CEC5DE30E94E0FA87FDAA
:1090B0000AC020E030E040E85FE3C501B4010E944F
:1090C0003DF41816ACF4E4E2F0E184918F010F5FF7
:1090D0001F4F882311F40C9418510E94009DF80131
:1090E000F4CF8DEC882E8CEC982EA92C8EE3B82E24
:1090F00080E515DC882309F443C08091710A9091C2
:10910000720A892B71F4ECEEFFE084918F010F5FFE
:109110001F4F882311F40C9418510E94009DF801F0
:10912000F4CF80910C058F5F80930C05C1DB6B0140
:109130007C01609311057093120580931305909341
:10914000140520E030E0A9010E94E0FA87FD0AC082
:1091500020E030E048EC51E4C701B6010E943DF444
:10916000181674F4E4ECFFE084918F010F5F1F4F39
:10917000882311F40C9418510E94009DF801F4CF3B
:1091800086E416DC882319F193DB6B017C0120E077
:1091900030E040E85FE30E94E0FA87FD0AC020E08B
:1091A00030E040E850E4C701B6010E943DF41816D3
:1091B000A4F4EBE9FFE084918F010F5F1F4F882338
:1091C00011F40C9418510E94009DF801F4CFC12CA9
:1091D000D12C50EEE52E5FE3F52EA7019601C701D5
:1091E000B6010E94A2F49B01AC0160E070E084E44F
:1091F00090E40E9496F92091401C3091411C4091CE
:10920000421C5091431C0E94A2F42B013C01A50179
:109210009401C501B4010E94A2F4A70196010E9425
:10922000A2F42CEE31E548EB5DE30E9496F99B0138
:10923000AC01C301B2010E94A2F46093401C709380
:10924000411C8093421C9093431C88E4B1DB88232B
:10925000C9F02EDB0E94FEF970930E0560930D0598
:10926000655A71096437710568F0EDE6FFE0849195
:109270008F010F5F1F4F882309F4DAC70E94009DFA
:10928000F801F5CF85E54BDB8823E9F00E942E99A4
:10929000611571058105910511F00E9435F08091ED
:1092A000710A9091720A892B11F002DB04C060E010
:1092B00070E088E492E46093080570930905809358
:1092C0000A0590930B0582E52ADB81110DC0E9E3C5
:1092D000FFE084918F010F5F1F4F882309F4A8C717
:1092E0000E94009DF801F5CF8091710A9091720A59
:1092F000892BA9F0ADDA2F967FAF6EAF2F97161698
:1093000017069CF0E5E0FFE084918F010F5F1F4F8F
:10931000882309F48DC70E94009DF801F5CF8AE1EA
:1093200090E02F969FAF8EAF2F9788E541DB882383
:1093300061F0BEDA209167043091680440916904BD
:1093400050916A040E94B9F808C06091530470916A
:1093500054048091550490915604609304057093D1
:109360000505809306059093070589E521DB882391
:1093700061F09EDA20916B0430916C0440916D0491
:1093800050916E040E94B9F808C060915704709122
:1093900058048091590490915A0460930005709389
:1093A0000105809302059093030560910405709177
:1093B0000505809106059091070540E055E00E9463
:1093C00020E681110DC0EBEDFEE084918F010F5F6F
:1093D0001F4F882309F42CC70E94009DF801F5CF88
:1093E00084E49DDA91E089270E94E29920E030E050
:1093F00040EA50E460915B0470915C0480915D04EC
:1094000090915E040E943DF487FF14C0198A1A8A65
:109410001B8A1C8A80E090E0A0EAB0E489839A83EA
:10942000AB83BC83BE016F5E7F4FCE0101960E946D
:10943000699B0DDC0E942E996B017C01A8E8CA0E85
:10944000A3E1DA1EE11CF11C80910F05909110053B
:109450003EDC60910F0570911005072E000C880B03
:10946000990B0E9443F49B01AC0160914D047091F3
:109470004E0480914F04909150040E94B9F84B0122
:109480005C0120E030E0A9010E94E0FA87FF04C0FF
:10949000B7FAB094B7F8B09420E030E040E450E47C
:1094A000C501B4010E94E0FA18160CF50E942E992D
:1094B000DC01CB018C199D09AE09BF09B7FD0FC0B6
:1094C0000E942E996B017C01B8E8CB0EB3E1DB1E44
:1094D000E11CF11C0E94955E8AE00E94009D80E0E4
:1094E0000E946DA48091901480939114B2CF8091CA
:1094F0000D0590910E050E94E75F60910D0570913A
:109500000E05072E000C880B990B0E9443F49B015B
:10951000AC01609163047091640480916504909142
:1095200066040E94B9F84B015C0120E030E0A9011B
:109530000E94E0FA87FF04C0B7FAB094B7F8B0947D
:1095400020E030E040E450E4C501B4010E94E0FABC
:1095500018160CF50E942E99DC01CB018C199D097F
:10956000AE09BF09B7FD0FC00E942E996B017C01A7
:10957000E8E8CE0EE3E1DE1EE11CF11C0E94955EE0
:109580008AE00E94009D80E00E946DA4809190146A
:1095900080939114B2CF10925F04109260041092E5
:1095A0006104109262048FE594E00E94FBDB8091DD
:1095B0000C058823A1F108DA2091110530911205DC
:1095C00040911305509114056091581C7091591CDD
:1095D00080915A1C90915B1C0E94BAF86093581CB1
:1095E0007093591C80935A1C90935B1C20E030E0D0
:1095F00040E751E460911A0670911B0680911C06A9
:1096000090911D060E9496F969837A838B839C83CF
:10961000CE0101960E941F40D7D90E9427DA80E22E
:10962000E0EEF4E0DF01282F1D922A95E9F7E0EC47
:10963000F4E0DF01282F1D922A95E9F7E0EAF4E033
:10964000DF011D928A95E9F7BFD980913C1C90916A
:109650003D1CA0913E1CB0913F1C8093541C9093E4
:10966000551CA093561CB093571C19821A821B825A
:109670001C829E012F5F3F4F44E55CE160E57CE189
:109680008CE49CE1ABD99E01255C3F4F44E55CE155
:1096900060E57CE18CE49CE1A1D96196BFAD619766
:1096A000BB2329F067E574E083E594E004C060E043
:1096B00075E084E095E00E945DE6298F3A8F4B8F3C
:1096C0005C8F6D8F7E8F3FAF2D962FAF2D972D9690
:1096D000EFAD2D97E7FD83C4FFADF7FD80C424E017
:1096E000E202F0011124E155F24F40805180628086
:1096F00073803FAD84E03802F0011124E556F24F4B
:10970000D080C180328023808D2D9C2DA32DB22D41
:109710008FAB98AFA9AFBAAFAE01495C5F4FB20152
:10972000C3010E9420E6882309F45DC420E030E0F4
:1097300040EA50E4B201C3010E94BAF8F62E072FA6
:10974000182FE92E862F902FA12FBE2D8BAB9CAB0F
:10975000ADABBEAB8D2D9C2DA32DB22D8FA798AB9D
:10976000A9ABBAAB2D969FAD2D97911152C0AFAD5D
:10977000A11105C05F2D402F312F2E2D04C0542D77
:10978000452D362D272D852F942FA32FB22F8BAB50
:109790009CABADABBEABBFADB43034F4F42C052DF7
:1097A000162DE72CBB2369F020E030E040EA50E4BE
:1097B0006D2D7C2D832D922D0E94B9F8362F272FE9
:1097C00003C09601832D922D432F522FBC014FA72A
:1097D00058AB69AB7AABEFADE4300CF0A7C020E03A
:1097E00030E040EA50E46D2D7C2D832D922D0E94B7
:1097F000BAF821966FAF219723967FAF23972596CE
:109800008FAF259727969FAF2797FFADF11185C0A2
:1098100099C02D962FAD2D9724300CF453C03FAD39
:1098200034305CF020E030E040EA50E4B201C301A3
:109830000E94B9F8362F272F03C0342D252DC301E0
:10984000432F522FBC014BAB5CAB6DAB7EAB8FADEE
:109850008111E5C420E030E040EA50E4B201C301E8
:109860000E94B9F8F62E072F182FE92E20E030E0DD
:1098700040EA50E46D2D7C2D832D922D0E94BAF884
:109880006FA778AB89AB9AAB9FAD992309F44EC013
:1098900020E030E040EA50E46D2D7C2D832D922DA8
:1098A0000E94B9F821966FAF219723967FAF239737
:1098B00025968FAF259727969FAF2797AFADA430FA
:1098C00064F140C0BFADB1110DC020E030E040EA0E
:1098D00050E4B201C3010E94B9F8F62E072F182FE9
:1098E000E92E0FC0EFADE430B4F120E030E040EA03
:1098F00050E4B201C3010E94B9F86BAB7CAB8DABF5
:109900009EAB2196DFAE21972396CFAE2397259667
:109910003FAE259727962FAE279742ED842E43E53D
:10992000942E4BE7A42E41E4B42E29C02196DFAE3D
:1099300021972396CFAE239725963FAE259727965E
:109940002FAE279732ED832E33E5932E3BEFA32ED8
:1099500030E4B32E14C02196DFAE21972396CFAE0C
:10996000239725963FAE259727962FAE279722ED72
:10997000822E23E5922E2BEFA22E21E4B22E8BA96C
:109980009CA9ADA9BEA92C968CAF9DAFAEAFBFAFC1
:109990002C979C01AD01B201C3010E94B9F8698BFB
:1099A0007A8B8B8B9C8B4FA458A869A87AA8A301AB
:1099B00092016D2D7C2D832D922D0E94B9F86D8B17
:1099C0007E8B8F8B988F2C962CAD3DAD4EAD5FADC1
:1099D0002C97609153047091540480915504909198
:1099E00056040E94B9F82C966CAF7DAF8EAF9FAF36
:1099F0002C97A301920160915704709158048091B3
:109A0000590490915A040E94B9F82B013C018F2D02
:109A1000902FA12FBE2D89839A83AB83BC8321967F
:109A20008FAD219723969FAD23972596AFAD2597B0
:109A30002796BFAD27978D839E83AF83B88780918C
:109A40003C1C90913D1CA0913E1CB0913F1C89870D
:109A50009A87AB87BC872DEC3CEC4CEC5CE3C501F2
:109A6000B4010E94A2F42091401C3091411C40910D
:109A7000421C5091431C0E94A2F420915F0430913B
:109A8000600440916104509162040E94BAF86D87AD
:109A90007E878F87988B2C962CAD3DAD4EAD5FADFC
:109AA0002C97CA01B9010E94A2F46B017C01A301A9
:109AB0009201C301B2010E94A2F49B01AC01C70153
:109AC000B6010E94BAF820E030E040E050E40E9485
:109AD000E0FA18160CF047C00E9427DA1BA21CA25D
:109AE0001DA21EA220E030E040E05FE360915B0435
:109AF00070915C0480915D0490915E040E94BAF8BC
:109B00006F8F78A389A39AA39E012D5D3F4FAE016D
:109B1000415E5F4F67E574E083E594E00E94EE44A8
:109B20001BA21CA21DA21EA220E030E040E05FE3C9
:109B300060913C1C70913D1C80913E1C90913F1C9B
:109B40000E94BAF86F8F78A389A39AA39E012D5D16
:109B50003F4FAE01415E5F4FBE01615D7F4FCE0161
:109B6000C3960E94EE441F8E18A219A21AA29E014B
:109B7000215E3F4F4CE35CE1BE01615D7F4FCE0152
:109B8000C3960E94EE440E9453DA40903B025090EC
:109B90003C0260903D0270903E02E0901206F09010
:109BA00013060091140610911506A0900E06B090B1
:109BB0000F06C0901006D09011069501A601B701BE
:109BC000C8010E94E0FA181614F47501860120E01D
:109BD00030E040E251E4B701C8010E9496F9609379
:109BE0003B0270933C0280933D0290933E0240E022
:109BF000BE016F5E7F4FCE0101960E9422B7409258
:109C00003B0250923C0260923D0270923E020E94E2
:109C1000E444AFEABDE02296BFAFAEAF22972A96EA
:109C20001FAE1EAE2A9701E010E029960FAC2997CF
:109C300002C0000F111F0A94E2F72A96EEADFFADA5
:109C40002A9731962A96FFAFEEAF2A9721E030E0AF
:109C500029960FAC299702C0220F331F0A94E2F70E
:109C600063963FAF2EAF639790EA292E94E0392E8A
:109C700080EE94E028969FAF8EAF2897A0ECB4E0DA
:109C80002696BFAFAEAF2697EBE9FDE02496FFAF77
:109C9000EEAF249728962EAD3FAD289765963FAF3F
:109CA0002EAF6597D9018D919C919C012023312382
:109CB000232B09F4ADC06396EEADFFAD63978E2301
:109CC0009F23892B09F4A4C02696AEADBFAD26977D
:109CD0008D919C9180239123892B09F099C020E0DC
:109CE00030E040E050E42296AEADBFAD22976D91DA
:109CF0007D918D919C910E94BAF86B017C0120E0CE
:109D000030E040E050E42296EEADFFAD2297648152
:109D10007581868197810E94B9F84B015C0120E032
:109D200030E040E850ECC701B6010E943DF487FDE9
:109D300070C120E030E046E553E4C701B6010E945F
:109D4000E0FA181634F4C12CD12C86E5E82E83E411
:109D5000F82ECBA6DCA6EDA6FEA62496AEADBFAD32
:109D600024974D905D906D907C9020E030E040E82D
:109D70005FE3C301B2010E943DF487FD51C120E0C1
:109D800030E046E553E4C301B2010E94E0FA181640
:109D900034F4412C512CA6E56A2EA3E47A2E4F8E82
:109DA00058A269A27AA24FA258A669A67AA620E074
:109DB00030E040E850ECC501B4010E943DF487FD5D
:109DC00036C120E030E046E553E4C501B4010E940D
:109DD000E0FA181634F4812C912CE6E5AE2EE3E47B
:109DE000BE2E8BA29CA2ADA2BEA2AE01495D5F4F6A
:109DF000C701B6010E9420E6811120C12696EEAD72
:109E0000FFAD269780819181802B912B9183808358
:109E100028962EAD3FAD28972E5F3F4F28963FAF37
:109E20002EAF28976596AEADBFAD65978D919C918D
:109E300080239123892B09F4A6C0F90180819181A7
:109E400080239123892B09F49EC0F10180819181A7
:109E500080239123892B09F096C020E030E040E078
:109E600050E42496AEADBFAD24976D917D918D9158
:109E70009C910E94BAF82B013C0120E030E040E0C8
:109E800050E42496EEADFFAD249764817581868100
:109E900097810E94B9F84B015C012296AEADBFAD2F
:109EA0002297CD90DD90ED90FC9020E030E040E8EE
:109EB00050ECC701B6010E943DF487FDFFC020E0D1
:109EC00030E046E553E4C701B6010E94E0FA1816F7
:109ED00034F4C12CD12C66E5E62E63E4F62ECBA239
:109EE000DCA2EDA2FEA2CBA6DCA6EDA6FEA620E09B
:109EF00030E040E85FE3C301B2010E943DF487FD1A
:109F0000E4C020E030E046E553E4C301B2010E9422
:109F1000E0FA181634F4412C512C46E5642E43E443
:109F2000742E4FA258A669A67AA620E030E040E839
:109F30005FE3C501B4010E943DF487FDCDC020E080
:109F400030E046E553E4C501B4010E94E0FA18167A
:109F500034F4812C912C26E5A22E23E4B22E8F8E90
:109F600098A2A9A2BAA2AE01495D5F4FC701B6018E
:109F70000E9420E68111B7C0F10180819181802B80
:109F8000912B91838083F2E02F0E311C26962EAD0B
:109F90003FAD26972E5F3F4F26963FAF2EAF2697B9
:109FA00024968EAD9FAD2497049624969FAF8EAFD6
:109FB00024979AEA291694E0390609F06BCE229686
:109FC000AEADBFAD229714962296BFAFAEAF22972B
:109FD0002A96EEADFFAD2A97359709F024CE8091F1
:109FE0009014809391142F962EAD3FAD2F97215052
:109FF00031092F963FAF2EAF2F97232B09F4B3C013
:10A000002D963FAD2D9737FDAEC08FAD87FF45CB69
:10A01000AAC0C12CD12CB0E8EB2EB0ECFB2E99CE0F
:10A02000412C512CF0E86F2EFFE37F2EB8CE812C0F
:10A03000912C70E8A72E70ECB72ED3CEAE01415E06
:10A040005F4FC501B4010E9420E6882309F4D6CEF3
:10A0500080917304882321F1B701A60185EB9EE06E
:10A060000E9402C24FA158A569A57AA58FEA9EE079
:10A070000E9402C24BA15CA16DA17EA185EA9EE077
:10A080000E9402C24F8D58A169A17AA18FE99EE07A
:10A090000E9402C289E20E94009D8AE00E94009D07
:10A0A0009E01215E3F4FAE014D5D5F4FBE01695D78
:10A0B0007F4FCE018B960E9464DAA0CEC12CD12CAA
:10A0C00050E8E52E50ECF52E0ACF412C512C30E80B
:10A0D000632E3FE3732E25CF812C912C90E8A92E7F
:10A0E0009FE3B92E3CCFAE01415E5F4FC701B60181
:10A0F0000E9420E6882309F43FCF809173048823CF
:10A1000021F1B701A6018BE79EE00E9402C24FA198
:10A1100058A569A57AA585E79EE00E9402C24BA1D9
:10A120005CA16DA17EA18BE69EE00E9402C24F8DD4
:10A1300058A169A17AA185E69EE00E9402C289E247
:10A140000E94009D8AE00E94009D9E01215E3F4F7B
:10A15000AE014D5D5F4FBE01695D7F4FCE018B96B5
:10A160000E9464DA09CF0E9427DA80E090E0A0EA3A
:10A17000B0E48093541C9093551CA093561CB0934C
:10A18000571C19821A821B821C829E012F5F3F4F2F
:10A1900044E55CE160E57CE18CE49CE10E94EE44F6
:10A1A0008091040590910505A0910605B0910705E1
:10A1B00080934C1C90934D1CA0934E1CB0934F1C4D
:10A1C0008091000590910105A0910205B0910305D1
:10A1D0008093501C9093511CA093521CB093531C1D
:10A1E00019821A821B821C829E012F5F3F4F44E519
:10A1F0005CE160E57CE18CE49CE10E94EE446096C9
:10A20000FFAD6097F11114C010924C0410924B04F2
:10A210000E944F5F80E090E00E94E75F09C02FAD91
:10A22000F42C052D162DE72C24300CF031CB1ECB51
:10A23000CC5ADF4F0FB6F894DEBF0FBECDBFDF9113
:10A24000CF911F910F91FF90EF90DF90CF90BF9033
:10A25000AF909F908F907F906F905F904F903F90C6
:10A260002F9008951F920F920FB60F9211240BB6E4
:10A270000F922F933F938F939F93EF93FF93209190
:10A28000C3123091C4128091C5129091C612281742
:10A29000390731F4809131018F7D8093310114C0F1
:10A2A000E091C512F091C612ED5BFD4E20818091C8
:10A2B000C5129091C61201968F7799279093C61276
:10A2C0008093C51220933601FF91EF919F918F915A
:10A2D0003F912F910F900BBE0F900FBE0F901F90CC
:10A2E00018951F920F920FB60F9211240BB60F9272
:10A2F0002F934F935F938F939F93EF93FF9380914F
:10A30000300182FD1CC0209136018091471390914D
:10A3100048134091491350914A1301968F7799271A
:10A320004817590771F0E0914713F0914813E9532A
:10A33000FD4E2083909348138093471302C0809171
:10A340003601FF91EF919F918F915F914F912F91E6
:10A350000F900BBE0F900FBE0F901F9018952F926D
:10A360003F924F925F926F927F928F929F92AF92A5
:10A37000BF92CF92DF92EF92FF920F931F93CF93F2
:10A38000DF93CDB7DEB762970FB6F894DEBF0FBE8E
:10A39000CDBFF8948FEF9FEF909389008093880052
:10A3A0002AE02A8B212C312C78948091670590919A
:10A3B0006805A0916905B0916A05892B8A2B8B2BC2
:10A3C00009F00FC280915F1C8823E1F010925F1C9E
:10A3D00080915D1C90915E1C892B09F402C2109241
:10A3E0001F0510925E1C10925D1C9091650D80916E
:10A3F000660D981709F4F5C18091660D8F5F8F7017
:10A400008093660D80915D1C90915E1C892B09F4F0
:10A41000E8C14091630550916405609165057091B4
:10A42000660580915F0590916005A0916105B091EE
:10A4300062050091560510E020E030E0841B950B8A
:10A44000A60BB70B081719072A073B0710F4D90109
:10A45000C801E82F840F951FA61FB71F80936305BF
:10A4600090936405A0936505B093660520918400E0
:10A4700030918500245E3F4F40913B0550913C0553
:10A4800060913D0570913E0580912B0590912C05C2
:10A49000A0912D05B0912E05840F951FA61FB71F03
:10A4A00080933B0590933C05A0933D05B0933E05FA
:10A4B000B7FD1CC0889A80911C1C90911D1CA09116
:10A4C0001E1CB0911F1C40910802042E000C550B5D
:10A4D000660B770B840F951FA61FB71F80931C1C5C
:10A4E00090931D1CA0931E1CB0931F1C40913F0510
:10A4F00050914005609141057091420580912F0572
:10A5000090913005A0913105B0913205840F951FCF
:10A51000A61FB71F80933F0590934005A093410568
:10A52000B0934205B7FD1CC08E9A8091201C90917B
:10A53000211CA091221CB091231C40910902042EE1
:10A54000000C550B660B770B840F951FA61FB71FCA
:10A550008093201C9093211CA093221CB093231C59
:10A560004091430550914405609145057091460521
:10A570008091330590913405A0913505B091360551
:10A58000840F951FA61FB71F809343059093440522
:10A59000A0934505B0934605B7FD3FC080911905CE
:10A5A000F0910A028823C9F08091170582FF02C04A
:10A5B000F7FD06C080911605882311F40C94565BB4
:10A5C000809117059091180593FF02C0F7FD0CC00C
:10A5D00080911505811108C006C080910B018095FE
:10A5E000887080930901419A4091241C5091251C48
:10A5F0006091261C7091271C8F2FFF0F990BAA0BBF
:10A60000BB0B840F951FA61FB71F8093241C90932C
:10A61000251CA093261CB093271C40914705509100
:10A6200048056091490570914A05809137059091E0
:10A630003805A0913905B0913A05840F951FA61FE2
:10A64000B71F8093470590934805A0934905B093A1
:10A650004A05B7FD3AC04091281C5091291C6091D1
:10A660002A1C70912B1CC0900B020C2C000CDD08D6
:10A67000EE08FF084C0D5D1D6E1D7F1D4093281CCC
:10A680005093291C60932A1C70932B1C4091270522
:10A69000509128056091290570912A05841B950B1E
:10A6A000A60BB70B8093470590934805A0934905E7
:10A6B000B0934A0590911A058091540593FF02C00A
:10A6C000815001C08F5F8093540580913B0590912C
:10A6D0003C05A0913D05B0913E05B7FD15C04091E8
:10A6E0002705509128056091290570912A05841B42
:10A6F000950BA60BB70B80933B0590933C05A0935D
:10A700003D05B0933E05889880913F0590914005A6
:10A71000A0914105B0914205B7FD15C040912705B4
:10A72000509128056091290570912A05841B950B8D
:10A73000A60BB70B80933F0590934005A09341056E
:10A74000B09342058E988091430590914405A09165
:10A750004505B0914605B7FD3AC040912705509197
:10A7600028056091290570912A05841B950BA60B7D
:10A77000B70B8093430590934405A0934505B09390
:10A780004605809119058823E1F08091170582FF25
:10A7900004C080910A0287FD05C0809116058823B8
:10A7A00009F48CC7809117059091180593FF04C098
:10A7B00080910A0287FD0BC080911505811107C0A9
:10A7C00005C080910B018870809309014198E15088
:10A7D00041F0809184009091850082179307C8F31F
:10A7E0004BCE8091150290911602A0911702B09164
:10A7F0001802892B8A2B8B2B09F08AC08091550572
:10A80000882309F453C08090630590906405A0905C
:10A810006505B0906605C0905005D0905105E09058
:10A820005205F090530540915405C814D904EA0428
:10A83000FB0480F48091200590912105209124054E
:10A84000309125052817390728F4415040935405C5
:10A85000019714C08C149D04AE04BF04E0F48091F1
:10A860002005909121052091220530912305821722
:10A87000930788F44F5F4093540501969093210508
:10A8800080932005409111025091120260911302B1
:10A89000709114020EC08FEF9FEFDC0180931102C4
:10A8A00090931202A0931302B09314024FEF5FEF44
:10A8B000BA018091540587FD02C0169801C0169A0E
:10A8C00080918400909185004C962091540522231C
:10A8D000B9F0149A2091540527FF02C02F5F01C0E0
:10A8E000215020935405149820915405222369F394
:10A8F000209184003091850028173907C8F3E5CFEF
:10A900004093150250931602609317027093180239
:10A910008091670590916805A0916905B0916A05DD
:10A92000892B8A2B8B2B09F046C6A0915D1CB09118
:10A930005E1C109711F40C94005D8090630590905C
:10A940006405A0906505B090660540915F05509143
:10A950006005609161057091620584169506A606F2
:10A96000B706D8F010921F0510925E1C10925D1C65
:10A970009091650D8091660D981711F40C94005D0F
:10A980008091660D8F5F8F708093660D40EDC42EB1
:10A9900047E0D42EE12CF12C1AC440915B05509174
:10A9A0005C0560915D0570915E05481559056A0565
:10A9B0007B0508F4AAC14091570550915805609154
:10A9C000590570915A05D6960D911D912D913C9186
:10A9D000D997401751076207730708F077C14115EF
:10A9E00051056105710549F480901B0590901C0587
:10A9F000A0901D05B0901E0564C1E12CF980842E45
:10AA0000952F862F0A811B81FD81EE813F8128854C
:10AA10009C80E091621BE89D912CFF273091631B85
:10AA2000389D900CF11D1090641B189CF00DE99F4F
:10AA3000900CF11D399FF00DE89FF00D092D1F2F8F
:10AA4000099DE12D332722270F9FE00D311D2E1D7B
:10AA5000199DE00D311D2E1D1F9F300D211D032F4F
:10AA6000122F099DF12C332722270F9FF00C311D47
:10AA70002E1D199DF00C311D2E1D1F9F300D211D07
:10AA8000032F122FEE2780901B0590911C058091BB
:10AA90001D05009086040E2809F483C030918204BD
:10AAA000309FE1198E089E098E0920918304209F12
:10AAB000E01981089E098E09F0908404F09E8018A8
:10AAC00091098E09319FE01981089E098E09219F05
:10AAD000801891098E09F19E90198109099DF12C28
:10AAE000332722270F9FF00C311D2E1D199DF00CCE
:10AAF000311D2E1D1F9F300D211D032F122F309150
:10AB00007E04309FE10D8E1C9E1D8E1D20917F04C2
:10AB1000209FE00D811C9E1D8E1DF0908004F09EF4
:10AB2000800C911D8E1D319FE00D811C9E1D8E1D80
:10AB3000219F800C911D8E1DF19E900D811D099D00
:10AB4000F12C332722270F9FF00C311D2E1D199D4C
:10AB5000F00C311D2E1D1F9F300D211D032F122FB4
:10AB600030917A04309FE1198E089E098E09209158
:10AB70007B04209FE01981089E098E09F0907C04D7
:10AB8000F09E801891098E09319FE01981089E0975
:10AB90008E09219F801891098E09F19E90198109D3
:10ABA00082C030918204309FE10D8E1C9E1D8E1D4F
:10ABB00020918304209FE00D811C9E1D8E1DF0902E
:10ABC0008404F09E800C911D8E1D319FE00D811C30
:10ABD0009E1D8E1D219F800C911D8E1DF19E900D3E
:10ABE000811D099DF12C332722270F9FF00C311D69
:10ABF0002E1D199DF00C311D2E1D1F9F300D211D86
:10AC0000032F122F30917E04309FE1198E089E0988
:10AC10008E0920917F04209FE01981089E098E09EA
:10AC2000F0908004F09E801891098E09319FE01900
:10AC300081089E098E09219F801891098E09F19E35
:10AC400090198109099DF12C332722270F9FF00CC1
:10AC5000311D2E1D199DF00C311D2E1D1F9F300D15
:10AC6000211D032F122F30917A04309FE10D8E1C8D
:10AC70009E1D8E1D20917B04209FE00D811C9E1D3A
:10AC80008E1DF0907C04F09E800C911D8E1D319FD6
:10AC9000E00D811C9E1D8E1D219F800C911D8E1D1F
:10ACA000F19E900D811D11249C82F9820A831B83E1
:10ACB000FD83EE833F832887912C992AA12CB12C08
:10ACC000A82A89EE99E121E0298B14C0D2968D90B3
:10ACD0009D90AD90BC90D597F4CFB694A7949794DF
:10ACE0008794D988DD0CD98A04962AE185309207A9
:10ACF00009F4EAC4FC0105911591259134910815D8
:10AD000019052A053B0548F3DFC4409050055090D3
:10AD100051056090520570905305481459046A0417
:10AD20007B0408F0C3C180914F05811121C0FD0152
:10AD3000EE5BFF4FE080F1800281138178962081E5
:10AD4000318142815381D2966D917D918D919C91FB
:10AD5000D5970E9431C1DD24D394D0924F05E09164
:10AD60005D1CF0915E1C82A993A9A4A9B5A98EC10E
:10AD700040914B0550914C0560914D0570914E05E9
:10AD8000DA960D911D912D913C91DD974017510759
:10AD90006207730708F073C141155105610571051C
:10ADA00049F480911B0590911C05A0911D05B0915F
:10ADB0001E056CC1F0E0E985842F352F262FAA856A
:10ADC0007B856C855D85BE854F859889B091621BBA
:10ADD000B89F612D55274091631B489F600D511D01
:10ADE0001090641B189E500DB39F600D511D439F22
:10ADF000500DB29F500DA62F752FA69FB12D442741
:10AE00009927A59FB00D411D9F1F769FB00D411D35
:10AE10009F1F759F400D911DA42F792FA69FE12D97
:10AE200044279927A59FE00D411D9F1F769FE00DA8
:10AE3000411D9F1F759F400D911DA42F792FBB278A
:10AE400080911B0530911C0520911D050090860402
:10AE50000F2A09F483C0409182044A9FB1198F0BD5
:10AE60003F0B2F0B909183049A9FB01981093F0BE0
:10AE70002F0BE0918404EA9F801931092F0B479F23
:10AE8000B01981093F0B2F0B979F801931092F0BA8
:10AE9000E79F30192109A69FE12D44279927A59FF7
:10AEA000E00D411D9F1F769FE00D411D9F1F759F67
:10AEB000400D911DA42F792F40917E044A9FB10D22
:10AEC0008F1F3F1F2F1F90917F049A9FB00D811DF0
:10AED0003F1F2F1FE0918004EA9F800D311D2F1F1F
:10AEE000479FB00D811D3F1F2F1F979F800D311D64
:10AEF0002F1FE79F300D211DA69FE12D4427992785
:10AF0000A59FE00D411D9F1F769FE00D411D9F1FD6
:10AF1000759F400D911DA42F792F40917A044A9F6F
:10AF2000B1198F0B3F0B2F0B90917B049A9FB01997
:10AF300081093F0B2F0BE0917C04EA9F80193109B6
:10AF40002F0B479FB01981093F0B2F0B979F80193B
:10AF500031092F0BE79F3019210982C040918204EB
:10AF60004A9FB10D8F1F3F1F2F1F909183049A9FFF
:10AF7000B00D811D3F1F2F1FE0918404EA9F800DBB
:10AF8000311D2F1F479FB00D811D3F1F2F1F979F02
:10AF9000800D311D2F1FE79F300D211DA69FE12D34
:10AFA00044279927A59FE00D411D9F1F769FE00D27
:10AFB000411D9F1F759F400D911DA42F792F40911A
:10AFC0007E044A9FB1198F0B3F0B2F0B90917F048A
:10AFD0009A9FB01981093F0B2F0BE0918004EA9FE3
:10AFE000801931092F0B479FB01981093F0B2F0B97
:10AFF000979F801931092F0BE79F30192109A69FD0
:10B00000E12D44279927A59FE00D411D9F1F769FA5
:10B01000E00D411D9F1F759F400D911DA42F792F9D
:10B0200040917A044A9FB10D8F1F3F1F2F1F9091AF
:10B030007B049A9FB00D811D3F1F2F1FE0917C0460
:10B04000EA9F800D311D2F1F479FB00D811D3F1FAF
:10B050002F1F979F800D311D2F1FE79F300D211D42
:10B060001124E987AA877B876C875D87BE874F8716
:10B07000988B90E0932BA0E0B0E0A22B07C0A65ADB
:10B08000BF4F8D919D910D90BC91A02D29EE39E17E
:10B0900041E0498BF90145915591659174914817AB
:10B0A00059076A077B0708F499C3A7C38091540521
:10B0B0008823E1F0FD01E85BFF4F4081518160E0B2
:10B0C00070E0009111021091120220911302309150
:10B0D0001402401751076207730741F010921502DE
:10B0E00010921602109217021092180240910D024F
:10B0F00050910E0260910F027091100277FF5FC0B5
:10B10000AE5ABF4FCD90DD90ED90FC9089EE99E165
:10B1100021E0FC0145915591659174914C155D05B7
:10B120006E057F0550F4F694E794D794C794220FE8
:10B1300004967AE18530970761F72093560580E2FF
:10B14000C816D104E104F10428F470E2C72ED12C12
:10B15000E12CF12C90E2C91AD108E108F108C114E0
:10B16000A8E0DA06E104F10408F403C4B4E0DB9ECD
:10B17000C001112487519A4EFC01329625913491D9
:10B18000EC2D6627E39FA001E29F410D561F069418
:10B19000461F561F112460E070E0FC012591349198
:10B1A000C901A0E0B0E0841B950BA60BB70B809300
:10B1B0000D0290930E02A0930F02B0931002C09064
:10B1C0000D02D0900E02E0900F02F09010028091DC
:10B1D0005D1C90915E1C892B09F0E5C10E94B0C1F5
:10B1E00090935E1C80935D1C892B09F4DCC1E09177
:10B1F0005D1CF0915E1C808183FF3EC0858996892D
:10B20000A789B08D80931C1C90931D1CA0931E1CBD
:10B21000B0931F1C818D928DA38DB48D8093201CC3
:10B220009093211CA093221CB093231C858D968D96
:10B23000A78DB0A18093241C9093251CA093261C5D
:10B24000B093271C81A192A1A3A1B4A18093281C33
:10B250009093291CA0932A1CB0932B1C9091650DF0
:10B260008091660D981709F4B9CF8091660D8F5FB4
:10B270008F708093660DB2CFC588D688E788F08C32
:10B2800081E0C114D104E104F10409F480E0018DEE
:10B29000128D238D348D011511052105310509F01D
:10B2A0008260458D568D678D70A1411551056105F0
:10B2B000710509F0846080931F0510924B05109270
:10B2C0004C0510924D0510924E05109257051092A4
:10B2D00058051092590510925A0585A196A1A7A16B
:10B2E000B0A580935F0590936005A0936105B0932E
:10B2F0006205882499245401881A990AAA0ABB0A6B
:10B300008092470590924805A0924905B0924A055F
:10B310008092430590924405A0924505B09246055F
:10B3200080923F0590924005A0924105B09242055F
:10B3300080923B0590923C05A0923D05B0923E055F
:10B34000CC0CDD1CEE1CFF1CC0922B05D0922C05F2
:10B35000E0922D05F0922E05000F111F221F331FC2
:10B3600000932F051093300520933105309332055B
:10B37000440F551F661F771F4093330550933405C4
:10B38000609335057093360541A152A163A174A164
:10B39000440F551F661F771F40933705509338059C
:10B3A0006093390570933A05880F991FAA1FBB1F38
:10B3B0008093270590932805A0932905B0932A052B
:10B3C000109263051092640510926505109266054F
:10B3D00082A593A5A4A5B5A580935B0590935C0574
:10B3E000A0935D05B0935E0586A597A5A0A9B1A918
:10B3F0008093500590935105A0935205B093530547
:10B4000081A580932605DF01A95BBF4F9C91909396
:10B410005505992339F115962D913C91119730934B
:10B4200025052093240512972D913C911197309377
:10B4300023052093220510921502109216021092F5
:10B4400017021092180212972D913C91A90160E009
:10B4500070E04093110250931202609313027093B4
:10B4600014020CC088248A94982C540180921102F2
:10B4700090921202A0921302B0921402EA5BFF4F64
:10B48000908120911A0592130AC020910C0230E09D
:10B49000482F082E000C550B4217530731F090939C
:10B4A0001A0580930C020E9483C10E946CCD2FEF7D
:10B4B0003FEFA90120930D0230930E0240930F023B
:10B4C00050931002E0915D1CF0915E1CDF01DE964E
:10B4D000ED90FD900D911C9122A933A944A955A985
:10B4E000EA5AFF4F60817181828193810E9431C14C
:10B4F00010924F05E0915D1CF0915E1CEA5AFF4FDF
:10B5000080809180A280B38089EE99E121E0FC01E6
:10B510004591559165917491481559056A057B05CA
:10B5200058F4B694A79497948794220F0496A5E0B4
:10B53000BAE1A817B90759F72093560590E2891682
:10B540009104A104B10428F4B0E28B2E912CA12C1B
:10B55000B12C30E2831A9108A108B108811448E0A7
:10B560009406A104B10408F428C254E0959EC001D9
:10B57000112487519A4EFC01329625913491782DF1
:10B580006627739FA001729F410D561F0694461FA8
:10B59000561F1124FC01C590D490E12CF12CC41A43
:10B5A000D50AE108F108C0926705D0926805E092DB
:10B5B0006905F0926A050091670510916805209170
:10B5C000690530916A05409115025091160260910B
:10B5D000170270911802F02E198BF22FE32F4017EB
:10B5E00051076207730720F4F42E598BF62FE72FCB
:10B5F0008F2D9989AF2FBE2F0097E1E0AE07B105DF
:10B6000020F08FEF9FEFA0E0B0E0081B190B2A0B92
:10B610003B0B0093670510936805209369053093F1
:10B620006A054F3FFFEF5F076F077F0761F0481B19
:10B63000590B6A0B7B0B40931502509316026093D3
:10B64000170270931802F8942091840030918500BD
:10B65000205F3F4F4A8941504A8B442341F0280ED6
:10B66000391E2216330610F40C94D45101C019016E
:10B670003092890020928800789462960FB6F894F0
:10B68000DEBF0FBECDBFDF91CF911F910F91FF9015
:10B69000EF90DF90CF90BF90AF909F908F907F9072
:10B6A0006F905F904F903F902F90089580910B0185
:10B6B00080958870809309010C94E05280910B0171
:10B6C0008870809309016EC839893093560580E2ED
:10B6D00088169104A104B10428F430E2832E912C41
:10B6E000A12CB12C30E2831A9108A108B108811471
:10B6F00088E09806A104B10420F1E4E09E9EC00118
:10B70000112487519A4EFC01329625913491F82DDF
:10B71000EE27F39F7001F29FE10CFE1E0694EE1ED1
:10B72000FE1E1124FC01C590D490860120E030E07B
:10B73000480159018E189F08A108B10875016401DC
:10B7400022C0950184013695279517950795F80134
:10B75000EC7FCF0187519E4EFC01C590D490FC0137
:10B76000329625913491E82DE770E29FC001E39F66
:10B77000900D112423E0969587952A95E1F7C81A34
:10B78000D90AE12CF12C4C0D5D1D6E1D7F1D4093DF
:10B790005705509358056093590570935A05909139
:10B7A000550580915405992309F474C0882309F440
:10B7B0000ECDA85BBF4F8D919C91A0E0B0E0409171
:10B7C00011025091120260911302709114028417B9
:10B7D0009507A607B70709F060C0F9CCB695A795FD
:10B7E00097958795D988DD0CD98A2C5F3F4F45E026
:10B7F0005AE14217530709F04DCC59895093560529
:10B8000080329105A105B10520F480E290E0A0E02E
:10B81000B0E08097A109B109811558E09507A1050D
:10B82000B10508F443C074E0979F9001112427519B
:10B830003A4EF901329645915491EE27859FB00119
:10B84000849F610D7E1F06946E1F7E1F1124F901D7
:10B85000C590D490E12CF12CC61AD70AE108F10862
:10B8600080914B0590914C05A0914D05B0914E05EE
:10B870008C0D9D1DAE1DBF1D80934B0590934C05F7
:10B88000A0934D05B0934E0580915505811130C0B0
:10B8900080915405882309F49ACC109215021092D5
:10B8A0001602109217021092180291CCAC01BD0141
:10B8B0007695679557954795FA01EC7F9F0127513B
:10B8C0003E4EF901C590D490F901329645915491BC
:10B8D0008770849F9001859F300D1124F3E0369589
:10B8E0002795FA95E1F7C21AD30AE12CF12CB8CFCB
:10B8F0008989480E511C611C711C80915D1C9091BE
:10B900005E1C481459046A047B04D8F42091540541
:10B91000222309F45CCCFC01E85BFF4F20813181DC
:10B92000A90160E070E000911102109112022091D3
:10B93000130230911402401751076207730709F48C
:10B9400046CC109215021092160210921702109215
:10B950001802FC01E85BFF4F80819181A0E0B0E01C
:10B960008093110290931202A0931302B0931402D9
:10B970002ECCD701C601B695A79597958795FC0162
:10B98000EC7FCF0187519E4EFC0125913491FC0143
:10B990003296459154916C2D6770649FC001659FEC
:10B9A000900D112463E0969587956A95E1F7281B21
:10B9B000390BC901A0E0B0E0FACBD501C401B695BE
:10B9C000A79597958795FC01EC7FCF0187519E4EF7
:10B9D000FC01C590D490FC01329625913491482DFC
:10B9E0004770429FC001439F900D1124A3E096959C
:10B9F0008795AA95E1F7C81AD90AE12CF12CD3CD85
:10BA000080EDC82E87E0D82EE12CF12CE7CBCF9229
:10BA1000DF92EF92FF920F931F93CF93DF936C010E
:10BA20007A018B01C0E0D0E0CE15DF0581F0D801AE
:10BA30006D918D01D601ED91FC910190F081E02D89
:10BA4000C6011995892B11F02196EECF7E01C70111
:10BA5000DF91CF911F910F91FF90EF90DF90CF90EA
:10BA60000895FF920F931F93CF93DF938C01EB0107
:10BA7000F42E80E20E94009D8FEFF81611F084E50D
:10BA800001C082E40E94009D8AE30E94009DF801AB
:10BA9000608171818281938142E00E9411A148817D
:10BAA00059816A817B818DEA9CE10E9402C262E039
:10BAB00070E080E090E0DF91CF911F910F91FF90B7
:10BAC0000C9467DE1F920F920FB60F9211240BB6E3
:10BAD0000F922F933F934F935F936F937F938F9327
:10BAE0009F93AF93BF93EF93FF93809196059091AF
:10BAF0009705A0919805B0919905892B8A2B8B2BDE
:10BB000059F190919505E0919305F091940580810C
:10BB1000892780838091960590919705A09198053B
:10BB2000B0919905181619061A061B060CF056C096
:10BB30008091960590919705A0919805B0919905EF
:10BB40000197A109B1098093960590939705A09359
:10BB50009805B093990542C080911D02E9EBFCE184
:10BB6000E4919FEF90931D02E230C9F050F4EE2370
:10BB700099F0E13081F590916F009D7F90936F0077
:10BB80002AC0E43019F1E0F0E53029F59091730016
:10BB90009D7F909373001FC010926E001CC0909107
:10BBA00070009D7F9093700091E09093B000909111
:10BBB000B100987F94609093B1001092B3000BC0D5
:10BBC000909171009D7F9093710005C090917200DB
:10BBD0009D7F9093720060E00E9436DDFF91EF91AF
:10BBE000BF91AF919F918F917F916F915F914F9195
:10BBF0003F912F910F900BBE0F900FBE0F901F9093
:10BC000018958F929F92AF92BF92CF92DF92EF9250
:10BC1000FF920F931F93CF93DF93F0E2FF2EE12C5F
:10BC2000AE2DB0E0BD016F0D711D759567956E1558
:10BC300011F0F6120BC0E7E8FAE165917491072E56
:10BC4000000C880B990B0E9443F462C09B012150A9
:10BC50003109220F331F220F331FF901E75FF54E21
:10BC600005911491AB01440F551F440F551FFA0164
:10BC7000E75FF54EC591D4918017910714F4F62E25
:10BC8000D1CFC817D90714F4E62ECACFF901E55F62
:10BC9000F54EE590F490FA01E55FF54EC590D4902D
:10BCA000BC01601B710B072E000C880B990B0E94C6
:10BCB00043F44B015C01B6016E197F09072E000C9D
:10BCC000880B990B0E9443F49B01AC01C501B401A0
:10BCD0000E94A2F44B015C01C01BD10BBE01DD0F21
:10BCE000880B990B0E9443F49B01AC01C501B40180
:10BCF0000E9496F94B015C01B701FF0C880B990B70
:10BD00000E9443F49B01AC01C501B4010E94BAF842
:10BD1000DF91CF911F910F91FF90EF90DF90CF9027
:10BD2000BF90AF909F908F9008950F931F93CF93E4
:10BD3000DF93CDB7DEB728970FB6F894DEBF0FBEFE
:10BD4000CDBF6091510470915204072E000C880BF6
:10BD5000990B0E9443F46D837E838F839887809133
:10BD6000630490916404A0916504B0916604898392
:10BD70009A83AB83BC834DEFBE016B5F7F4FCE01D7
:10BD800001966FDE60914B0470914C04072E000CFD
:10BD9000880B990B0E9443F46D837E838F83988771
:10BDA00080914D0490914E04A0914F04B0915004A5
:10BDB00089839A83AB83BC834FEFBE016B5F7F4F58
:10BDC000CE0101964EDEE5EBFCE184918F010F5F21
:10BDD0001F4F882321F00E94009DF801F6CFE091CB
:10BDE0009205F0E0E057FA4F608170E080E090E06B
:10BDF0000E94F7A0E0EBFCE184918F010F5F1F4FE1
:10BE0000882321F00E94009DF801F6CF60919105F2
:10BE100070E080E090E00E94F7A028960FB6F894BA
:10BE2000DEBF0FBECDBFDF91CF911F910F9108955F
:10BE30000F930FB70F9300916E000B7F00936E006E
:10BE400078940F930BB70F930CB70F921F922F9309
:10BE50003F934F935F936F937F938F939F93AF9392
:10BE6000BF93EF93FF931124F0D1FF91EF91BF9116
:10BE7000AF919F918F917F916F915F914F913F9182
:10BE80002F911F900F900CBF0F910BBF0F9104606B
:10BE9000F89400936E000F910FBF0F911895CF92F9
:10BEA000DF92EF92FF92C0904D04D0904E04E0904C
:10BEB0004F04F090500460914B0470914C04665014
:10BEC0007109072E000C880B990B0E9443F49B010B
:10BED000AC01C701B6010E943DF487FF1FC020E0FE
:10BEE00030E040E050E4C701B6010E94BAF80E9479
:10BEF00003FA7093C9056093C8050E942E99DC016E
:10BF0000CB01805A9541AF4FBF4F8093C4059093AA
:10BF1000C505A093C605B093C70508C01092C40517
:10BF20001092C5051092C6051092C705FF90EF90BC
:10BF3000DF90CF900895CF92DF92EF92FF92C09062
:10BF40006304D0906404E0906504F090660460910E
:10BF500051047091520467507109072E000C880B30
:10BF6000990B0E9443F49B01AC01C701B6010E94EA
:10BF70003DF487FF1FC020E030E040E450E4C701FB
:10BF8000B6010E94BAF80E9403FA7093C305609349
:10BF9000C2050E942E99DC01CB01805A9541AF4F1A
:10BFA000BF4F8093BE059093BF05A093C005B0938B
:10BFB000C10508C01092BE051092BF051092C005C1
:10BFC0001092C105FF90EF90DF90CF9008952091DF
:10BFD0002602309127022F503109821793070CF463
:10BFE0009C01309352042093510480E0A4CF10921E
:10BFF0008C0580E090E0EBDF10924C0410924B0433
:10C000004EDF0E949AC280E090E0E1DF109290053E
:10C010002C9810924C0410924B0410929105809130
:10C02000020180728093000108958F929F92AF92D7
:10C03000BF92CF92DF92EF92FF920F931F93CF9315
:10C04000DF93F0E4FF2EE12CAE2DB0E0BD016F0DCB
:10C05000711D759567956E1511F0F6120BC0E2E033
:10C06000FCE165917491072E000C880B990B0E94DE
:10C0700043F462C09B0121503109220F331F220F6C
:10C08000331FF901EC5FF44E05911491AB01440F9D
:10C09000551F440F551FFA01EC5FF44EC591D49122
:10C0A0008017910714F4F62ED1CFC817D90714F4CE
:10C0B000E62ECACFF901EA5FF44EE590F490FA015A
:10C0C000EA5FF44EC590D490BC01601B710B072E43
:10C0D000000C880B990B0E9443F44B015C01B601E4
:10C0E0006E197F09072E000C880B990B0E9443F4F0
:10C0F0009B01AC01C501B4010E94A2F44B015C019B
:10C10000C01BD10BBE01DD0F880B990B0E9443F4BD
:10C110009B01AC01C501B4010E9496F94B015C0181
:10C12000B701FF0C880B990B0E9443F49B01AC01F3
:10C13000C501B4010E94BAF8DF91CF911F910F9110
:10C14000FF90EF90DF90CF90BF90AF909F908F9037
:10C15000089560E08091D5059091D60552DD6093F9
:10C1600063047093640480936504909366048091E3
:10C17000D3059091D40559DF60934D0470934E041C
:10C1800080934F0490935004A89510928D050895C4
:10C19000DF92EF92FF920F931F93CF93DF93F82ECE
:10C1A000D62EE72E8A0180911902882309F439C01E
:10C1B000EFEEF6E28491EF012196882321F00E94B0
:10C1C000009DFE01F7CFED2DFE2D8491EF0121960C
:10C1D000882321F00E94009DFE01F7CFEAE9FAE1F1
:10C1E0008491EF012196882321F00E94009DFE0199
:10C1F000F7CFF7FC0BC06F2DFF0C770B880B990B5B
:10C200000E94F7A08AE00E94009D0BC0E5E9FAE1D8
:10C210008491EF012196882321F00E94009DFE0168
:10C22000F7CF80919A05811108C01092190281E020
:10C2300080939A05C8010E9428A4DF91CF911F9195
:10C240000F91FF90EF90DF90D2CE0F931F93CF937B
:10C25000DF9380911C028F37A0F08F57909190054B
:10C260009093E605992311F02C9A01C02C98209107
:10C2700091052093E50590910201222369F09095A4
:10C280000BC09091E605891708F02C989091E50570
:10C29000891728F0909102019072909300018F5FAE
:10C2A00080931C029091E40581E089278093E40546
:10C2B00080911B0285301CF4C1E0C80F01C0C0E0B2
:10C2C000823009F4B8C054F4882301F1813009F0B8
:10C2D000E7C088E080937B0085E4C4C0843009F423
:10C2E000C9C00CF4BBC0853009F0DAC09091E305F9
:10C2F000911102C08093E3058091E3058150809302
:10C30000E305882309F4CCC0C5E0CAC080911A02B5
:10C310008F5F80311CF480931A02C2C010921A02FF
:10C3200080918D05811113C08091D9059091DA0516
:10C330009093D6058093D5058091D7059091D80527
:10C340009093D4058093D30581E080938D058AE096
:10C35000E9EDF5E0DF011D928A95E9F71092D80525
:10C360001092D7050091D5051091D605119501952C
:10C3700011098091510490915204D1E018161906C8
:10C380002CF080919005811101C0D0E0809135069C
:10C39000909136069195819591098017910734F413
:10C3A0004BE35CE16CE57CE180E0F2DE809124020D
:10C3B000909125029195819591090817190744F4E8
:10C3C000DD2331F04EE65CE16FE87CE180E0E0DE09
:10C3D00080914B0490914C0411E0181619062CF032
:10C3E00080919105811101C010E02091D305309119
:10C3F000D40580913306909134068217930734F068
:10C400004BE45CE16CE57CE18FEFC2DE209122021F
:10C41000309123028091D3059091D4058217930720
:10C420000CF43EC01123E1F14EE75CE16FE87CE1E2
:10C430008FEFAEDE35C080917A0086FD2EC08091F0
:10C440007800909179002091D9053091DA05820F1A
:10C45000931F9093DA058093D90522C088E08093DA
:10C460007B0086E480937C0080917A0080648093D6
:10C470007A0016C080917A0086FD11C08091780004
:10C48000909179002091D7053091D805820F931FA4
:10C490009093D8058093D70503C0C2E001C0C4E0E3
:10C4A000C0931B020E946CCD80918E0590918F05E8
:10C4B000009799F0019790938F0580938E05892BB3
:10C4C00061F481EA9CE19093EE1B8093ED1BDF9178
:10C4D000CF911F910F910C94B19DDF91CF911F913E
:10C4E0000F9108952F923F924F925F926F927F9299
:10C4F0008F929F92AF92BF92CF92DF92EF92FF9274
:10C500000F931F93CF93DF9300D01F92CDB7DEB769
:10C510005C017A8369831A0107FD0DC0802F002E0C
:10C52000000C990B9C838B83FC01E25FF34E8081AE
:10C530008823E1F008C08091D205882399F0E1E0DA
:10C54000F0E0FC83EB83F5011082EB81FC81EE0FC0
:10C55000FF1FEE0FFF1FE653FA4F10821182128267
:10C56000138230C081E090E09C838B83F90140808E
:10C570005180628073808B819C81880F991F880F06
:10C58000991F9C0126533A4F4901A3019201F401DE
:10C5900060817181828193810E943DF4882391F0B2
:10C5A000F401408251826282738211E020E030E027
:10C5B000A901C301B2010E94E0FA18160CF010E0C4
:10C5C000F5011083F50180818230F1F0833009F4A8
:10C5D00066C0813009F084C0EB81FC81EE0FFF1F43
:10C5E000EE0FFF1FE653FA4F2081318142815381C4
:10C5F000F10160817181828193810E943DF487FD08
:10C600006FC082E0F50180832B813C81220F331FB4
:10C61000220F331F26533A4F3C832B83B60180E011
:10C6200090E00E9441F49B01AC01EB81FC816081B0
:10C630007181828193810E94B9F89B01AC01F10163
:10C6400060817181828193810E94E0FA87FD14C02C
:10C650000E942E994B015C019701A8EEB3E00E9465
:10C66000AAF8860E971EA81EB91EE981FA8180825B
:10C670009182A282B38234C00E942E99E981FA810C
:10C68000C080D180E280F380DC01CB018C199D0950
:10C69000AE09BF09B7FD24C083E0F50180830F3FD9
:10C6A00019F044E05CE102C047E15CE16BE27CE14F
:10C6B000802F0F900F900F900F90DF91CF911F91CF
:10C6C0000F91FF90EF90DF90CF90BF90AF909F9031
:10C6D0008F907F906F905F904F903F902F9058CDAC
:10C6E0000F900F900F900F90DF91CF911F910F91AE
:10C6F000FF90EF90DF90CF90BF90AF909F908F9082
:10C700007F906F905F904F903F902F9008957F9211
:10C710008F929F92AF92BF92CF92DF92EF92FF9251
:10C720000F931F93CF93DF9320E030E048E452E46F
:10C730006091630470916404809165049091660433
:10C740000E94E0FA18164CF4EFE8FAE1E491C1E037
:10C7500001C0CC0FEA95EAF701C0C0E089E8E82EF5
:10C760008AE1F82E0FE81AE196E0A92E912CD0E08C
:10C77000CC24C394D12CF7017490F801849077FCF9
:10C7800023C0892D90E0082C02C0959587950A94C6
:10C79000E2F780FD19C0BE01082C02C075956795AF
:10C7A0000A94E2F76170B62EB1946B2D872D0E942A
:10C7B00036DD6B2D70E0872D0E94A0DDC60101C023
:10C7C000880F8A94EAF7982AAA94FFEFEF1AFF0AD3
:10C7D0000F5F1F4FA110CFCFDF91CF911F910F910E
:10C7E000FF90EF90DF90CF90BF90AF909F908F9091
:10C7F0007F9008952F923F924F925F926F927F9217
:10C800008F929F92AF92BF92CF92DF92EF92FF9260
:10C810000F93CF93DF93CDB7DEB760970FB6F89441
:10C82000DEBF0FBECDBF80918B0581113AC18091D3
:10C830008D05811118C060960FB6F894DEBF0FBE4B
:10C84000CDBFDF91CF910F91FF90EF90DF90CF9010
:10C85000BF90AF909F908F907F906F905F904F9020
:10C860003F902F90089575DC0E942E994B015C013A
:10C8700080910E1C811117C08091870590918805C9
:10C88000A0918905B0918A050097A105B10559F0DD
:10C89000A5019401281B390B4A0B5B0B57FD03C004
:10C8A00081E080930E1C6091510470915204072E18
:10C8B000000C880B990B0E9443F469837A838B8365
:10C8C0009C8344E1C42ED12C5CE3E52EF12C00E0E6
:10C8D0009E012F5F3F4F43E654E06AEB75E089EB22
:10C8E00095E000DE4090630450906404609065041D
:10C8F000709066046091370670913806072E000C20
:10C90000880B990B0E9443F49B01AC01C301B20157
:10C910000E94E0FA18160CF4C8C060E0609390051D
:10C920008091BE059091BF05A091C005B091C10551
:10C930000097A105B10521F1A5019401281B390B30
:10C940004A0B5B0B57FD1CC06091C2057091C3057B
:10C9500080E090E00E9441F49B01AC01609163048F
:10C960007091640480916504909166040E943DF486
:10C9700087FF4FC24AED5AE16CEE7AE180E008DCB5
:10C980008091830590918405A0918505B0918605DD
:10C99000A5019401281B390B4A0B5B0B57FD0FC0F7
:10C9A000B6DED501C4018C53964FAF4FBF4F809375
:10C9B000830590938405A0938505B09386058091A7
:10C9C000C4059091C505A091C605B091C705009713
:10C9D000A105B10511F1881A990AAA0ABB0AB7FC88
:10C9E0001CC06091C8057091C90580E090E00E946C
:10C9F00041F49B01AC0160914D0470914E04809113
:10CA00004F04909150040E943DF487FF3BC148EBD6
:10CA10005AE16BEC7AE18FEFBBDB60914B047091D4
:10CA20004C04072E000C880B990B0E9443F4698379
:10CA30007A838B839C8395E0C92ED12C24E1E22E4E
:10CA4000F12C0FEF9E012F5F3F4F4DE454E064EB5C
:10CA500075E088EB95E046DD8091D20581110FC12C
:10CA6000C0904D04D0904E04E0904F04F0905004DC
:10CA700020E030E040EA50E4C701B6010E94E0FA4D
:10CA800087FD0BC020E030E047E053E4C701B6016A
:10CA90000E943DF418160CF0F7C060E06093910519
:10CAA000CACE8BEF9AE10E9428A460912602709171
:10CAB0002702072E000C880B990B0E9443F49B0160
:10CAC000AC01C301B2010E943DF487FF26CF209044
:10CAD00051043090520420ED3CEC4CE45DE3609155
:10CAE0007F057091800580918105909182050E945B
:10CAF000A2F46B017C012091B0053091B105409109
:10CB0000B2055091B305C301B2010E94B9F89B016F
:10CB1000AC01C701B6010E94A2F46B017C0123E3C2
:10CB200033E343E75FE36091AC057091AD0580911D
:10CB3000AE059091AF050E94A2F49B01AC01C70124
:10CB4000B6010E94BAF86B017C016093AC0570934A
:10CB5000AD058093AE059093AF054092B00550921D
:10CB6000B1056092B2057092B3052114310409F445
:10CB70004CC1B101330C880B990B0E9443F4A30103
:10CB800092010E94B9F82B013C0120E030E040E224
:10CB900051EC0E943DF487FD38C180910E1C81113B
:10CBA00034C120E030E040E251E4C301B2010E9410
:10CBB000E0FA18160CF457C18091AB05811170C1D1
:10CBC0008091A7059091A805A091A905B091AA050B
:10CBD0008D839E83AF83B88720917B0530917C0540
:10CBE00040917D0550917E05C301B2010E94A2F4DF
:10CBF00069877A878B879C87A30192016D817E81EB
:10CC00008F8198850E94BAF86D837E838F83988781
:10CC10006093A7057093A8058093A9059093AA0532
:10CC200020917705309178054091790550917A05EA
:10CC30000E94A2F429853A854B855C850E94BAF84A
:10CC4000A70196010E94B9F86B017C0120E030E059
:10CC50004FE753E40E94E0FA20E030E0A901181603
:10CC60000CF406C1C701B6010E943DF487FD1FC147
:10CC7000C701B6010E94FEF9759567954FCE1092D7
:10CC80009105D9CD0CD9C9CE60914B0470914C045B
:10CC9000072E000C880B990B0E9443F4A701960104
:10CCA0000E94B9F84B015C01209173053091740525
:10CCB00040917505509176050E94A2F469877A87A4
:10CCC0008B879C872091A3053091A4054091A505F1
:10CCD0005091A605C501B4010E94BAF86D837E8308
:10CCE0008F8398876093A3057093A4058093A5050F
:10CCF0009093A60520916F053091700540917105C4
:10CD0000509172050E94A2F46D877E878F87988B61
:10CD100020ED3CEC4CE45DE360916B0570916C059B
:10CD200080916D0590916E050E94A2F42B013C014B
:10CD300020919F053091A0054091A1055091A20539
:10CD4000C701B6010E94B9F89B01AC01C301B20151
:10CD50000E94A2F42B013C0123E333E343E75FE3AA
:10CD600060919B0570919C0580919D0590919E0519
:10CD70000E94A2F49B01AC01C301B2010E94BAF867
:10CD80002B013C0160939B0570939C0580939D054E
:10CD900090939E05C0929F05D092A005E092A105B8
:10CDA000F092A2052D853E854F85588969857A8543
:10CDB0008B859C850E94BAF8A30192010E94B9F864
:10CDC0006B017C0120E030E04FE753E40E94E0FA81
:10CDD00020E030E0A9011816FCF4C501B4010E945E
:10CDE000E0FA181684F4A50194016D817E818F818B
:10CDF00098850E94B9F86093A3057093A405809369
:10CE0000A5059093A6056FE749CE81E08093AB0519
:10CE100084CD80E090D8B4CDC701B6010E943DF426
:10CE200087FD07C0C701B6010E94FEF97595679599
:10CE300035CE20E030E0A901C501B4010E943DF4E7
:10CE400087FF2BCEA50194016D817E818F8198850E
:10CE50000E94B9F86093A3057093A4058093A5057B
:10CE60009093A6051ACE81E08093AB056FE756CD6F
:10CE7000C301B2010E94E0FA1816C4F7A30192019F
:10CE80006D817E818F8198850E94B9F86093A70596
:10CE90007093A8058093A9059093AA056FE73ECDEE
:10CEA0001092AB051D821E821F82188695CE20E04F
:10CEB00030E0A901C301B2010E943DF487FF2DCDEE
:10CEC000A30192016D817E818F8198850E94B9F8BE
:10CED0006093A7057093A8058093A9059093AA0570
:10CEE0001CCDCF92DF92EF92FF926B017C0183E326
:10CEF000C816D104E104F10468F082E3C81AD1082D
:10CF0000E108F10862E370E080E090E00E9467DEF3
:10CF100071DCEDCFC701B6010E9467DEFF90EF9094
:10CF2000DF90CF9067CC8F929F92AF92BF92CF92BB
:10CF3000DF92EF92FF920F931F93CF93DF93CDB7C2
:10CF4000DEB764970FB6F894DEBF0FBECDBF0E9468
:10CF5000CBD6811121C188E0EBE5F2E0DE0111962C
:10CF600001900D928A95E1F784E50E94D8448823C8
:10CF700059F00E9428446B0180E1C816D10438F4AE
:10CF80009FE0C92ED12C03C02EE1C22ED12C1092CD
:10CF90004C0410924B040E944F5FE8EFFFE1849134
:10CFA0008F010F5F1F4F882321F00E94009DF80121
:10CFB000F6CF83E50E94D844882319F00E942844C4
:10CFC00002C06FEF70E077277093550B6093540B9E
:10CFD00080E090E0A0EAB0E48D879E87AF87B88BB1
:10CFE00020E030E040E050E460915B0470915C042C
:10CFF00080915D0490915E040E94BAF84B015C013F
:10D0000020E030E04DE453E40E943DF487FD06C08B
:10D01000812C912C8DE4A82E83E4B82E89869A86E3
:10D02000AB86BC86BE01635F7F4FCE0109960E942E
:10D03000699B80E090E0A8ECB2E4898B9A8BAB8B83
:10D04000BC8B80E090E0A8E4B2E48D879E87AF8738
:10D05000B88B89879A87AB87BC87AE014F5E5F4FDD
:10D06000BE01635F7F4FCE0109960E94489BDD247D
:10D070000D2C000CEE08FF08C701B6010E9443F416
:10D080009B01AC0160914D0470914E0480914F045E
:10D09000909150040E94E0FA18162CF50E94DD7958
:10D0A00041E0BE016F5F7F4F8CE49CE10E9422B79C
:10D0B000E5EDFFE184918F010F5F1F4F882321F081
:10D0C0000E94009DF801F6CF8091650D9091660D4C
:10D0D000891B8F7021F080E00E946DA4F5CF80E065
:10D0E0000E946DA4C9CF1092550B1092540B80E092
:10D0F00090E0A8ECB2E4898B9A8BAB8BBC8B80E080
:10D1000090E0AEE3B3E48D879E87AF87B88B80E075
:10D1100090E0A0E2B1E489879A87AB87BC87AE0133
:10D120004F5E5F4FBE01635F7F4FCE0109960E9445
:10D13000489B83E992E09E878D8784E690E09A87FA
:10D140008987BE01635F7F4FCE0109960E94C2D4DA
:10D1500086E295E09E878D8786E990E09A878987A9
:10D16000BE01635F7F4FCE0109960E94C2D481ED5C
:10D170009FE19093EE1B8093ED1B0E94B19DE5EB28
:10D18000FFE184917F019FEFE91AF90A882321F0DA
:10D190000E94009DF701F5CF64960FB6F894DEBFAC
:10D1A0000FBECDBFDF91CF911F910F91FF90EF90F8
:10D1B000DF90CF90BF90AF909F908F900895CF92C7
:10D1C000DF92EF92FF920F931F93CF93DF9388E547
:10D1D0000E948F44D82E89E40E948F44C82E882351
:10D1E00019F00E9428441CC0DD20C1F00E94584460
:10D1F00020E030E040E251E40E94B9F820E030E065
:10D2000040EC51E40E94BAF82BEA3AEA4AEA5CE3BD
:10D210000E94A2F40E94FEF9653010F01FEF01C0D9
:10D22000162F89E50E948F44082F8AE40E948F44BC
:10D23000C82F882319F00E9428441CC00023C1F085
:10D240000E94584420E030E040E251E40E94B9F8E6
:10D2500020E030E040EC51E40E94BAF82BEA3AEAD0
:10D260004AEA5CE30E94A2F40E94FEF9653010F0E5
:10D27000DFEF01C0D62F8AE50E948F44E82E81118E
:10D2800005C081E50E948F44F82E01C0F12CC11029
:10D2900001C0C0E02C2F30E0D11001C000E0200F11
:10D2A000311D2130310521F4E1101AC0F11018C0F0
:10D2B000EFEEF6E28491EF012196811103C0E0E3E5
:10D2C000FFE104C00E94009DFE01F4CF8491EF01B4
:10D2D0002196882309F455C00E94009DFE01F6CFD7
:10D2E00017FD02C0D7FF17C0EFEEF6E28491EF0101
:10D2F0002196811103C0E1E1FFE104C00E94009D7D
:10D30000FE01F4CF8491EF0121968823D1F10E9490
:10D31000009DFE01F7CF0E9458449B01AC01012FF4
:10D32000110F110BAD2FDD0FBB0BFF2099F085E026
:10D33000809FF001819FF00D1124EA0FFB1FEE0F7B
:10D34000FF1FEE0FFF1FE659F44E6081718182814D
:10D35000938103C060E070E0CB01E5E0E09FE00175
:10D36000E19FD00D1124CA0FDB1FCC0FDD1FCC0FA6
:10D37000DD1FC659D44E0E94BAF8688379838A8328
:10D380009B83DF91CF911F910F91FF90EF90DF90E2
:10D39000CF9008952F923F924F925F926F927F921B
:10D3A0008F929F92AF92BF92CF92DF92EF92FF92B5
:10D3B0000F931F93CF93DF93CDB7DEB761970FB66F
:10D3C000F894DEBF0FBECDBF83E50E948F44882353
:10D3D00049F00E944944182F811106C080E00E9444
:10D3E000E29902C01091171C80915304909154044B
:10D3F000A0915504B091560489839A83AB83BC8372
:10D400008091570490915804A0915904B0915A0406
:10D410008D839E83AF83B88780915B0490915C0479
:10D42000A0915D04B0915E0489879A87AB87BC8721
:10D430000E94B599882309F49AC083E40E948F441E
:10D44000882309F494C00E9458441B012C0105E074
:10D45000612C712C38EC388B82EC898BA12CB12C8F
:10D4600098EC9E87E2E4EF87015080F125E02D875C
:10D47000209F400111243D8531503D873F3FA1F35E
:10D48000F401E30FF11DEE0FFF1FEE0FFF1FE65932
:10D49000F44EC080D180E280F3809601A701B501EF
:10D4A0008E859F850E94E0FA18161CF45601EE86C0
:10D4B000FF869601A701B301888999890E943DF4EE
:10D4C00087FFD9CF3601E88AF98AD5CF93014889F9
:10D4D0005989B5018E859F850E94BAF820E030E019
:10D4E00040E05FE30E94A2F4A20191010E94BAF819
:10D4F0002B013C012DEB37E346E855EB0E94E0FAA7
:10D5000087FD0AC02DEB37E346E855E3C301B201BE
:10D510000E943DF418165CF580E00E94E29935E027
:10D52000D32E45E0C42EDA949FEFD91601F105E021
:10D53000CD9C500111240150B0F37501E00EF11C97
:10D54000C701880F991F880F991FFC01E659F44EF7
:10D550007F01A301920160817181828193810E9488
:10D56000B9F8F7016083718382839383E4CF86E502
:10D570000E948F44882399F00E94B599882379F0FE
:10D58000EBEFFEE184917F012FEFE21AF20A88238C
:10D5900021F00E94009DF701F5CF0E94A9CC8AE5F9
:10D5A0000E948F44882321F00E9458440E945CDC32
:10D5B000812F0E94E299111103C0E4E0F7E21CC040
:10D5C0008091171C8111F9CFEFEEF6E284918F0163
:10D5D0000F5F1F4F882321F00E94009DF801F6CFB6
:10D5E000ECEDFEE184918F010F5F1F4F882329F33B
:10D5F0000E94009DF801F6CF84918F010F5F1F4FAD
:10D60000882321F00E94009DF801F6CF8091171C1D
:10D61000811103C06DE174E002C069E174E08EEC39
:10D620009EE10E9438C28AE00E94009DE4E0F7E299
:10D6300084918F010F5F1F4F882321F00E94009D6E
:10D64000F801F6CFE1ECFEE184918F010F5F1F4FEF
:10D65000882321F00E94009DF801F6CFC090181C8D
:10D66000D090191CE0901A1CF0901B1C20E030E0B8
:10D67000A901C701B6010E94E0FA18164CF442E075
:10D68000C701B6010E9411A18AE00E94009D0CC052
:10D69000ECEBFEE184918F010F5F1F4F882321F097
:10D6A0000E94009DF801F6CF4CE050E063E574E085
:10D6B000CE0101960E94D6FB892BD1F061960FB660
:10D6C000F894DEBF0FBECDBFDF91CF911F910F91B8
:10D6D000FF90EF90DF90CF90BF90AF909F908F9092
:10D6E0007F906F905F904F903F902F900C943F747D
:10D6F00061960FB6F894DEBF0FBECDBFDF91CF911C
:10D700001F910F91FF90EF90DF90CF90BF90AF905F
:10D710009F908F907F906F905F904F903F902F9051
:10D72000089580916F00982F927081FF05C08091BD
:10D730006F008D7F80936F008091660D8093650DE3
:10D740008093640D8093630D84E68093620D28EED0
:10D7500033E030938F0520938E05992329F0809133
:10D760006F00826080936F0081E080935F1C0E9455
:10D77000938D0E9410BF8091171C882321F082E9AD
:10D7800094E10E941AC38CE0E2E9F4E1A3E5B4E07D
:10D7900001900D928A95E1F70C94C79B2F923F92CE
:10D7A0004F925F926F927F928F929F92AF92BF92B1
:10D7B000CF92DF92EF92FF920F931F93CF93DF935D
:10D7C000CDB7DEB7CD54D1090FB6F894DEBF0FBE8A
:10D7D000CDBF85E40E94D844882321F00E942844CC
:10D7E0007B0102C0E12CF12C83E40E94D844882301
:10D7F00021F00E942844162F01C015E085E50E9403
:10D80000D844882319F00E94494403C085E50E944A
:10D810008F4488ABF7FC07C0412C512C86E1682E61
:10D8200083E4782E06C0412C512C0CE8602E02E4D3
:10D83000702E83E50E94D844882321F00E9458442A
:10D840002B013C01E114F10411F4109292053E2CDD
:10D850000E942E996C877D878E879F870E2D001FD3
:10D860000027001F83E0801B082F8C859D85AE85D7
:10D87000BF858C53964FAF4FBF4F809383059093D6
:10D880008405A0938505B093860561E06E0D623036
:10D8900068F0E2E9FEE184918F010F5F1F4F88235A
:10D8A00009F4CCC40E94009DF801F5CFE7FC12C03A
:10D8B000EE2DEE0FFF0BEA5DFD4F608171816F5021
:10D8C0007109072E000C880B990B0E9443F46B0121
:10D8D0007C0106C0C12CD12CB0EFEB2EB2E4FB2EA4
:10D8E000C301B2010E94FEF9072E000C880B990BB0
:10D8F0000E9443F46C8B7D8B8E8B9F8BA7019601CE
:10D900000E94E0FA18166CF4E3E5FEE184918F01C1
:10D910000F5F1F4F882309F491C40E94009DF801F6
:10D92000F5CFEEE7FEE184917F012FEFE21AF20AD4
:10D93000882321F00E94009DF701F5CF0E94F75F38
:10D9400037FE04C08FE78093910508C0E32D032CB8
:10D95000000CFF0BE057FA4F8FE78083802F90E099
:10D960002C853D854E855F85205A35414F4F5F4F51
:10D970002AAF3BAF4CAF5DAF21E0209339023FEFC0
:10D9800033120BC04DEB5DE15FAF4EAFA7E8BDE1D9
:10D990002296BFAFAEAF22970AC0EBEAFDE1FFAF20
:10D9A000EEAF24E73DE122963FAF2EAF22972C85C4
:10D9B0003D854E855F8528A739A74AA75BA729AB78
:10D9C0003AAB4BAB5CAB1DAA1EAA1FAA18AE19AE90
:10D9D0001E8E00E40F8F0CE108A306E409A31AA22F
:10D9E0001BA21CA21DA2C12CD12C7601CA8EDB8EDB
:10D9F000EC8EFD8EC886D986EA86FB862FE730E05E
:10DA000040E050E0288B398B4A8B5B8BFFE78F2EF1
:10DA1000912CA12CB12C1CA61DA61EA61FA601E0B0
:10DA2000198E188E1D821E821F82212C232D032CFD
:10DA3000000C330BA90140575A4F24965FAF4EAFED
:10DA40002497220F331F220F331FD901AD59BB4F2B
:10DA5000BFA3AEA39C01092E000C440B550B2896C6
:10DA60002CAF3DAF4EAF5FAF289704969C01990F46
:10DA7000440B550B2C962CAF3DAF4EAF5FAF2C97A0
:10DA8000412F110F550B2E965FAF4EAF2E97809101
:10DA90003902882309F473C20E942E992B013C019C
:10DAA00080918D05882309F4C7C00E94A96037FCC6
:10DAB00011C0AEA1BFA1BC91BD83EEA1FFA1F181B8
:10DAC000FE83AEA1BFA11296BC91BF83EEA1FFA1C0
:10DAD00023800BC010914D041D8310914E041E83B2
:10DAE00010914F041F83209050042D813E814F815F
:10DAF000522D6AA17BA18CA19DA10E943DF487FFBC
:10DB000007C01D811AA31E811BA31F811CA32DA268
:10DB10002E8D3F8D48A159A16D817E818F81922DDF
:10DB20000E943DF487FF07C01D811E8F1E811F8F3D
:10DB30001F8118A329A28091830590918405A0914B
:10DB40008505B0918605A3019201281B390B4A0B6C
:10DB50005B0B57FD10C00E948763D301C2018C5339
:10DB6000964FAF4FBF4F8093830590938405A0934A
:10DB70008505B09386052D813E814F81522D6C899C
:10DB80007D898E899F89002309F440C00E943DF45D
:10DB900087FF52C0B301A2018C859D85AE85BF85EC
:10DBA000481B590B6A0B7B0BDB01CA018858934158
:10DBB000A109B109B7FD40C0D501C401088919897F
:10DBC0002A893B89801B910BA20BB30BB595A795B6
:10DBD0009795879537FE03C08093910505C02496DD
:10DBE000EEADFFAD249780834CA75DA76EA77FA7FE
:10DBF0000C890AA31D891BA30E890CA31F891DA3D1
:10DC000048A659A66AA67BA600E016C00E94E0FAC4
:10DC1000181694F4D301C20128A539A54AA55BA51D
:10DC2000821B930BA40BB50BAC01BD0148585341AB
:10DC30006109710977FFA6C120E030E040EA51E4B4
:10DC40006C897D898E899F890E94BAF82D813E81D9
:10DC50004F81522D0E943DF487FF0DC0EFEDFDE195
:10DC600084918F010F5F1F4F882309F488C10E94A0
:10DC7000009DF801F5CFD301C20129A93AA94BA90A
:10DC80005CA9821B930BA40BB50BB7FD83C00E944C
:10DC9000955E8AE00E94009DD301C2018053984F97
:10DCA000AF4FBF4F89AB9AABABABBCAB1DA911114A
:10DCB00054C02EA93FA948AD59AD6D817E818F8199
:10DCC000922D0E94E0FA1816BCF528966CAD7DAD39
:10DCD0008EAD9FAD28970E9443F42D813E814F81E8
:10DCE000522D0E94BAF86EAB7FAB88AF99AFA301FB
:10DCF0009201205A35414F4F5F4F2AAF3BAF4CAF97
:10DD00005DAF2C966CAD7DAD8EAD9FAD2C970E9416
:10DD100043F49B01AC016C897D898E899F890E94A7
:10DD2000B9F82D813E814F81522D0E943DF4881F0C
:10DD30008827881F8DAB2EC0D301C2012AAD3BAD11
:10DD40004CAD5DAD821B930BA40BB50BB7FD22C090
:10DD50004EAD5FAD60ED7DE11AC020E030E040EAFD
:10DD600051E46C897D898E899F890E94B9F89B0155
:10DD7000AC016D817E818F81922D0E943DF487FFE1
:10DD800009C022964EAD5FAD22976BE97DE1832DF0
:10DD90000E94C860D301C201880F991FAA1FBB1F30
:10DDA00028A539A54AA55BA5821B930BA40BB50B2F
:10DDB0002C853D854E855F85821B930BA40BB50B8F
:10DDC00081309F49A442B10568F0E6E5FDE1849108
:10DDD0008F010F5F1F4F882309F4D1C00E94009D5F
:10DDE000F801F5CF2E964EAD5FAD2E97888D998DAB
:10DDF000481759070CF04BCE84E594E09A83898349
:10DE000089E690E09C838B83BE016F5F7F4FCE01DC
:10DE100003960E94C2D48DE796E09A83898382EDAF
:10DE200090E09C838B83BE016F5F7F4FCE01039692
:10DE30000E94C2D4E9EFFCE184918F010F5F1F4F74
:10DE4000882321F00E94009DF801F6CF37FC03C023
:10DE50000CE114E002C008E214E0B80188EE9CE195
:10DE60000E9438C2488559856A857B8584EE9CE18D
:10DE70000E9402C28AE00E94009DB80183ED9CE1ED
:10DE80000E9438C24A8D5B8D6C8D7D8D8FEC9CE13C
:10DE90000E9402C28AE00E94009DB8018EEB9CE1C4
:10DEA0000E9438C2B701A6018AEB9CE10E9402C21F
:10DEB0008AE00E94009D08A9002309F4BFC137FE33
:10DEC0002FC0288539854A855B852093730530935B
:10DED000740540937505509376052CEA35EC47E2BE
:10DEE0005EE36A8D7B8D8C8D9D8D0E94A2F4609384
:10DEF0006F057093700580937105909372052CEAFD
:10DF000035EC47E25EE3C701B6010E9496F96093E3
:10DF10006B0570936C0580936D0590936E058EC1B3
:10DF200088859985AA85BB8580937B0590937C0520
:10DF3000A0937D05B0937E052CEA35EC47E25EE3C5
:10DF40006A8D7B8D8C8D9D8D0E94A2F460937705E8
:10DF5000709378058093790590937A052CEA35ECD7
:10DF600047E25EE3C701B6010E9496F960937F0520
:10DF70007093800580938105909382055FC10E9414
:10DF8000F75F5CC1088D198D012B09F42DC12CA5FB
:10DF90003DA54EA55FA5280F391F4A1F5B1F2C8783
:10DFA0003D874E875F872CA53DA54EA55FA5281B05
:10DFB000390B4A0B5B0B688979898A899B890E9496
:10DFC0004DF82C853D854E855F850E947EF8DA01EF
:10DFD000C901880D991DAA1DBB1D84319105A1059C
:10DFE000B105FCF04C015D018C3E9105A105B10528
:10DFF0002CF05BEE852E912CA12CB12C40E88416E0
:10E000009104A104B104DCF08EEF90E0A0E0B0E058
:10E0100088199909AA09BB09888B998BAA8BBB8B94
:10E0200012C044E1842E912CA12CB12C04E110E00B
:10E0300020E030E0088B198B2A8B3B8B04C0888A48
:10E04000998AAA8ABB8AEBE4FEE184918F010F5F73
:10E050001F4F882321F00E94009DF801F6CFC501D3
:10E06000B4010E94F7A0E6E4FEE184918F010F5F06
:10E070001F4F882321F00E94009DF801F6CF688988
:10E0800079898A899B890E94F7A04E8D5F8D68A14E
:10E0900079A18FE39EE10E9402C24AA15BA16CA11B
:10E0A0007DA188E39EE10E9402C2088D198D033094
:10E0B00011050CF499C0688979898A899B890E9425
:10E0C00043F420E030E040E850E40E94A2F46B0109
:10E0D0007C012E8D3F8D48A159A16AA17BA18CA105
:10E0E0009DA10E94B9F82BED3FE049E450E40E9465
:10E0F000A2F420E030E040E05FE30E94A2F49B0144
:10E10000AC01C701B6010E9496F9688779878A87B2
:10E110009B876C857D858E859F850E9443F42FE6C5
:10E1200032E143E85AE30E94A2F46B017C01488586
:10E1300059856A857B8582E39EE10E9402C2B70110
:10E14000A6018CE29EE10E9402C22AE939E949E176
:10E150005FE3688579858A859B850E94A2F468873C
:10E1600079878A879B879B01AC010E94BAF8A70137
:10E1700096010E9496F96A8F7B8F8C8F9D8F2885E0
:10E1800039854A855B85C701B6010E94A2F420E06B
:10E1900030E040E05EE30E94A2F46B017C01ECE120
:10E1A000FEE184918F010F5F1F4F882321F00E94B1
:10E1B000009DF801F6CF488559856A857B8586E103
:10E1C0009EE10E9402C24A8D5B8D6C8D7D8D80E147
:10E1D0009EE10E9402C2B701A6018AE09EE10E9470
:10E1E00002C28AE00E94009D88899989AA89BB8918
:10E1F000880D991DAA1DBB1DB595A7959795879567
:10E2000037FE03C08093910505C02496EEADFFADA7
:10E2100024978083088D198D0F5F1F4F198F088FEA
:10E220001C891E8F0D890F8F1E8918A30F8909A3C2
:10E230004C865D866E867F8601E0FECCC35BDF4F39
:10E240000FB6F894DEBF0FBECDBFDF91CF911F9107
:10E250000F91FF90EF90DF90CF90BF90AF909F9085
:10E260008F907F906F905F904F903F902F90089588
:10E27000CF92DF92EF92FF920F931F93CF93DF9392
:10E28000CDB7DEB7A0970FB6F894DEBF0FBECDBFF7
:10E290008091E30D882351F080916710823018F44B
:10E2A00082E08093671083E08093661080E090E0C6
:10E2B000A0EAB0E489839A83AB83BC8380E090E0DA
:10E2C000ADE4B3E48D839E83AF83B88780E090E0B4
:10E2D000A0EAB1E489879A87AB87BC8788E592E09A
:10E2E0000E94509D8111A7C185E40E948F4488231C
:10E2F00081F00E9458446B017C0120E030E0A901CC
:10E300000E94E0FA87FF0BC0F7FAF094F7F8F09458
:10E3100006C0C12CD12C80E8E82E80E4F82EF7FA54
:10E32000F094F7F8F094C98ADA8AEB8AFC8A8AE5D5
:10E330000E94D844882379F08AE50E94D844882333
:10E3400019F00E94584403C060E070E0CB01698777
:10E350007A878B879C8788E50E94D844882379F048
:10E3600088E50E94D844882319F00E94584403C0CD
:10E3700060E070E0CB0169837A838B839C8389E5BD
:10E380000E94D844882379F089E50E94D8448823E4
:10E3900019F00E94584403C060E070E0CB016D8327
:10E3A0007E838F83988785E50E948F44882329F098
:10E3B0000E9458446B017C010CC0E091200B84E06A
:10E3C000E89FF0011124E052F44EC080D180E28039
:10E3D000F38020E030E0A901C701B6010E94E0FA15
:10E3E00087FF04C0F7FAF094F7F8F094F7FAF09486
:10E3F000F7F8F094CD8ADE8AEF8AF88E198E1A8E9D
:10E400001B8E1C8E8CE40E948F44882329F00E946E
:10E4100058446B017C010CC0E091200B94E0E99F13
:10E42000F0011124EC51F44EC080D180E280F380E1
:10E4300020E030E0A901C701B6010E94E0FA87FFA1
:10E4400004C0F7FAF094F7F8F094CD8EDE8EEF8EDC
:10E45000F8A282E40E94D844882321F00E94284434
:10E46000162F01C01AE00091781CAE014B5E5F4F81
:10E47000BE016F5F7F4FCE0141960E944EA9882357
:10E4800009F4D5C010924A04E4E0F7E284917F01D8
:10E490009FEFE91AF90A882321F00E94009DF701F5
:10E4A000F5CFE9E8FFE184917F019FEFE91AF90ACE
:10E4B000882321F00E94009DF701F5CF61E0812FB4
:10E4C00083D50E942E99DC01CB018054984DA64F34
:10E4D000BF4F8093870590938805A0938905B093DB
:10E4E0008A0510920E1C83E08093FC1B81E08093D0
:10E4F000400480914004882309F47FC060E0812FAC
:10E5000063D580914A04811107C090914A0480919B
:10E510000E1C892B80934A0480914A04882309F4B5
:10E5200068C080916710833018F48E5F8093671005
:10E53000E4E0F7E284917F019FEFE91AF90A88236A
:10E5400021F00E94009DF701F5CFEFE6FFE18491F5
:10E550007F019FEFE91AF90A882339F00E94009D94
:10E56000F701F5CF81E00E946DA4809140048111F4
:10E57000F9CF0E94F9A30E94D4A8E4E0F7E28491C5
:10E580007F019FEFE91AF90A882321F00E94009D7C
:10E59000F701F5CFE0E5FFE184917F019FEFE91AF4
:10E5A000F90A81111FC00E942E99DC01CB01805411
:10E5B000984DA64FBF4F8093870590938805A093F1
:10E5C0008905B0938A0510920E1C81E08093400467
:10E5D00010924A0480916710843040F082508093FA
:10E5E000671004C00E94009DF701D6CF61E0812F23
:10E5F000EBD481E00E946DA47CCF81E08093FC1B72
:10E6000080E090E0A0E0B0E48D879E87AF87B88B74
:10E610008091560B882359F0212FAE01435F5F4F45
:10E62000BE01635E7F4FCE0149960E94A1DE01309C
:10E6300011F40E9453C2A0960FB6F894DEBF0FBE2D
:10E64000CDBFDF91CF911F910F91FF90EF90DF90A1
:10E65000CF900895CF93DF93E4E0F7E28491EF0148
:10E660002196882321F00E94009DFE01F7CF83E5CB
:10E670000E948F44882321F00E94494480933A02EB
:10E68000E2E1F1E28491EF012196882321F00E94DA
:10E69000009DFE01F7CF80913A02811103C0EEE0A8
:10E6A000F1E202C0EAE0F1E28491EF0121968823D1
:10E6B00021F00E94009DFE01F7CFE2E0F1E284919B
:10E6C000EF012196882321F00E94009DFE01F7CFE3
:10E6D00020916704309168044091690450916A0464
:10E6E0006091140B7091150B8091160B9091170B84
:10E6F0000E94BAF8AB01BC0180E091E20E9402C224
:10E7000020916B0430916C0440916D0450916E0423
:10E710006091180B7091190B80911A0B90911B0B43
:10E720000E94BAF8AB01BC018DEF90E20E9402C2D8
:10E7300020916F04309170044091710450917204E3
:10E7400060911C0B70911D0B80911E0B90911F0B03
:10E750000E94BAF8AB01BC018AEF90E20E9402C2AB
:10E76000E2EFF0E28491EF012196882321F00E94EC
:10E77000009DFE01F7CF209167043091680440911D
:10E78000690450916A0460912D0270912E0280916B
:10E790002F02909130020E94BAF8AB01BC0180EFC9
:10E7A00090E20E9402C220916B0430916C0440916F
:10E7B0006D0450916E04609131027091320280912B
:10E7C0003302909134020E94BAF8AB01BC018DEE85
:10E7D00090E20E9402C220916F0430917004409137
:10E7E00071045091720460913502709136028091EB
:10E7F0003702909138020E94BAF8AB01BC018AEE50
:10E8000090E20E9402C28AE0DF91CF910C94009DB9
:10E81000FF920F931F93CF93DF93F82E092F162F9C
:10E82000E5EEF0E28491EF012196882321F00E9429
:10E83000009DFE01F7CFEF2DF02F8491EF0121967F
:10E84000882321F00E94009DFE01F7CFE3EEF0E265
:10E850008491EF012196882321F00E94009DFE0102
:10E86000F7CF612F70E080E090E00E94F7A08AE08F
:10E87000DF91CF911F910F91FF900C94009D4F92CB
:10E880005F926F927F928F929F92AF92BF92CF9240
:10E89000DF92EF92FF92CF93DF9320916704309144
:10E8A00068044091690450916A0460915304709126
:10E8B000540480915504909156040E94BAF8AB011B
:10E8C000BC0180EE90E20E9402C220916B04309164
:10E8D0006C0440916D0450916E04609157047091E6
:10E8E00058048091590490915A040E94BAF8AB01DF
:10E8F000BC018CED90E20E9402C220916F04309125
:10E900007004409171045091720460915B047091A5
:10E910005C0480915D0490915E040E94BAF8AB01A2
:10E92000BC0188ED90E20E9402C240915F045091C8
:10E930006004609161047091620484ED90E20E9431
:10E9400002C280916F00982F927081FF05C0809164
:10E950006F008D7F80936F0040901C1C50901D1C99
:10E9600060901E1C70901F1C8090201C9090211C99
:10E97000A090221CB090231CC090241CD090251C79
:10E98000E090261CF090271C992329F080916F00BD
:10E99000826080936F00EAECF0E28491EF012196AF
:10E9A000882321F00E94009DFE01F7CFC301B20130
:10E9B0000E94F7A0E6ECF0E28491EF012196882313
:10E9C00021F00E94009DFE01F7CFC501B4010E9415
:10E9D000F7A0E2ECF0E28491EF012196882321F088
:10E9E0000E94009DFE01F7CFC701B6010E94F7A06B
:10E9F0008AE0DF91CF91FF90EF90DF90CF90BF90B2
:10EA0000AF909F908F907F906F905F904F900C94FD
:10EA1000009D2F923F924F925F926F927F928F92C2
:10EA20009F92AF92BF92CF92DF92EF92FF920F939D
:10EA30001F93CF93DF93CDB7DEB762970FB6F894ED
:10EA4000DEBF0FBECDBF80912A0683FD95C183E551
:10EA50000E94D8448C87811106C082E50E94D84468
:10EA6000882309F489C10E9458440E94FEF9CB0111
:10EA70000E9467460E94584420E030E040EA50E49B
:10EA80000E94E0FA181614F40E9453C2E6EBF0E27A
:10EA90008491FB83EA83882371F0082E000C990B84
:10EAA0000E9466B34A815B814F5F5F4F5B834A83FD
:10EAB000FA018491F0CF8DE090E00E9466B38AE085
:10EAC00090E00E9466B381E0809339028091200B30
:10EAD000809392051A821B821C821D8218861986D9
:10EAE0001A861B8619821D86FCE3FE872CE12F8780
:10EAF00036E4388B312C212C40E8498B5FEB5A8B64
:10EB0000812C912C540160914B0470914C04072E80
:10EB1000000C880B990B0E9443F47B018C019B0134
:10EB2000AC01632D722D89899A890E943DF4882356
:10EB300041F120914D0430914E0440914F04509189
:10EB400050048C85B70181110CC0C8010E943DF4AE
:10EB5000881F8827881F89833E2C2F2C098B1A8BAE
:10EB600010C0C8010E943DF487FF06C0EAEBF0E246
:10EB70008491FB83EA83E8C03E2C2F2C098B1A8BEF
:10EB800019820E942E996B017C01DC01CB01288542
:10EB900039854A855B85821B930BA40BB50BB7FDAA
:10EBA0003BC0D701C60188519C4FAF4FBF4F8887EC
:10EBB0009987AA87BB870E94955EEEEBF0E284916D
:10EBC0003F019FEF691A790A882321F00E94009D76
:10EBD000F301F5CF81149104A104B104B9F0D5017A
:10EBE000C401805F984DAF4FBF4FBC01CD016C1980
:10EBF0007D098E099F0928EE33E040E050E00E9435
:10EC00005CF8CA01B9010E94F7A003C08FE30E941B
:10EC1000009D8AE00E94009D80E00E946DA40E94F9
:10EC20002E996093FB0A7093FC0A8093FD0A9093DF
:10EC3000FE0AA0914D04AE83B0914E04BF830091B3
:10EC40004F04109150040E944B182E813F81A8015F
:10EC5000632D722D89899A890E94B9F82B013C0194
:10EC600020E030E0A9010E94E0FA87FF04C077FAB3
:10EC7000709477F8709481149104A104B10459F44C
:10EC800020E030E040E85FE3C301B2010E943DF4C0
:10EC900087FF0DC00AC020E030E040E450E4C3012B
:10ECA000B2010E94E0FA181614F446015701E981F6
:10ECB000EE2391F12A813B814C815D812115310543
:10ECC0004105510541F0D701C601821B930BA40BEE
:10ECD000B50BB7FD21C02E813F81A8016D857E85D2
:10ECE0008F8598890E94B9F820E030E040EC5FE31E
:10ECF0000E943DF487FD3ACFD701C601805A954165
:10ED0000AF4FBF4F8A839B83AC83BD839E819D871A
:10ED1000AF81AE870F87188B80913902882309F461
:10ED200025CF81149104A104B10409F4ECCEB0E123
:10ED3000CB1AB7E2DB0AE108F108C818D908EA08DB
:10ED4000FB08F7FE13CFDFCE882361F0082E000CFE
:10ED5000990B0E9466B3EA81FB813196FB83EA83BB
:10ED60008491F2CF8DE090E00E9466B38AE090E05B
:10ED70000E9466B38091390262960FB6F894DEBFA6
:10ED80000FBECDBFDF91CF911F910F91FF90EF90FC
:10ED9000DF90CF90BF90AF909F908F907F906F90BB
:10EDA0005F904F903F902F900895EF92FF920F93B6
:10EDB0001F93CF93DF93CDB7DEB769970FB6F89463
:10EDC000DEBF0FBECDBF83E50E94D844811103C0D2
:10EDD000EEE9F0E208C00E9428446E347105C1F7E4
:10EDE0000E940AC3E4C084918F010F5F1F4F8823E4
:10EDF00021F00E94009DF801F6CFE5E9F0E2849150
:10EE00008F010F5F1F4F882321F00E94009DF801A2
:10EE1000F6CF80913A0690913B060E94F9D5E8E83A
:10EE2000F0E284918F010F5F1F4F882321F00E9431
:10EE3000009DF801F6CF80913C0690913D060E941E
:10EE4000F9D5EDE7F0E284918F010F5F1F4F882322
:10EE500021F00E94009DF801F6CF80913A06909132
:10EE60003B0620913C0630913D06821B930B20917E
:10EE7000781C215041E050E0223010F040E050E09A
:10EE8000841B950B0E94F9D58AE00E94009DE5E75E
:10EE9000F0E284918F010F5F1F4F882321F00E94C1
:10EEA000009DF801F6CF80913E0690913F06A0911B
:10EEB0004006B09141068E8B9F8BA88FB98FBE0103
:10EEC0006F5F7F4FCE0146960E941E9CE8E6F0E2FF
:10EED00084918F010F5F1F4F882321F00E94009DB6
:10EEE000F801F6CFCE0101967C018C01F8018191E9
:10EEF0008F01882319F00E94009DF8CF809142066F
:10EF000090914306A0914406B09145068E8B9F8B4D
:10EF1000A88FB98FBE016F5F7F4FCE0146960E94CA
:10EF20001E9CE8E5F0E284918F010F5F1F4F88235C
:10EF300021F00E94009DF801F6CFF70181917F0139
:10EF4000882319F00E94009DF8CF8AE00E94009D5E
:10EF5000E0E5F0E284918F010F5F1F4F882321F0DD
:10EF60000E94009DF801F6CFE0E4F0E284918F0169
:10EF70000F5F1F4F882321F00E94009DF801F6CFFC
:10EF800020E030E04AE754E460914606709147067D
:10EF900080914806909149060E9496F942E00E94AD
:10EFA00011A18DE60E94009D8AE00E94009D699655
:10EFB0000FB6F894DEBF0FBECDBFDF91CF911F918A
:10EFC0000F91FF90EF9008958F929F92AF92BF9212
:10EFD000CF92DF92EF92FF920F931F93CF93DF9325
:10EFE00000D01F92CDB7DEB7F82E662351F01092F5
:10EFF000F1051092ED051092EE051092EF051092BA
:10F00000F0050E942E998090ED059090EE05A0905D
:10F01000EF05B090F0059B01AC01281939094A09A8
:10F020005B0957FD4CC02091F105F7FC16C04F2D30
:10F030000F2C000C550B4C5F5F4FE22F022E000C83
:10F04000FF0B4E175F07DCF12F153CF044EFC42E89
:10F05000DD24D394E12CF12C06C038EEC32E33E02E
:10F06000D32EE12CF12CDC01CB018C0D9D1DAE1DAE
:10F07000BF1D8093ED059093EE05A093EF05B0932F
:10F08000F005022F017010E024E2209FC001219FB3
:10F09000900D901B112480599C4F9C838B8382E39D
:10F0A00090E09A838983BE016D5F7F4FCE01019608
:10F0B0000E94C2D48091F1058F5F8093F1050F907B
:10F0C0000F900F900F90DF91CF911F910F91FF90B4
:10F0D000EF90DF90CF90BF90AF909F908F9008956A
:10F0E000AF92BF92CF92DF92EF920F931F93CF9385
:10F0F000DF93CDB7DEB760970FB6F894DEBF0FBED3
:10F10000CDBF5C018B010E94E444E090200B8CE4B5
:10F11000C82E8CE1D82E84E0E89EF0011124E25E36
:10F12000FD4F2081318142815381F50160817181E0
:10F13000828193810E9496F9F60124853585468562
:10F1400057850E94BAF8F601648775878687978786
:10F150001D861E861F86188A80819181A281B381B7
:10F1600089839A83AB83BC8384819581A681B7818F
:10F170008D839E83AF83B88780859185A285B38573
:10F1800089879A87AB87BC87AE01475F5F4FBE0117
:10F190006B5F7F4FCE0101960E94D9CBCE010D96B9
:10F1A0006C0128E53CE1AE01475F5F4FBE016B5F3C
:10F1B0007F4F0C9792D40E9427460E94938D6096B1
:10F1C0000FB6F894DEBF0FBECDBFDF91CF911F9178
:10F1D0000F91EF90DF90CF90BF90AF9008958F92F6
:10F1E0009F92AF92BF92EF92FF920F931F93CF9394
:10F1F000DF9300D01F92CDB7DEB7182F809149045E
:10F200008770873069F48FE40E94D844882319F00E
:10F210000E94494403C08FE40E948F448111BEC004
:10F220000E94938D80E00E94E29980913B02909130
:10F230003C02A0913D02B0913E028093E90590937B
:10F24000EA05A093EB05B093EC0580910002909144
:10F2500001029093E8058093E70584E690E090939F
:10F2600001028093000281E080934B0611111BC0C4
:10F2700088E50E948F44F82E89E50E948F44082F6C
:10F280008AE50E948F44E82EF11006C0011109C0E2
:10F29000811107C0F02E0CC0002319F0F02E182F9A
:10F2A00008C010E006C0FF24F39401E0EE24E394CC
:10F2B00011E00E94E44482E50E94D844882361F072
:10F2C0000E9458444B015C0120E030E0A9010E94FB
:10F2D0003DF4882371F106C0812C912C80EAA82E80
:10F2E00080E4B82E111104C0F11002C0002391F186
:10F2F0008092541C9092551CA092561CB092571CA0
:10F30000A501940160915B0470915C0480915D049F
:10F3100090915E040E943DF487FF0BC019821A820F
:10F320001B821C82BE016F5F7F4F84E59CE10E94BF
:10F33000699B111105C0F11003C0011106C00AC07C
:10F3400080E00E94C2A21123C1F381E00E94C2A208
:10F35000111102C0EE2019F082E00E94C2A20E94A8
:10F36000C79B80914A0680934B068091E905909156
:10F37000EA05A091EB05B091EC0580933B029093D8
:10F380003C02A0933D02B0933E028091E70590912C
:10F39000E805909301028093000271DA0F900F90BC
:10F3A0000F900F90DF91CF911F910F91FF90EF90F1
:10F3B000BF90AF909F908F9008959F92AF92BF9211
:10F3C000CF92DF92EF92FF920F931F93CF93DF9331
:10F3D00087E5A82E82E0B82E0CE41CE1C3E5D4E05A
:10F3E00097E6C92E94E0D92E24E7E22E24E0F22EEF
:10F3F000912CF50181915F010E948F44882309F1CE
:10F400000E945844F7012081211104C02091780402
:10F41000222339F0288139814A815B810E94BAF820
:10F420000AC0F3E09F1639F0F60120813181428154
:10F4300053810E94B9F8F8016083718382839383BA
:10F4400009C088819981AA81BB81F8018083918359
:10F45000A283B38393940C5F1F4F2496F4E0CF0EE6
:10F46000D11C2FEFE21AF20A84E09812C2CF86E490
:10F470000E94D8448823C9F00E94584420E030E01C
:10F48000A9010E94E0FA181684F40E94584420E072
:10F4900030E040E752E40E9496F960933B0270939B
:10F4A0003C0280933D0290933E0280912A0683FDA8
:10F4B00028C080913906882321F120915F04309182
:10F4C000600440916104509162046091581C7091F5
:10F4D000591C80915A1C90915B1C0E94B9F8209194
:10F4E00046063091470640914806509149060E94D1
:10F4F000BAF8609346067093470680934806909347
:10F500004906DF91CF911F910F91FF90EF90DF900F
:10F51000CF90BF90AF909F9008952F923F924F92BF
:10F520005F926F927F929F92AF92BF92CF92DF9243
:10F53000EF92FF920F931F93CF93DF93CDB7DEB778
:10F5400064970FB6F894DEBF0FBECDBF1A012B0132
:10F55000922EF32EC82ED12CF601EB58F94DE491E2
:10F56000AA24A3941E160CF4A12CBB24B39420E06F
:10F5700030E0A901C201B1010E94E0FA18160CF0B6
:10F58000B12CCC0CDD1CCC0CDD1CC6018D5A9B4F64
:10F590003C01FC0110821182128213820E94C79BDF
:10F5A000F3012082318242825382E090200B20E0DE
:10F5B00030E0A901B801892D9F2D0E943DF48111F1
:10F5C0000AC0F601E85DF94D85919591A591B49138
:10F5D0008C019A2EFB2EC801A92DBF2D898B9A8BE9
:10F5E000AB8BBC8B80915B0490915C04A0915D041B
:10F5F000B0915E04409157045091580460915904B1
:10F6000070915A04009153041091540420915504B0
:10F610003091560409831A832B833C834D835E8388
:10F620006F83788789879A87AB87BC871D861E86FC
:10F630001F86188AAE01475F5F4FBE016B5F7F4F29
:10F64000CE0101960E94D9CBCE010D966C018E01A0
:10F650000F5E1F4F2FE534E0AE01475F5F4FBE01E5
:10F660006B5F7F4F0C9739D20E94938DAB1459F08A
:10F6700080916006882319F01092600604C084E12E
:10F6800090E20E9428A464960FB6F894DEBF0FBEE5
:10F69000CDBFDF91CF911F910F91FF90EF90DF9041
:10F6A000CF90BF90AF909F907F906F905F904F9062
:10F6B0003F902F9008952F923F924F925F926F92BA
:10F6C0007F928F929F92AF92BF92CF92DF92EF92F2
:10F6D000FF920F931F93CF93DF93CDB7DEB762975F
:10F6E0000FB6F894DEBF0FBECDBF8DE690E00E944E
:10F6F000509D8111D9C180912A0683FDD5C183E532
:10F700000E94D8448C87811106C082E50E94D844AB
:10F7100089838823B1F00E9458440E94FEF9CB01EE
:10F720000E94E75F0E94584420E030E04AEA52E439
:10F730000E943DF418160CF4B2C10E949AC221E056
:10F740002983E6EAF0E284918F01882351F0082EA4
:10F75000000C990B0E9466B30F5F1F4FF801849154
:10F76000F4CF8DE090E00E9466B38AE090E00E94C2
:10F7700066B30E944BC4F981FF2309F495C181E06F
:10F78000809339021A821B821C821D821886198678
:10F790001A861B8619821D862CE32E873CE13F8743
:10F7A00046E4488B312C212C50E8598B8FEB8A8B07
:10F7B000812C912C54016091510470915204072EB8
:10F7C000000C880B990B0E9443F47B018C019B0178
:10F7D000AC01632D722D89899A890E943DF488239A
:10F7E00059F1209163043091640440916504509173
:10F7F00066049C85B701802F91110CC0912F0E9447
:10F800003DF4881F8827881F89833E2C2F2C098B65
:10F810001A8B12C0912F0E943DF487FF08C080917F
:10F820003902EEEAF0E28491FB83EA83E8C03E2CE1
:10F830002F2C098B1A8B19820E942E996B017C0147
:10F84000DC01CB01288539854A855B85821B930BBA
:10F85000A40BB50BB7FD3BC0D701C60188519C4F27
:10F86000AF4FBF4F88879987AA87BB870E94955E55
:10F87000E2EBF0E284913F019FEF691A790A882355
:10F8800021F00E94009DF301F5CF81149104A104A1
:10F89000B104B9F0D501C401805F984DAF4FBF4F9F
:10F8A000BC01CD016C197D098E099F0928EE33E05A
:10F8B00040E050E00E945CF8CA01B9010E94F7A044
:10F8C00003C08FE30E94009D8AE00E94009D80E0BB
:10F8D0000E946DA40E942E996093FB0A7093FC0A0B
:10F8E0008093FD0A9093FE0AA0916304AE83B091C9
:10F8F0006404BF8300916504109166040E944B1854
:10F900002E813F81A801632D722D89899A890E94D9
:10F91000B9F82B013C0120E030E0A9010E94E0FA97
:10F9200087FF04C077FA709477F87094811491047B
:10F93000A104B10459F420E030E040E85FE3C301E2
:10F94000B2010E943DF487FF0DC00AC020E030E004
:10F9500040E450E4C301B2010E94E0FA181614F426
:10F9600046015701E981EE2391F12A813B814C81C7
:10F970005D81211531054105510541F0D701C601D1
:10F98000821B930BA40BB50BB7FD21C02E813F81C9
:10F99000A8016D857E858F8598890E94B9F820E041
:10F9A00030E040EC5FE30E943DF487FD38CFD701A3
:10F9B000C601805A9541AF4FBF4F8A839B83AC836A
:10F9C000BD839E819D87AF81AE870F87188B809105
:10F9D0003902882309F423CF81149104A104B104CE
:10F9E00009F4E9CEB0E1CB1AB7E2DB0AE108F1088D
:10F9F000C818D908EA08FB08F7FE11CFDCCE882327
:10FA000061F0082E000C990B0E9466B3EA81FB811D
:10FA10003196FB83EA838491F2CF8DE090E00E94DF
:10FA200066B38AE090E00E9466B3809166108130F0
:10FA300009F03AC0EAEAF0E28491FB83EA83882382
:10FA400071F0082E000C990B0E9466B34A815B810D
:10FA50004F5F5F4F5B834A83FA018491F0CF8DE063
:10FA600090E00E9466B38AE090E062960FB6F89448
:10FA7000DEBF0FBECDBFDF91CF911F910F91FF90E1
:10FA8000EF90DF90CF90BF90AF909F908F907F903E
:10FA90006F905F904F903F902F900C9466B30E94B0
:10FAA00053C231E039834DCE62960FB6F894DEBF73
:10FAB0000FBECDBFDF91CF911F910F91FF90EF90BF
:10FAC000DF90CF90BF90AF909F908F907F906F907E
:10FAD0005F904F903F902F9008952F923F924F92BA
:10FAE0005F926F927F928F929F92AF92BF92CF92CE
:10FAF000DF92EF92FF920F931F93CF93DF93CDB7D7
:10FB0000DEB7C857D1090FB6F894DEBF0FBECDBF20
:10FB1000E0918E05F0918F05EF2B11F00C942E865D
:10FB20002896DFAECEAE28976E2C79016A015B0174
:10FB3000FC0120813181428153816C962CAF3DAF15
:10FB40004EAF5FAF6C9720912C1C30912D1C4091D3
:10FB50002E1C50912F1C6C966CAD7DAD8EAD9FAD63
:10FB60006C970E94A2F40E94EBFAE0966CAF7DAF16
:10FB70008EAF9FAFE097D5018D919D910D90BC9177
:10FB8000A02DA0968CAF9DAFAEAFBFAFA097209138
:10FB9000301C3091311C4091321C5091331CBC01FF
:10FBA000CD010E94A2F40E94EBFAE4966CAF7DAF07
:10FBB0008EAF9FAFE497D6012D913D914D915C9111
:10FBC000A4962CAF3DAF4EAF5FAFA4972091341CED
:10FBD0003091351C4091361C5091371CA4966CAD69
:10FBE0007DAD8EAD9FADA4970E94A2F40E94EBFA6A
:10FBF000E8966CAF7DAF8EAF9FAFE897D7012D91A0
:10FC00003D914D915C9122962CAF3DAF4EAF5FAFD1
:10FC100022972091381C3091391C40913A1C509108
:10FC20003B1C22966CAD7DAD8EAD9FAD22970E94A0
:10FC3000A2F40E94EBFA60966CAF7DAF8EAF9FAFDF
:10FC4000609780912A0683FF1CC060962CAD3DAD65
:10FC50004EAD5FAD60972093970D3093980D409314
:10FC6000990D50939A0D22968CAD9DADAEADBFAD62
:10FC700022978093870D9093880DA093890DB09360
:10FC80008A0DD801BC91B9A7F801F181F9ABD8016F
:10FC90001296BC91BEABF801F381FAAF8091650D6D
:10FCA0009091660D891B8F708F3021F480E00E9447
:10FCB0006DA4F4CF0091650DE9960FAFE99780919F
:10FCC000650D082F10E01CA30BA380918B0D909164
:10FCD0008C0DA0918D0DB0918E0DE0968CAC9DACED
:10FCE000AEACBFACE097881A990AAA0ABB0A809109
:10FCF0008F0D9091900DA091910DB091920DE49681
:10FD00002CAC3DAC4EAC5FACE497281A390A4A0AD9
:10FD10005B0A8091930D9091940DA091950DB091F7
:10FD2000960DE8962CAD3DAD4EAD5FADE897281B26
:10FD3000390B4A0B5B0B2DA33EA34FA358A7809111
:10FD4000970D9091980DA091990DB0919A0D609694
:10FD50000CAD1DAD2EAD3FAD6097081B190B2A0BE6
:10FD60003B0B0DA71EA72FA738AB012B022B032B94
:10FD700009F4BCC080910D1C81114BC060916304DB
:10FD80007091640480916504909166040E94FEF96C
:10FD90002091510230915202621773070CF039C062
:10FDA00060962CAD3DAD4EAD5FAD60972093970D45
:10FDB0003093980D4093990D50939A0D22968CADE7
:10FDC0009DADAEADBFAD22978093870D9093880D0A
:10FDD000A093890DB0938A0DE4E0F7E284918F013E
:10FDE0000F5F1F4F811103C0E1E4F1E204C00E94E4
:10FDF000009DF801F3CF84918F010F5F1F4F88237F
:10FE000021F00E94009DF801F6CF1DA61EA61FA698
:10FE100018AA94E0699E80011124025E1D4F6DA511
:10FE20007EA58FA598A90E9443F4D8012D913D91FC
:10FE30004D915C910E94A2F46B017C0120E030E0C6
:10FE4000A9010E94E0FA87FF04C0F7FAF094F7F8DE
:10FE5000F0946091381C7091391C80913A1C9091FB
:10FE60003B1C0E94FEF99B01AC01A8E5B2E00E9498
:10FE70009AF80E9443F4A70196010E943DF487FF7F
:10FE800039C060960CAD1DAD2EAD3FAD60970093AF
:10FE9000970D1093980D2093990D30939A0D2296FB
:10FEA0002CAD3DAD4EAD5FAD22972093870D3093C5
:10FEB000880D4093890D50938A0DE4E0F7E2849118
:10FEC0008F010F5F1F4F811103C0E2E2F1E204C016
:10FED0000E94009DF801F3CF84918F010F5F1F4FA7
:10FEE000882321F00E94009DF801F6CF1DA61EA6D2
:10FEF0001FA618AAD501C4018827B7FD83959927A5
:10FF0000AA27BB27782E57FE03C0382F3260732EE6
:10FF10008DA19EA1AFA1B8A5B7FF03C0972D946096
:10FF2000792E0DA51EA52FA538A937FF03C0172DC3
:10FF30001860712E24E0629E80011124025E1D4F24
:10FF40006DA57EA58FA598A90E9443F4D8012D9197
:10FF50003D914D915C910E94A2F46B017C0120E0E7
:10FF600030E0A9010E94E0FA87FF04C0C701B60192
:10FF7000905802C0C701B60120E030E040E05FE3E6
:10FF80000E94BAF80E9403FA6AAB7BAB8CAB9DABC4
:10FF900088E60BA11CA1809FF001819FF00D112428
:10FFA000EE51FB4E1082EA5BFF4F7082B501A40157
:10FFB000B7FE07C044275527BA01481959096A09ED
:10FFC0007B0988E60BA11CA1809FF001819FF00DA9
:10FFD0001124EE51FB4E458B568B678B708F2C9600
:10FFE0002CAE3DAE4EAE5FAE2C9757FE0DC08827AF
:10FFF0009927DC0182199309A409B5092C968CAFC5
:020000021000EC
:100000009DAFAEAFBFAF2C9728E60BA11CA1209FE0
:10001000F001219FF00D1124EE51FB4E2C968CAD7A
:100020009DADAEADBFAD2C97818F928FA38FB48F56
:100030000DA11EA12FA138A537FF07C0309520952F
:10004000109501951F4F2F4F3F4FE8E67E2EABA135
:10005000BCA17A9EF0017B9EF00D1124EE51FB4E67
:10006000058F168F278F30A38AA99BA9ACA9BDA99C
:1000700081A392A3A3A3B4A323964FAF2397752E76
:10008000F62FE72F2C968CAD9DADAEADBFAD2C9766
:10009000481759076A077B0778F429969FAD299777
:1000A00023969FAF23972A967FAC2A972B96FFAD76
:1000B0002B972C96EFAD2C9723968FAD2397972DEA
:1000C000AF2FBE2F80179107A207B30710F4D901F5
:1000D000C8010AA91BA92CA93DA980179107A2074D
:1000E000B30710F4D901C80128E60BA11CA1209F79
:1000F000F001219FF00D1124EE51FB4E85A396A334
:10010000A7A3B0A70697A105B10508F4A0C5DF0114
:10011000AE59BF4F8091540B9091550B8D939C938A
:1001200061A6452B462B472B09F05F9888E60BA16B
:100130001CA1809FF001819FF00D1124EE51FB4E18
:10014000818D928DA38DB48D892B8A2B8B2B11F0F1
:100150008A98479888E60BA11CA1809FF001819F97
:10016000F00D1124EE51FB4E858D968DA78DB0A11B
:10017000892B8A2B8B2B31F0809108018170809321
:10018000060147982AA93BA94CA95DA9232B242B3A
:10019000252B09F465C580912F06882319F081501D
:1001A00080932F06611004C0129880E280932F067E
:1001B0006090260670902706009128061091290667
:1001C0009301A80169A579A98EA99AAD0E943DF471
:1001D00087FF04C069A679AA0EAB1AAFC501B401A6
:1001E0000E9443F42091CE143091CF144091D0144A
:1001F0005091D1140E94A2F426966CAF7DAF8EAFC1
:100200009FAF2697698B7A8B8B8B9C8BC201B10138
:100210000E9443F42091D2143091D3144091D4140D
:100220005091D5140E94A2F42B013C016D8B7E8B62
:100230008F8B988F6DA17EA18FA198A50E9443F40A
:100240002091D6143091D7144091D8145091D914DC
:100250000E94A2F44B015C01698F7A8F8B8F9C8F77
:100260002091DA143091DB144091DC145091DD14AC
:10027000C701B6010E94A2F46B017C016D8F7E8FD5
:100280008F8F98A388E60BA11CA1809FF001819F0E
:10029000F00D1124EE51FB4E258936894789508D8A
:1002A0002DA33EA34FA358A7263031054105510584
:1002B00008F4DFC42896AEADBFAD2897CD90DD9091
:1002C000ED90FC9020E030E0A901C701B6010E944A
:1002D0003DF48111EDC426962CAD3DAD4EAD5FAD24
:1002E0002697CA01B9010E94A2F46B017C01A30107
:1002F0009201C301B2010E94A2F49B01AC01C701AB
:10030000B6010E94BAF86B017C01A5019401C501F8
:10031000B4010E94A2F49B01AC01C701B6010E9486
:10032000BAF80E9425FB28E60BA11CA1209FF00132
:10033000219FF00D1124EE51FB4E6587768787874C
:10034000908B88E60BA11CA1809FF001819FF00D8E
:100350001124EE51FB4E4584568467847088A301B6
:10036000920160E070E080E89FE30E9496F9649655
:100370006CAF7DAF8EAF9FAF649729A539A94EA909
:100380005AAD0E94A2F44B015C018091650D9091E1
:10039000630D891B8F7027968FAF2797A501940156
:1003A00060E074E284E799E40E9496F90E94EBFA17
:1003B0006B017C0127968FAD27978250863008F419
:1003C00086C4A5019401C301B2010E94A2F49B015D
:1003D000AC010E94A2F468966CAF7DAF8EAF9FAF68
:1003E000689788E6ABA1BCA18A9F80018B9F100D06
:1003F00011240E511B4E68962CAD3DAD4EAD5FAD38
:100400006897D80111962D933D934D935C93149763
:1004100095962D913D914D915C9198972EAB3FAB68
:1004200048AF59AFCA01B9010E9441F46AAF7BAF2E
:100430008CAF9DAF9B01AC01C501B4010E94A2F439
:100440000E9480F90E9403FAA8966CAF7DAF8EAF30
:100450009FAFA897F801EE5AFF4F608371838283A4
:1004600093838E010F5E1F4F2A961FAF0EAF2A9700
:100470000051110924961FAF0EAF24970EE016E02D
:10048000AC961FAF0EAFAC978E010F5D1F4F1AA336
:1004900009A324960EAD1FAD2497AA961FAF0EAFE9
:1004A000AA97312C212C10E819A70FE309AB2A9643
:1004B000AEADBFAD2A972D913D914D915D912A969C
:1004C000BFAFAEAF2A97C501B4010E94A2F46B0181
:1004D0007C01AA96EEADFFADAA97619371938193CB
:1004E0009193AA96FFAFEEAFAA9720E030E0A90162
:1004F0000E94E0FA87FF04C0F7FAF094F7F8F0944E
:10050000AC96AEADBFADAC974D905D906D907D90CB
:10051000AC96BFAFAEAFAC97A7019601C301B201D5
:100520000E943DF487FD0DC409A11AA12A962EADA3
:100530003FAD2A970217130709F0B9CF20E030E04A
:1005400040E85FE3632D722D89A599A90E943DF4CF
:1005500087FF58C07E0131E1E30EF11C24960EADF9
:100560001FAD2497232D322D49A559A9D8016D918E
:100570007D918D919C910E94A2F4F80161937193F9
:10058000819391938F01EE16FF0661F728E60BA188
:100590001CA1209FC001219F900D11249C012E5170
:1005A0003B4E790189010E5A1F4FA8966CAD7DAD67
:1005B0008EAD9FADA8970E9441F4232D322D49A501
:1005C00059A90E94A2F40E9403FAD8016D937D9369
:1005D0008D939C931397232D322D49A559A9632DF3
:1005E000722D89A599A90E94A2F468962CAD3DAD03
:1005F0004EAD5FAD68970E94A2F4F70161837283EC
:10060000838394832AAD3BAD4CAD5DAD64966CADF8
:100610007DAD8EAD9FAD64970E94A2F469A77AA7C5
:100620008BA79CA70DA11EA12FA138A5012B022BE2
:10063000032B09F09EC388E62BA13CA1829F800179
:10064000839F100D11240E511B4EF801818D928D48
:10065000A38DB48D892B8A2B8B2B09F08AC3858DB2
:10066000968DA78DB0A1892B8A2B8B2B09F081C386
:100670002091F81B3091F91B4091FA1B5091FB1B04
:1006800069A57AA58BA59CA50E94A2F40E9480F979
:100690000E9403FA2B013C01F801E95BFF4F108235
:1006A00088E62BA13CA1829F8001839F100D11241D
:1006B0000E511B4EF801E25AFF4F40825182628276
:1006C0007382C301B2010E9441F429A53AA54BA54A
:1006D0005CA50E9496F96AAF7BAF8CAF9DAFD80145
:1006E00051966D937D938D939C935497F801E95B9C
:1006F000FF4F8081882381F17801B8E4EB0EF11C73
:1007000037962091020630910306409104065091DD
:10071000050660817181828193810E94A2F42AADD5
:100720003BAD4CAD5DAD0E94A2F42091381C3091E0
:10073000391C40913A1C50913B1C0E94A2F49B0131
:10074000AC0160E074E284EF99E40E9496F90E94A3
:1007500003FAF7017183608388E60BA11CA1809FD7
:10076000F001819FF00D1124EE51FB4E2181328169
:10077000438154812C962CAF3DAF4EAF5FAF2C9789
:10078000CA01B9010E9425FB362E272E8C0142EFAB
:1007900055E062965FAF4EAF62973E0151E1650E44
:1007A000711C82EF95E09FAB8EAB24964EAC5FAC94
:1007B00024973DA62DA209A719AB1AAAD201CD9064
:1007C000DD90ED90FD902D0120E030E0A901C70102
:1007D000B6010E94E0FA87FF04C0F7FAF094F7F838
:1007E000F094EEA9FFA981909190A190B190FFABF8
:1007F000EEABA7019601C501B4010E943DF487FD4F
:10080000D8C564147504D1F627965FAD2797552394
:1008100009F448C6C090670DD090680DE090690D4E
:10082000F0906A0D2DEB37E346E855E3C701B601BA
:100830000E943DF487FD36C6C701B6010E9425FB24
:100840006B017C019B01AC01632D722DC8010E94DC
:100850003DF487FD03C03C2C2D2C87019601A70198
:10086000632D722DC8010E9496F968966CAF7DAF1A
:100870008EAF9FAF68978BE69DE028969FAF8EAFB7
:10088000289720E030E040E85FE32AAB3BAB4CAB7D
:100890005DAB1EAA2896AEADBFAD28972D913D91B8
:1008A0004D915D912896BFAFAEAF289768966CAD1D
:1008B0007DAD8EAD9FAD68970E94A2F44B015C01A7
:1008C0002496EEADFFAD2497C190D190E190F190C8
:1008D0002496FFAFEEAF2497FEA9FF2391F02AA93B
:1008E0003BA94CA95DA90E94A2F44B015C012AA975
:1008F0003BA94CA95DA9C701B6010E94A2F46B01F6
:100900007C01A7019601C501B4010E94E0FA20E034
:1009100030E0A90118160CF092C5C701B6010E947B
:10092000E0FA18160CF486C520E030E0A901C501F4
:10093000B4010E943DF487FD7DC52601370177FA99
:10094000709477F87094A3019201C501B4010E94DC
:10095000E0FA181614F4240135016296AEADBFAD6D
:100960006297CD90DD90ED90FD906296BFAFAEAFF7
:100970006297A3019201C701B6010E943DF487FF6F
:1009800015C0A3019201C701B6010E9496F99B010F
:10099000AC016AA97BA98CA99DA90E94A2F46AABAB
:1009A0007BAB8CAB9DABBEA9BF5FBEABEBE7FDE005
:1009B00028962EAD3FAD2897E217F30709F06ACFCE
:1009C0003EA9332361F02AA93BA94CA95DA9632D57
:1009D000722DC8010E94A2F4362E272E8C0124EA23
:1009E00030E74DE75FE3632D722DC8010E94A2F44A
:1009F0006B017C0120912B0630912C0640912D0635
:100A000050912E060E943DF487FD42C58DA59DA103
:100A1000A9A5B9A980932B0690932C06A0932D0627
:100A2000B0932E0628E64BA15CA1249FC001259F10
:100A3000900D1124DC01AE51BB4E7D01232D322DD2
:100A4000A801632D722DC8010E94A2F4F7016187ED
:100A50007287838794876AAD7BAD8CAD9DAD9058CE
:100A60009B01AC010E94BAF8D7011D962D913D91D2
:100A70004D915C9150970E94A2F49B01AC016BE0F8
:100A800077ED83E29BE30E94B9F89B01AC018BE018
:100A900097EDA3E2BBE3F70185839683A783B08735
:100AA00010812C966CAD7DAD8EAD9FAD2C970E94C4
:100AB0003DF418160CF4FBC483E0182B88E62BA138
:100AC0003CA1829FF001839FF00D1124EE51FB4E5B
:100AD000108380E1FE013196ABE6BDE001900D92FE
:100AE0008A95E1F72C968CAD9DADAEADBFAD2C9740
:100AF0008093670D9093680DA093690DB0936A0D74
:100B0000E0960CAD1DAD2EAD3FADE09700938B0D83
:100B100010938C0D20938D0D30938E0DE4962CAD9B
:100B20003DAD4EAD5FADE49720938F0D3093900DAA
:100B30004093910D5093920DE8968CAD9DADAEAD66
:100B4000BFADE8978093930D9093940DA093950D6E
:100B5000B093960D60960CAD1DAD2EAD3FAD609778
:100B60000093970D1093980D2093990D30939A0D43
:100B70006C962CAD3DAD4EAD5FAD6C9720937B0D6B
:100B800030937C0D40937D0D50937E0DA0968CADDF
:100B90009DADAEADBFADA09780937F0D9093800DBE
:100BA000A093810DB093820DA4960CAD1DAD2EAD1A
:100BB0003FADA4970093830D1093840D2093850D72
:100BC0003093860D22962CAD3DAD4EAD5FAD229794
:100BD0002093870D3093880D4093890D50938A0D93
:100BE0009091650D8091660D981303C084E6809303
:100BF000620DE9968FADE9978F5F8F708093650DD9
:100C00008091650D9091640D81508F70891351C44E
:100C10001091660D1BA30091650D0DA728E61BA181
:100C20000DA51013D1C4812C912CA12CB12C1DA287
:100C300019A619AA1EAE212C312C00E010E02DA51A
:100C40003BA12313CEC42114310409F07FC5809148
:100C50006F00826080936F0081E0ECC680E0EAC69E
:100C600060902206709023060091240610912506BC
:100C7000A7CA818D928DA38DB48D0697A105B1056C
:100C800008F018CB858D968DA78DB0A10697A1058C
:100C9000B10508F00FCB20E030E0A901C701B60193
:100CA0000E94E0FA87FF04C0F7FAF094F7F8F09496
:100CB00088E60BA11CA1809FF001819FF00D1124FB
:100CC000EE51FB4EC586D686E786F08A3ACB8091F8
:100CD0001E0690911F06A0912006B0912106C8160D
:100CE000D906EA06FB0608F06CCB8C199D09AE0903
:100CF000BF09BC01CD01660F771F881F991F27967A
:100D00004FAD2797042F10E020E030E0A9019801B3
:100D10000E945CF8CA01B9010E9441F40E94EBFAFA
:100D20006C0D7D1D8E1D9F1D0E9441F49B01AC0129
:100D300060E074E284E799E40E9496F94B015C015B
:100D400040CBA7019601C301B2010E9496F97B0135
:100D50008C019B01AC01632D722D89A599A90E947C
:100D6000E0FA18160CF0E0CB3E2C2F2C09A719AB9B
:100D7000DBCB0AA91BA92CA93DA9012B022B032B14
:100D800049F020910A0630910B0640910C065091D3
:100D90000D0608C02091060630910706409108060E
:100DA0005091090669A57AA58BA59CA50E94A2F47D
:100DB0000E9480F90E9403FA2B013C012AA93BA959
:100DC0004CA95DA9232B242B252BC9F020E030E072
:100DD000A90160910206709103068091040690912A
:100DE00005060E943DF4882351F081E00DA51EA563
:100DF0002FA538A910161106120613060CF080E074
:100E000098E62BA13CA1929F8001939F100D112485
:100E10000E511B4E180137E4230E311CD1018C9367
:100E2000882309F4B3C020917B0D30917C0D409153
:100E30007D0D50917E0D6C966CAD7DAD8EAD9FADF0
:100E40006C970E94B9F86DA77EA78FA798AB2091E9
:100E50007F0D3091800D4091810D5091820DA096B3
:100E60006CAD7DAD8EAD9FADA0970E94B9F84B01E2
:100E70005C012091830D3091840D4091850D50913E
:100E8000860DA4966CAD7DAD8EAD9FADA4970E94EE
:100E9000B9F86B017C012DA53EA54FA558A9CA0143
:100EA000B9010E94A2F46DA77EA78FA798ABA501F8
:100EB0009401C501B4010E94A2F49B01AC016DA58F
:100EC0007EA58FA598A90E94BAF84B015C01A701E5
:100ED0009601C701B6010E94A2F49B01AC01C501B5
:100EE000B4010E94BAF80E9425FB6B017C0120919D
:100EF000870D3091880D4091890D50918A0D229671
:100F00006CAD7DAD8EAD9FAD22970E94B9F8A70163
:100F100096010E9496F96B017C01F801E25BFF4F9C
:100F2000608371838283938320E030E040E450E467
:100F30000E94E0FA18161CF4F101108227C02091DB
:100F40000206309103064091040650910506C70140
:100F5000B6010E94A2F49B01AC016091FE05709164
:100F6000FF0580910006909101060E9496F929A53F
:100F70003AA54BA55CA50E94A2F40E9403FA641551
:100F800075058605970510F42B013C018091AA1484
:100F90009091AB14A091AC14B091AD140EA91FA9FF
:100FA00028AD39AD80179107A207B30708F4DFC059
:100FB0002DA13EA14FA158A5232B242B252B41F178
:100FC0006091AE147091AF148091B0149091B114EF
:100FD0006415750586059705D8F42EA93FA948AD77
:100FE00059AD0E944DF86B017C012DA13EA14FA18E
:100FF00058A5C301B2010E944DF8C616D706E806EF
:10100000F90630F4C701B6010E945CF829013A01E3
:1010100088E60BA11CA1809FF001819FF00D112497
:10102000EE51FB4EC18CD28CE38CF48CC114D104F4
:10103000E104F10431F16091B2147091B314809124
:10104000B4149091B5146415750586059705C8F418
:101050002EA93FA948AD59AD0E944DF84B015C0146
:10106000A7019601C301B2010E944DF886169706AA
:10107000A806B90630F4C501B4010E945CF8290144
:101080003A0188E60BA11CA1809FF001819FF00D21
:101090001124EE51FB4EC58CD68CE78CF0A0C11408
:1010A000D104E104F10431F16091B6147091B714E8
:1010B0008091B8149091B91464157505860597054B
:1010C000C8F42EA93FA948AD59AD0E944DF84B0177
:1010D0005C01A7019601C301B2010E944DF886167A
:1010E0009706A806B90630F4C501B4010E945CF861
:1010F00029013A0188E60BA11CA1809FF001819F84
:10110000F00D1124EE51FB4EC1A0D2A0E3A0F4A03B
:10111000C114D104E104F10409F4C2CA6091BA1403
:101120007091BB148091BC149091BD146415750529
:101130008605970508F0B4CA2EA93FA948AD59AD58
:101140000E944DF84B015C01A7019601C301B20159
:101150000E944DF886169706A806B90608F0A0CAA0
:10116000C501B4010E945CF829013A0199CA2DA178
:101170003EA14FA158A5232B242B252BC9F160910B
:10118000AE147091AF148091B0149091B1146415A5
:1011900075058605970560F50E9441F42AAD3BADC3
:1011A0004CAD5DAD0E94A2F46B017C016DA17EA1EE
:1011B0008FA198A50E9441F44B015C01C301B201CB
:1011C0000E9441F4A50194010E94A2F49B01AC018C
:1011D000C701B6010E943DF487FF0AC0A501940132
:1011E000C701B6010E9496F90E9403FA2B013C0147
:1011F00088E60BA11CA1809FF001819FF00D1124B6
:10120000EE51FB4E818C928CA38CB48C8114910492
:10121000A104B104B9F16091B2147091B31480913A
:10122000B4149091B514641575058605970550F5AD
:101230000E9441F42AAD3BAD4CAD5DAD0E94A2F4DD
:101240006B017C01C501B4010E9441F44B015C01BA
:10125000C301B2010E9441F4A50194010E94A2F4CD
:101260009B01AC01C701B6010E943DF487FF0AC093
:10127000A5019401C701B6010E9496F90E9403FAE4
:101280002B013C0188E60BA11CA1809FF001819FEE
:10129000F00D1124EE51FB4E858C968CA78CB0A0DE
:1012A00081149104A104B104B9F16091B614709154
:1012B000B7148091B8149091B9146415750586051A
:1012C000970550F50E9441F42AAD3BAD4CAD5DADA4
:1012D0000E94A2F46B017C01C501B4010E9441F49B
:1012E0004B015C01C301B2010E9441F4A5019401CC
:1012F0000E94A2F49B01AC01C701B6010E943DF41B
:1013000087FF0AC0A5019401C701B6010E9496F9A2
:101310000E9403FA2B013C0188E60BA11CA1809FCF
:10132000F001819FF00D1124EE51FB4EC1A0D2A01F
:10133000E3A0F4A0C114D104E104F10409F4B0C99C
:101340006091BA147091BB148091BC149091BD143B
:10135000641575058605970508F0A2C90E9441F439
:101360002AAD3BAD4CAD5DAD0E94A2F44B015C01DA
:10137000C701B6010E9441F46B017C01C301B201B7
:101380000E9441F4A70196010E94A2F49B01AC01C6
:10139000C501B4010E943DF487FF82C9A7019601EF
:1013A000C501B4010E9496F90E9403FA2B013C0189
:1013B00077C9FAA9FF2331F1A5019401632D722D9C
:1013C000C8010E94A2F44B015C012DA53DA149A5D5
:1013D00059A9C701B6010E94A2F49B01AC01C50145
:1013E000B4010E943DF487FF22C0A7019601C50108
:1013F000B4010E9496F96DA77DA389A799AB21E05E
:101400002AABFFC9A7019601C501B4010E9496F954
:101410009B01AC016DA57DA189A599A90E94A2F4AB
:101420006DA77DA389A799AB31E03AABEAC941E04A
:101430004AABE7C9A7019601C501B40113C0C701B2
:10144000B6010E943DF487FD09C020E030E0A9010B
:10145000C501B4010E94E0FA18164CF4A5019401EC
:10146000C701B6010E94B9F82B013C0176CA2401DC
:10147000350177FA709477F87094A3019201C7014F
:10148000B6010E943DF487FD68CA2601370165CA8E
:101490002DA53DA149A559A9C701B6010E943DF45A
:1014A00087FFB4CA3DA42DA009A519A9AFCA81E040
:1014B00004CBF090650D8FEF8F0D8F708BA3B090E4
:1014C000640D8091650DB81609F454C0C12CD12C5F
:1014D0000BA10B1509F44EC0602E712C28E6269D39
:1014E0008001279D100D11240E511B4ED8018C91A7
:1014F00083FD2BC00EAF1AAB0115110541F11996F2
:10150000BC91BDA7F801F285FDA3D8011B96BC9143
:10151000B9A7F801F485F9ABD80115962D903D9047
:101520004D905C901897A20191016DA57DA189A5B0
:101530009F2F0E943DF4811186C1C114D10439F05E
:10154000F601808180FD7FC102C0CEAEDAAA8BA1F8
:1015500081508F708BA38091640D8B1103C0CEAC32
:10156000DAA8B6CF0BA10B1529F081E08B0D8F7097
:10157000B82EF1CF1091640D1BA3C12CD12C8091FA
:10158000650D0BA1801709F443CB802E912C28E622
:10159000289D8001299D100D11240E511B4ED8014C
:1015A0008C9183FD0AC05801C114D10439F0C601E1
:1015B0000E940CE6811102C0C5C156018BA18F5F4C
:1015C0008F708BA36501DBCF802F81508F70289F98
:1015D000F0011124EE51FB4E908193FF24CB8DA797
:1015E0001ECB48E6439FC0011124DC01AE51BB4E27
:1015F0001D018C9183FD19C015966D917D918D9182
:101600009C9118970E9425FBF62EE72ED82EC92E06
:101610000115110509F48CC0F801808180FD0AC014
:10162000D1018C9180FD06C083C0FDA0E9A4D9A89A
:10163000CEAC83C0F801808181608083C8010E94A4
:101640000CE6811171C0F8016181728183819481FE
:101650000E9425FB2B013C019B01AC0160E070E086
:1016600080E89FE30E9496F94B015C019B01AC016D
:101670006F2D7E2D8D2D9C2D0E94A2F469837A837F
:101680008B839C832DA139A549A95EADC501B40109
:101690000E94A2F4698B7A8B8B8B9C8BAE014F5F7F
:1016A0005F4FBE016F5E7F4FC8010E9460C7F801A7
:1016B000E95BFF4F80818823B9F1209102063091C8
:1016C00003064091040650910506379660817181AA
:1016D000828193810E94A2F42091381C3091391CA0
:1016E00040913A1C50913B1C0E94A2F44B015C01BA
:1016F0009B01AC01C301B2010E94A2F40E9403FA53
:10170000F801E65BFF4F71836083A50194016F2DA3
:101710007E2D8D2D9C2D0E94A2F40E9403FAF801CB
:10172000E45BFF4F71836083D8018C918E7F8C9333
:101730008F2C9E2CAD2CBC2C81018BA18F5F8F70C8
:101740008BA3FDA2E9A6D9AACEAE79CAF101808108
:1017500081608083C8010E940CE681116FC0D101B5
:1017600011966D917D918D919C9114970E9425FB0E
:101770006B017C019B01AC0160E070E080E89FE3BD
:101780000E9496F92B013C012DEC3CEC4CE45DE30E
:101790000E94A2F469837A838B839C839401A501C0
:1017A000C301B2010E94A2F4698B7A8B8B8B9C8B54
:1017B000AE014F5F5F4FBE016F5E7F4FC1010E9460
:1017C00060C7F101E95BFF4F80818823B9F1209167
:1017D00002063091030640910406509105063796A3
:1017E00060817181828193810E94A2F42091381CD2
:1017F0003091391C40913A1C50913B1C0E94A2F43C
:101800004B015C019B01AC01C701B6010E94A2F42F
:101810000E9403FAF101E65BFF4F718360832DECB8
:101820003CEC4CE45DE3C501B4010E94A2F40E94CB
:1018300003FAF101E45BFF4F71836083F101808162
:101840008E7F808304CA28E6269DF001279DF00D37
:101850001124EE51FB4E808181FD43C0C114D1049F
:1018600041F0D6011596CD90DD90ED90FC90189743
:1018700008C08BE0C82E87EDD82E83E2E82E8BE3DC
:10188000F82EB8E6B69DF001B79DF00D1124EE518B
:10189000FB4E81899289A389B489BC01CD019058FE
:1018A0009B01AC010E94BAF8F80125853685478571
:1018B00050890E94A2F49B01AC01C701B6010E94AD
:1018C000B9F8E62E872E982EA92E262F372F482FCF
:1018D000592F6DA57DA189A599A90E943DF487FF87
:1018E00004C0EDA48DA099A4A9A82E2D382D492DB2
:1018F0005A2DC201B1010E943DF4882309F427CE7C
:10190000F8E6F69DC001F79D900D11249C012E5123
:101910003B4E6901D9018C9181608C93C8010E9472
:101920000CE6882329F0F60180818E7F80830FCE1C
:101930008E2D982DA92DBA2DF60185839683A78328
:10194000B08705CED6018C9181FD52C0D601159687
:101950002D913D914D915C9118972DA73EA74FA7D2
:1019600058AB1501B5E02B0E311CF80145805680AF
:1019700067807084A30192016DA57EA58FA598A9AB
:101980000E943DF487FF34C0F60181899289A389C2
:10199000B489BC01CD0190589B01AC010E94BAF8FA
:1019A000D6011D962D913D914D915C9150970E94CD
:1019B000A2F49B01AC016DA57EA58FA598A90E94FC
:1019C000B9F86B017C019B01AC01C301B2010E941B
:1019D000E0FA18166CF4D8018C9181608C93C501E3
:1019E0000E940CE68823E1F0F80180818E7F8083DD
:1019F00018E6189DF001199DF00D1124EE51FB4ED3
:101A000021853285438554856581768187819085DE
:101A10000E943DF48111D2CD0BA10093640DCECD77
:101A2000D101CD92DD92ED92FC9213970BA1009320
:101A3000640DDECFC858DF4F0FB6F894DEBF0FBE7F
:101A4000CDBFDF91CF911F910F91FF90EF90DF906D
:101A5000CF90BF90AF909F908F907F906F905F904E
:101A60004F903F902F9008958091650D9091660D55
:101A7000891B8F708F3021F480E00E946DA4F4CF19
:101A80008091650D8F5F8F70E091650D98E69E9F48
:101A9000F0011124EE51FB4EDF011D929A95E9F7FA
:101AA00098E0908340918B0D50918C0D60918D0D3D
:101AB00070918E0D458B568B678B708F40918F0D7B
:101AC0005091900D6091910D7091920D418F528FB8
:101AD000638F748F4091930D5091940D6091950D8B
:101AE0007091960D458F568F678F70A34091970D1B
:101AF0005091980D6091990D70919A0D41A352A348
:101B000063A374A32091650D9091660D291303C002
:101B100094E69093620D8093650D80916F008260D2
:101B200080936F0008959091650D8091660D9813D4
:101B300006C080918E0590918F05892B21F080E061
:101B40000E946DA4F0CF0895CF93DF938B3D924018
:101B5000B1F0EFEEF6E28491EF012196882321F0B7
:101B60000E94009DFE01F7CFECE5F1E28491EF01C8
:101B70002196882331F00E94009DFE01F7CF80E07E
:101B800001C081E0DF91CF9108952F923F924F9253
:101B90005F926F927F928F929F92AF92BF92CF92FD
:101BA000DF92EF92FF920F931F93CF93DF93CDB706
:101BB000DEB7C757D1090FB6F894DEBF0FBECDBF51
:101BC0002DB63EB6A7961FAE1EAEA79784E690E050
:101BD000A9969FAF8EAFA99701E09E012B593F4F69
:101BE00044E050E0BE01655A7F4FCE0189599F4FB6
:101BF0000E9401E09E012B593F4F42E050E0BE01A0
:101C000067597F4FCE0189599F4F0E9401E043E001
